:10B6E800414952434F54454300405053332E35305F
:10B6F80040465245004143435500532F4E21464191
:10B70800494C555245005245454E54455221532FF8
:10B718004E00434F4E5441435420414952434F54E5
:10B7280045430047505300403244400040334440B2
:10B738000046494E40564F4C214D454E55000A167D
:10B74800000180000300007E0000FE00001E0000D3
:10B75800360003E60001C4000000000FFFE020529D
:10B7680045434840534154532000204750534056C6
:10B77800414C49442000404B455932004543522032
:10B788005045525300434620454352414E004341E1
:10B7980052544520202000544845524D49515500E7
:10B7A800564152494F202020004241524F475241B2
:10B7B8004D00524F5554455320200050524F434896
:10B7C800452020005741595054532020004D4152E4
:10B7D80051554553200046494E2020202020002066
:10B7E80020202144495321202020204D4F5900205A
:10B7F8005452414345215649532000205452414355
:10B808004521494E5620004D41524B002044495293
:10B81800205452414345200020444952204E4F5263
:10B8280044202000215245544F55520153454C4560
:10B8380043405254450143414C455220414C540128
:10B84800564F4C53202020206869015741595054C5
:10B85800532020686901524F555445532020686988
:10B868000141495253504143456869015245474C8B
:10B8780041474553686900414343454C45522E684A
:10B88800690043414C455220414C542000414C54DE
:10B89800404241524F4D202000414C5420475053C4
:10B8A80020202000514E482020202040214850418F
:10B8B80000464C00435420424F52442056494445C8
:10B8C80020003E215245544F555200215245544FB5
:10B8D80055520152454C49524501454E564F59451E
:10B8E8000145464641434500215245544F555201B2
:10B8F80020555342204F4E4C592001544E4320317D
:10B90800232035374B01544E4320312320392E361E
:10B918000101505743403130234035374B015057D0
:10B9280043403130234031394B01014D58504031AB
:10B9380030234035374B014D5850203423203537BC
:10B948004B014D58502031232035374B014D58506D
:10B95800403130234031394B014D5850203123209C
:10B9680031394B00215245544F55520143524545F8
:10B97800522020205750014348414E4745522057F6
:10B988005001454646414345522057500101434F17
:10B998004D3A015245434556202020575001454E07
:10B9A800564F59455220575001454E564054534022
:10B9B800575053200101444953542057502D575094
:10B9C80001454646215453215750532000444953BA
:10B9D8005421564552530053415556202000504F8C
:10B9E800532041435455454C4C4500534155564509
:10B9F8005220202020002053544F524521575054A4
:10BA080020002046554C4C200040454646414345C1
:10BA18005200534552200049524441005553422098
:10BA28000055534220004C4953544500454E56207A
:10BA38000020455252205452414E534D49535320F1
:10BA48002000215245544F55520153454C40524F06
:0DBA5800555445014E4F555645415520505F
:10BA650054014348414E47452052544501494E56DD
:10BA750045525320525445014546462050542052C4
:10BA850054450145464641434520525445014359D5
:10BA95004C2052414449555301434F4D3A015245BB
:10BAA500434556202052544501454E564F592020B6
:10BAB50052544501434845434B2052540053454C8D
:10BAC50021524F555445004E4F5556004E4C452179
:10BAD500504F532120200040494E56455253455260
:10BAE50000494E5645525300214045464640575061
:10BAF50053200021404546462052544500504153AD
:10BB050020564944452020002140454E5640525478
:10BB150045200020205241444955530021524554A7
:10BB25004F5552014348415247452043545201560F
:10BB35004F495240435452014546464054534043B1
:10BB450054520101434F4D3A015245434556204356
:10BB5500545201454E5620204354522000564F4919
:10BB65005220435452004445504C414345520044F1
:10BB750045504C41434552204100454348202058FB
:10BB85002F5920205245544F5552004546462044D2
:10BB95004953200043454E54204F55490043454ED7
:10BBA50054204E4F4E00202020454348454C00442C
:10BBB500495354204B4D0044495354204E4D0021C8
:10BBC5005245544F555201564152494F2020206845
:10BBD5006901434F4E4620584320686901434F4E43
:10BBE500462052544568690147454E4552414C200F
:10BBF500686901434F4E462045435268690101017A
:10BC050043462053494D504C01434F4E4620555312
:10BC1500494E4501564F4C20544553542020002190
:10BC25005245544F555201544F4E204445534301FC
:10BC350054582044212D014D4F4420444553430180
:10BC4500494E5620444553430156415220544340E2
:10BC55002020402301564F4C554D45015641524930
:10BC65004F204E554C2001544F4E414C49544501EF
:10BC7500504552494F4445015641522041564020B6
:10BC8500304023014E4554544F2D015445535445DE
:10BC95005220534F4E00544F4E20444553432000ED
:10BCA50053494E4B54214F4646004E4F4E20445566
:10BCB500414C2020200043414C4942204455414CF1
:10BCC5000058435420535441424C45403130404D77
:10BCD5004E004156414E542043414C494252414742
:10BCE5004500215245544F55520154524143452078
:10BCF50020014155544F43454E5401014D4F592F95
:10BD05004449535401415050524F434845014C2F2B
:10BD15004401014F52492056542054014F524920A5
:10BD25004354205401574159505421425247002150
:10BD35005245544F555201444550415254202020FC
:10BD450001444542555401504153202020203A01D9
:10BD55004D554C5449504C45014445524E490143BB
:10BD6500594C53494740202040230153454C4052EC
:10BD750054452020010101015220434C014F5249F5
:10BD850020434C205400215245544F555201015532
:10BD95004E495401434C49434B40302C402023012C
:10BDA500434F4E5452415354014E4D454121313874
:10BDB5003301494D50454C4C455201494D502D4399
:10BDC500414C01432D564152494F015445432020D2
:0DBDD5002040303040250141004E4F2041FC
:10BDE2004750532F464C00414C54492D4750532045
:10BDF2002000464C47542D4C4556454C0041475077
:10BE020053203C3E20464C002057414954004E4F9F
:10BE120020464C49474854004045584954204C4F0D
:10BE220047403F40004D4D2E59590020606869003F
:10BE32003C2D20202020202D3E2020202053454C28
:10BE4200003C2D20202020202D3E20202045584936
:10BE520054003C52454320205245433E202020536B
:10BE6200454C00522D4F464600202052454300418A
:10BE72004343454C455241542E00472D554E49549B
:10BE82005300215245544F5552015245434D4F44A0
:10BE920045202058015245432E2031352F2301528F
:10BEA20045432E2036302F230152504C41592F53F7
:10BEB200454E440145464641434552405453014391
:10BEC2004F4D3A00205C2020202053454E44004034
:10BED2005750204558495354414E54202020204069
:10BEE20000574159504F494E5400205245544F5526
:10BEF2005220210052454345564F4952004C494277
:10BF02005220003C2D204C495354202D3E202045E8
:10BF12005849540053454C004E4558540050524F16
:10BF22004348205450005052454345205450004548
:10BF32004646205345474D0045464620544F5554EA
:10BF42000041525220202020202020200020415257
:10BF52005200455252204750532020004D454D4F2C
:10BF620049524500524F5554450050524F4348459F
:10BF7200004C495354450045544500414C5440300F
:10BF82000052544520564944452020002054524F27
:10BF92005040575053200053454C404C4953544550
:10BFA200002053454C40575040212000214052452B
:10BFB200434556402020002020404F204B40202067
:10BFC20021004F4B00564152004649580047415408
:10BFD200452158004C474E452044455020200053EF
:10BFE2005443594C200040415252005450200040CA
:10BFF2006A40494E20004067404F55540020455248
:10C00200524555522021002046494E20202000450D
:10C01200444954004F405540490045444954204E3C
:10C022004C4520204D454D4F4952004E4558542015
:10C0320053454C4543542045584954005843542DC8
:10C04200464C4947485420005553454400454E54F8
:10C05200455220004D4D2E4D4D4D20004D4D275344
:10C06200532E530057475321383400204055405433
:10C07200404D402000554054404D0020555443202F
:10C08200004C4F43414C00535749535347440041DE
:10C092004C540053554940580041564740203040C7
:10C0A2002300353030003136343000205D2031300D
:10C0B200404B632F70005D2020203140632F23000E
:10C0C200205D202035404B5453005D2032303040FB
:10C0D20046504D00406340204B63004654204B6362
:10C0E20000406340204E4D004654204E4D004D2FDF
:10C0F20053003230305E003530305E003122003283
:10C102002200332200352200382200464C370046F6
:10C112004C313600464C333300464C3635004631FE
:10C12200303000463136300046323630005E252649
:10C1320040534F47005E25264054415300414C5422
:10C142000056415200225E2F24004B545300532FBD
:0DC152004E002224004B5400225E004E4D92
:10C15F0000302C3500312C3000322C3000302C3692
:10C16F0000312C3200322C3500332C3800372C356F
:10C17F0000403135004033300040363000544153D9
:10C18F004B00464C2D4441544500545000544F46EB
:10C19F00005354410046494E004C414E0053455404
:10C1AF00204F46465345540049534120484549477F
:10C1BF004854004155544F2D474F2000535441527E
:10C1CF00540020434845434B40414C4C005241449E
:10C1DF002044495354004053454C40484549474833
:10C1EF00543A00475053404241524F40414C4C004B
:0DC1FF0053494E4B40312D3221632F230058
:106F3B00304D2475A7049005C2E0F51CE0F51DE06B
:106F4B00F51EE0F51FE0F56DE0F56EE0F56FE0F591
:106F5B0054127AFD12753B2275C70375C6E475B9D9
:106F6B0001E5BCB48143127AFD1261158E628F6309
:106F7B007568F9756900127011203C2D203B2B129E
:106F8B00714612711A856D1C856E1D856F1E855499
:106F9B001F12707D203C12203243201D231271469C
:106FAB0012753BE532242850DC2212707D203CF90F
:106FBB00203DF6203205201DBD80EF301DB880EA44
:106FCB0012714612753B856D1C856E1D856F1E8576
:106FDB00541F12713012753B203DCE80991273698C
:106FEB00201D0D75531074001272CC203DBB808692
:106FFB00E553540FC553C4540F2035051271E1806E
:10700B00031272CC808BC23CD23B1270CDFD12703E
:10701B00CDFC1270CDC39573F565EC9574F564EDED
:10702B009575600504600A800EE56424E0501180BC
:10703B0006E564242040091270CD1270CD0270CD8C
:10704B001270CDFD1270CDFC1270CDC39576F56725
:10705B00EC9577F566ED9578600904600122E5669D
:10706B00F48002E5668562F0A474E025F04002C26C
:0D707B003B22C23C1270CDA2E7923DA2E67E
:10708800921DA2E592324026A2E492E592E692E7AA
:10709800FC1270CD2565F565EC3564F5641270CD8C
:1070A800FC1270CD2567F567EC3566F56622A2E41B
:1070B8009235540F79C6F71270CD09F7301D0512B5
:1070C80070CDF55322E5697023E5686030240440EB
:1070D8002CE56875F004A485F0C7F5C675B901E517
:1070E800BCB4811985BD68756902801E540370108F
:1070F80005C675B901E5BC056953690F22D23C2262
:10710800147004E5BD80F0147004E5BE80E9E5BFA5
:1071180080E575A7009006F6E56DF0A3E56EF0A38F
:10712800E56FF0A3E554F02275A7009006F6E0F5A8
:107138006DA3E0F56EA3E0F56FA3E0F55422E564D6
:10714800B2E7F56D85656EAB67E566FC30E707C3AA
:10715800E49BFBE49CFCAA62A963125E0FE566301F
:10716800E707C3E49DFDE49EFEEEB2E7F56F8D549C
:107178002275380C1273D212741DD553012275383A
:107188000C1273A3127413D55301227538001273AD
:0E719800BB1273E2D55301227538001273A3A7
:1071A6001273E2D55301227538031273D212744E4C
:1071B600D55301227538031273A3127444D55301B3
:1071C6002275380F1273BB127473D55301227538AA
:1071D6000F1273A3127473D55326229071E623738C
:1071E6008091807780688059804A803B802C801D02
:1071F600800E80DA80CB80BC80AD809E808F8080C0
:107206007538151273D2127495D553012275381537
:107216001273A312748AD55301227538091273BBEF
:1072260012745BD55301227538091273A312745B6D
:10723600D55301227538061273D2127405D553013F
:10724600227538061273A31273FAD55301227538C4
:10725600121273BB12742BD5530122753812127396
:10726600A312742BD5530122027179753815127346
:10727600D2127495D553012275380F1273A3127466
:1072860073D553012275380F1273BB127473D5531D
:1072960001227538031273A3127444D55301227563
:1072A60038031273D212744ED55301227538001268
:1072B60073A31273E2D55301227538001273BB1201
:1072C60073E2D55326229072D12373809E80A980C3
:1072D600B480BF80CA80D580E08010801B80268065
:1072E60031803C80478052805D806875380C12730F
:1072F600A3127413D553012275380C1273D212746B
:0E7306001DD55301227538121273A312742B79
:10731400D55301227538121273BB12742BD5530145
:10732400227538061273A31273FAD55301227538E5
:10733400061273D2127405D55301227538091273DB
:10734400A312745BD55301227538091273BB1274EE
:107354005BD55301227538151273A312748AD55361
:10736400012202727178C686040886037AED125DE2
:10737400CD78CAA60408A60378C686040886037ACC
:1073840062125DCD78CCA60408A60378C6860408EC
:1073940086037AB5125DCD78C8A60408A6032275C3
:1073A4001A6A751B0A78CA86180886191275E6784F
:1073B400CC86060886072278C88618088619E4F55C
:1073C4001AF51B1275E678C886060886072278C661
:1073D4008618088619751A00751B010275E6E51DE5
:1073E4002519F51DE51C3518F51CC3E51F9FF51F70
:1073F400E51E9EF51E22C3E51F9FF51FE51E9EF5A3
:107404001EC3E51D9519F51DE51C9518F51C22E50F
:107414001D2FF51DE51C3EF51CC3E51F9519F51F31
:10742400E51E9518F51E22C3E51D9FF51DE51C9E5E
:09743400F51CC3E51F9519F51FB5
:10743D00E51E9518F51E22E51F2FF51FE51E3EF5DD
:10744D001EE51D2519F51DE51C3518F51C22C3E596
:10745D001D9519F51DE51C9518F51CE51F2FF51F3C
:10746D00E51E3EF51E22E51D2FF51DE51C3EF51C06
:10747D00E51F2519F51FE51E3518F51E22C3E51D5F
:10748D009FF51DE51C9EF51CE51F2519F51FE51E35
:10749D003518F51E22E51A7009E51B70058C068D51
:1074AD000722ED851BF0A4A2F792D5ED851AF0A465
:1074BD00AEF0FFEC851BF0A4A2D53FEE35F0FF92A8
:1074CD00D5EC851AF0A42FFFE435F030D50104FE7C
:1074DD0022E4F51AF51BEF4E7003051B22EF65191B
:1074ED007006EE65187001227808C3EF33FFEE3396
:1074FD00FEEF9519F5F0EE95184003FEAFF0E51A85
:10750D0033F51AD8E5F4F51A751BFF7805C3EF337B
:10751D00FFEE33FEEF9519F5F0EE95184003FEAF33
:03752D00F0E51B6B
:1075300033F51BD8E5F4C403F51B22E51D9511E5D1
:107540001C9510500BE56E9511E56D9510500122BC
:10755000E51F9511E51E9510500BE5549511E56F4B
:107560009510500122E51D9513E51C9512400BE581
:107570006E9513E56D9512400122E51F9513E51EEA
:107580009512400BE5549513E56F95124001225377
:107590002CF8C3E51F9554FFE51E956FFE926050D1
:1075A00007C3E49FFFE49EFEC3E56E951DF519E554
:1075B0006D951CF5189261500BC3E49519F519E40B
:1075C0009518F518C3E5199FE5189E9262500AE5D3
:1075D00018CEF518E519CFF5191274DEE52C54070D
:1075E00075F003A4F538E5389075EC730276040263
:1075F000761802762602763E02765102766402768C
:107600007202768A851C16851D17C3E4951FF51531
:10761000E4951EF51402769D851C16851D17851EA2
:1076200014851F158077C3E4951DF517E4951CF5A7
:1076300016C3E4951FF515E4951EF514805FC3E4A9
:05764000951DF517E4A3
:10764500951CF516851E14851F15804CC3E4951FE2
:10765500F517E4951EF516851C14851D15803985CD
:107665001E16851F17851C14851D15802BC3E495D3
:107675001FF517E4951EF516C3E4951DF515E4955C
:107685001CF5148013851E16851F17C3E4951DF57B
:1076950015E4951CF5148000C3E5179513E51695BB
:1076A5001210D70122E5159513E514951210D7018F
:1076B50022E519F92517FFE518F83516FED3EF95DC
:1076C50011EE9510500122E5119517FDE51095165F
:1076D500FC402A4D60271274A2E5152FF515E51417
:1076E5003EF514E5159513E514951210D70122E51D
:1076F500199DF9E5189CF8851016851117E51729C8
:10770500FFE51638FEE5139FE5129E500BC3E51302
:107715009517F9E5129516F8E51A700AE51B700636
:10772500AA00AB018013E9851AF0A4E5F0FBE88512
:107735001AF0A42BFBE435F0FAE5152BFBE5143A1A
:06774500FAE5119BE510BE
:10774B009A10D70122EB9515FDEA9514FCC3E515AC
:10775B009511E514951010D717E5139BE5129A5068
:10776B0036E5139515FFE5129514FE127A1A80274C
:10777B00EB9511FFEA9510FEAA00C001127A1AD000
:10778B0003E5172BFBE5163AFAEB99F517EA98F593
:10779B0016851115851014C2D5E5466002D2D5AAFF
:1077AB0056E98AF0A4ABF0E88AF0A42B30D5047527
:1077BB00F00384F8700122E5172513FDE516351249
:1077CB00FCED8AF0A4ABF0EC8AF0A42B30D5047559
:1077DB00F00384FEE5152513FDE5143512FCED8A47
:1077EB00F0A4ABF0EC8AF0A42B30D50475F0038435
:1077FB00F9E5389078027302781A02782602782F0E
:10780B0002783802783E02784A027851027856C3E1
:10781B00743E9EFFC3743E99FE8032C3743E9EFF3E
:10782B00AE018029AF06C3743E99FE8020AF06AE31
:0D783B0001801AC3743E9EFEC3743E99FF87
:10784800800EC3743E99FF8007C3743E9EFEAF014D
:1078580008EF2437FFE51B7007E51A700CE8800E67
:10786800A2E7E51A50030460F488F0A4E5F060018B
:1078780004F923FA98FBC3E998C333F990788AE5A9
:1078880038730278A20278CF02790402793102793A
:107898005E02798B0279B80279E505A7800BEB3097
:1078A800E7032A8002291E1FFBEEC45403F583EE6A
:1078B8005408C42FF582EE5407243883F5F0E045C8
:1078C800F0F0D8DA05A72205A7800BEB30E7032AEA
:1078D8008002290E1FFBEEC45403F583EE5408C43E
:1078E8002FF582EE5407240B83F5F0E045F0F0D82D
:1078F800DA05A722804020100804020105A7800BA2
:10790800EB30E7032A8002291E0FFBEEC45403F56F
:1079180083EE5408C42FF582EE540724EC83F5F067
:10792800E045F0F0D8DA05A72205A7800BEB30E791
:05793800032A80022972
:10793D000E0FFBEEC45403F583EE5408C42FF582ED
:10794D00EE540724BF83F5F0E045F0F0D8DA05A733
:10795D002205A7800BEB30E7032A8002291F1EFBAF
:10796D00EEC45403F583EE5408C42FF582EE54078C
:10797D00249283F5F0E045F0F0D8DA05A72205A7AB
:10798D00800BEB30E7032A8002291F0EFBEEC45457
:10799D0003F583EE5408C42FF582EE540724658356
:1079AD00F5F0E045F0F0D8DA05A72205A7800BEB3E
:1079BD0030E7032A8002290F1EFBEEC45403F58322
:1079CD00EE5408C42FF582EE5407243883F5F0E009
:1079DD0045F0F0D8DA05A72205A7800BEB30E703B9
:1079ED002A8002290F0EFBEEC45403F583EE5408D2
:1079FD00C42FF582EE5407240B83F5F0E045F0F02B
:107A0D00D8DA05A7228040201008040201EC701F6F
:087A1D00ED20E740D2E023CF89
:107A250023CF30E7F980357B08801A7B1080167BE1
:107A35002080127B40800E20E4ED20E3EE20E2EF73
:107A450020E1F07B80EE8BF0A4CF8BF0A4E5F02F46
:107A5500FFEC8BF0A4CD8BF0A4E5F02D2499838F5A
:107A6500F0A433E5F033FBE98BF0A4E5F0C88BF027
:107A7500A428F9E435F0F822FFFEFCFAF8F6F4F252
:107A8500F0EFEDEBEAE8E6E5E3E1E0DEDDDBDAD9B0
:107A9500D7D6D4D3D2D0CFCECCCBCAC9C7C6C5C40E
:107AA500C3C1C0BFBEBDBCBBBAB9B8B7B6B5B4B328
:107AB500B2B1B0AFAEADACABAAA9A8A8A7A6A5A414
:107AC500A3A3A2A1A09F9F9E9D9C9C9B9A999998D8
:107AD5009797969594949392929190908F8F8E8D7F
:107AE5008D8C8C8B8A8A898988878786868585840B
:107AF500848383828281818075A700907B23E546FC
:107B0500FA24FA50027A05EA2323F978107F0493C0
:107B1500F60809E9DFF9907B3BEA93F556227FC227
:107B2500803E7F4680BA7E8C81747D1882E87A30EB
:107B350085D074608BA0808040201008127B47029E
:107B45007D9DD215D274D273C219C23A1261158EB7
:107B550047757D0075460575520212AA001201DCB3
:107B6500E53524EB500E12AA007F1990BB901281C7
:107B75003712F185E55275F016A4F570127D53752F
:107B85007E15127C1E7F237E0990BB6B12814912E4
:107B9500F18510000810010D10021280E2127CC65A
:107BA50075330180DA127D0B75330180D2757E0045
:107BB500127C1E7E0090BB7F12817C7F237E059008
:107BC500BB74128149127C6F12F185E55210000FCA
:107BD50010010510028780D5045403F55280CE129A
:107BE5007C1E7F237E0B90BBAD128149E546600765
:107BF50014600414124D2212F185E5461000081098
:107C0500010B10021180D860D6154680D2B405024A
:107C150080CD054680C9027B6275320012F2FC7F79
:107C2500017E1190BB6212817C7E0012E9BBE57E6C
:107C3500D26612EA1275170812EE48124D61757177
:107C450000C20612EB62741BFFF5177E0F90BBB4E2
:107C5500305D0390BBBC12817C12AA4312674612A9
:107C650052C7C206126F63022829E55260141460D8
:107C75001E1460297F647E2D791C127CB91E1FD9C4
:107C8500F9227F6A7E1F7928127CB91FD9FA227FD3
:107C9500487E2D791C127CB90F1ED9F9227F567E9C
:107CA5003379281F12F2170F0F12F2171F12F2174E
:107CB5001ED9F0221E12F2170E0E12F2171E02F234
:107CC50017E552605514606814606D800075709EEC
:107CD500127D408003757000E5732540F573E4352A
:107CE50074F574E43575F57522757016127CDD80B2
:107CF5000375702DE5762542F576E5773541F577FF
:107D0500E43578F57822E55260CB1460DC1460E147
:107D15008000757044127CF9800375705AE573957F
:097D250040F573E5749400F57457
:107D2E00E5759400F57522757071127D22800375CC
:107D3E007088E5769542F576E5779541F577E578A5
:107D4E009400F57822E546907D6993F540FEAD47A7
:107D5E00E4FFFC125EA28E418F4222020C183060AC
:107D6E00C07F4012189812283F12F185128018EB2E
:107D7E00700590B8C3800B127E2690BFB950039049
:107D8E00BFFF7F3F7E0412814912F18512F13A1234
:107D9E00F17B75370990BB21122725907DAD7302BB
:107DAE00023D027F6D027B41028049027D9D027D74
:107DBE00C5027DDE027D6F7F2E1220CD80D17F36F3
:107DCE007E0490BF8E12814912F18512F13A80BF66
:107DDE007F3712189812283F12F185127FFC125429
:107DEE0057D2AC1000A9306DFA127ED6203BCF4090
:107DFE00ED7568F9751600127F2340FB1280BF7F68
:107E0E00367E29E51612E79912F18505161281EED6
:107E1E0078C6B6F7E2027FF67C0512545712EFDEF3
:107E2E00744112EFEF745312EF9FEB12EFCD1282EB
:107E3E00005003DCE5227515F975160010000EE5ED
:107E4E00156025127E784005127E9F5002D3227F48
:107E5E003F7E29E51612E79912F1857F1412F15132
:107E6E000516E51664F870D4C3221287BD75B901E4
:107E7E00E5BCB4811AE5BDF51570037516F778C625
:0B7E8E00A6161289061288FE1288FE5C
:107E9900C30288FED3227F0575F019D5E0FDD5F020
:107EA900FA12545712EFDE744112EFEF744212EFD7
:107EB9009F7E0F78C6E60812EF9FDEF912EFD01207
:107EC9008200400122DF012275F00080CEC23B1200
:107ED9005457D2AC12F017204C3CB440F712F01CA6
:107EE900B4400312F01CB4412DF53812F01CB45300
:107EF9002512F01CFA12F01CE538701A12F01CB4A5
:107F09000D1412F01CB40A0EC3E5169A400302813F
:107F1900E5C2ACD23B22C2ACD322128244125457DE
:107F2900D2AC1000F112F017204CEBB440F412F06F
:107F39001CB4400312F01CB441DCF53812F01CB437
:107F490042D47E1078C612F01CF608DEF9E53870C6
:107F5900C512F01CB40DBF12F01CB40AB9C2ACC3EF
:107F690022027D9D7F0A12189812283F12F185126C
:107F79007FFC125473D2AC1000E712F01CB440F528
:107F8900F53812F01CB46EED12F01CE538600A12D7
:107F99005473744F12EFAB80DC125473744012EFB8
:107FA900EFE51612EFAB12EFBB7568F97516001203
:107FB9005473D2AC10003912F01CB440F7F53812E2
:107FC900F01CB44EC07E1078C612F01CF608DEF91B
:107FD900125473E5386007744F12EFAB80D11280E9
:107FE900BF0516745112EFAB78C6B6F7C212805CA2
:0C7FF900027D9D7515007516031287B4FB
:1080050075B901E5BC30E70205160515E51524200F
:1080150050EB227B007515F91287BD75B901E5BCDA
:10802500B481010B0515E515240450EC75150112F5
:1080350087B475B901E5BCB481010B0515E51524B7
:108045002050EC227F1C12189812289C40067515AA
:10805500F912805C027D9DE51560372404401A24E1
:108065001E5019E5152407400280271287BD12808E
:10807500980515E515240450F27515011287B47598
:10808500B901E5BC30E7031280980515E5152420F4
:1080950050EA221280AD1255F705C61255F705C6EE
:1080A5001255F705C60255F774FF80057404800163
:1080B500E4F5BCF5BDF5BEF5BF22E568606AF515CA
:1080C5000515E5152404501D7515011287B475B9FC
:1080D50001E5BC30E70280190515E515242050EBB4
:1080E500751500800C241C60F750E0E5152406503A
:1080F50037E56875F004A485F0C7F5C675BC81E55C
:1081050015F5BDF56878C6B6F70375BD000812818B
:108115002212811C12811C86BC0886BD0886BE08F9
:0981250086BF081255F705C622B9
:10D3F10012CCCD12D4F0128CC112D475128CC91278
:10D40100D48202CCD112CCCD12D4F0128CC17F5A6D
:10D41100C23C128BA3128D9F783F79437F607EEAD5
:10D4210012D4E4128CC97F65128BA3128D9F783DB3
:10D4310079417F207E4E12D4E4303C2012D6A612D0
:10D44100D501783F794312D460783D794112D46097
:10D4510012D6A678D7E65480F675370002C3BEC34C
:10D46100E796FF1819E796FE0809C3E69FF7181912
:10D47100E69EF7227F5B7E0690C09512817C1F801D
:10D481000A7F667E14745912E8B41F128A2C7E3901
:10D49100E402E8D37866E620E73418C3E69472081C
:10D4A100E694045029C318E6941F08E69404401E2C
:10D4B1007869E620E71818C3E6940E08E69401504F
:10D4C1000DC318E6947508E694004002D322C322E6
:10D4D100E67D0030E7011D08E62BFB18E63CFCE485
:0ED4E1003DFD22C3EB9FF6F71819EC9EF6F7FF
:10D4EF002212D495400CE47842F608F67840F608FC
:10D4FF00F6227864C3E6946AF55708E6944CF5561D
:10D50F000808C3E69458F55B08E694AEF55A7539EA
:10D51F0000AC56AD57EC12D063784C12D0F1AC5A28
:10D52F00AD5BEC12D063785012D0F17F2B7E867DED
:10D53F00777C1812D028785012D0E512CF3412D041
:10D54F0028785012D0E512CF3412D028785012D04C
:10D55F00E512CF3412D0287F367E847D257C64126D
:10D56F00D028785012D0E512CF3412D028784C1230
:10D57F00D0E512CF3412D0287F3F7EA27D607C8B06
:10D58F0012D028785012D0E512CF3412CD2212CDFE
:10D59F002212D0FD7F3F7E807D057CE6053912CFBC
:10D5AF0034784812D0F17F2C7E937D477C7F12D048
:10D5BF0028785012D0E512CF3412D028785012D0DC
:10D5CF00E512CF3412D028784C12D0E512CF341296
:10D5DF00D0287F357EB47DF87CDF12D028785012AA
:10D5EF00D0E512CF3412D028785012D0E512CF34B4
:10D5FF0012D0287F3F7EED7D227CCD12D028784C33
:10D60F0012D0E512CF3412CD2612CD22784412D08B
:10D61F00F17F317E397D9D7CE712D028784C12D076
:10D62F00E512CF3412D028784C12D0E512CF341235
:04D63F00D028784433
:10D6430012D0E512CD2612D0287F2C7E377D0C7C9C
:10D65300A312D028784C12D0E512CF3412D02878F8
:10D663004C12D0E512CF3412D028784C12D0E512E8
:10D67300CF3412CD2612D0FD7F3F7E807D027C9F6A
:10D68300053912CF34784412D0F1784812D0E5121C
:10D69300D09A8E428F43784412D0E512D09A8E40AE
:10D6A3008F4122753900AC42AD43EC12D063784808
:10D6B30012D0F1AC40AD41EC12D063784412D0F1FA
:10D6C3007F2B7E537D507C0912D028784812D0E5F9
:10D6D30012CF3412D028784812D0E512CF3412D0AA
:10D6E30028784412D0E512CF3412D0287F347EF24A
:10D6F3007DCD7CA312D028784812D0E512CF341206
:10D70300D028784812D0E512CF3412D0287F3F7E3C
:10D713000A7D2E7CAE12D028784412D0E512CF3485
:10D7230012CD2212CD22784C12D0F17F2B7E4F7D69
:10D73300AF7CB212D028784812D0E512CF3412D081
:10D7430028784812D0E512CF3412D028784812D066
:10D75300E512CF3412D0287F357EB17D4B7C9512F4
:10D76300D028784812D0E512CF3412D0287844124A
:10D77300D0E512CF3412D0287F3F7E497DCD7C4542
:10D7830012D028784812D0E512CF3412CD2612CD0C
:10D7930022785012D0F1784C12D0E512D09A8D55E0
:10D7A3008E568F57785012D0E512D09A8D598E5AD3
:04D7B3008F5B7864AC
:10D7B700E557246AF608E556344CF608E55534046F
:10D7C700F608E55B2458F608E55A34AEF608E43562
:03D7D70059F622DE
:10C20C0012CCCD12C89D12CCD17F6690C077128112
:10C21C007A12C27A7F5A78C412C25612C25E78C69B
:10C22C0012C25612C2417F6578C812C25612C25E43
:10C23C0078CA12C2567E2DE51B12E8D37E33E51A5E
:10C24C0012E8D37E39E51902E8D386040886030286
:10C25C005D6C7E15E51C12E8D37E1BE51B12E8D342
:10C26C007E21E51A12E8D37E27E51902E8D37F5A1E
:10C27C007E01E53A12E7E77E0B90CC91E53B930209
:10C28C00E8E6E6FF08E6FE08E6FD339217E4500107
:10C29C00F4FC12D10E75130A75390112D30C78D730
:10C2AC00E6C2E775F00A84F9303D02A9F012D10E0E
:10C2BC008913053912D2E530170A053912D2F8055F
:10C2CC003912D2F8A80302D0F112CCCD12C89DC2FB
:10C2DC003C7F5A7E03128F5012C27A12F1851000E5
:10C2EC000810011510022080EFE53A146004153A8D
:10C2FC008003753A3CD23C80DFE53AB43C05753A94
:10C30C000180F2053A80EE7E03128F4B7E0B128F6A
:10C31C005012C27A12F1851000081001151002207B
:10C32C0080EFE53BB40205753B158002153BD23C12
:10C33C0080DFE53BB41505753B0280F2053B80EED2
:10C34C007E0B128F4B7F5A78C412C25612C25E12E9
:07C35C00C3C7128DAF78C4C6
:10C3630012C41F78C612C25612C24112C3F9751CF9
:10C3730000128DAF78C612C41F7F6578C812C256EB
:10C3830012C25E12C3C7128DAF78C812C41F78CA17
:10C3930012C25612C24112C3F9751C00128DAF7836
:10C3A300CA12C41F303C14E53B24F4500B78C9E691
:10C3B3002410F618E63427F612C42512CCD11289BC
:10C3C3003102F185C2247E15E51C128EA0F51CD224
:10C3D300247E1BE51B128EA0F51B1023E77E21E5AF
:10C3E3001A128EA0F51A1023E67E27E519128EA0E5
:10C3F300F5191023E822C2247E2DE51B128EA0F529
:10C403001BD2247E33E51A128EA0F51A1023E77E81
:10C4130039E519128EA0F5191023E622ECF608EB84
:10C42300F62212CCA978C8E6FE0886073395E0FD0C
:10C43300FC12D0287FE87E037D007C0012D30C120F
:10C44300D02878CAE6FE0886073395E0FDFC12D2B1
:10C45300E512D0287F807E697D677CFF12D2E5ECF0
:10C4630012D05F12D0287F3F7E807D0D7C1D12CFBE
:10C473003412D0287F3D7E407D007C0012D0287886
:10C48300BC12D0E512CF3412D0287F3E7E807D00CF
:10C493007C0012CD2612D02878BC12D0E512CF34FE
:09C4A30012D0287F3F7E807D004D
:10C4AC007C0012CD2212D02878B412D0E512CF34F1
:10C4BC0012CFAC783C12D0F17F407E807D007C00A6
:10C4CC0012D028783C12D0E512CF3412D18B12D076
:10C4DC00287F3F7EA87D007C0012D02878B812D02F
:10C4EC00E512CF3412CF3412D0287F407E007D006D
:10C4FC007C0012D028783C12D0E512CF3412D18BAC
:10C50C0012D0287F3F7EC07D007C0012CF3412CD2C
:10C51C002612D02878B812D0E512CF3412D0287851
:10C52C003C12D0E512CD26785412D0F112D1757888
:10C53C005812D0F112D02812CF3412D02878C01251
:10C54C00D0E512CF34784412D0F1785412D0E512E1
:10C55C00D18B783C12D0F112D02812CF3412D028C3
:10C56C0078BC12D0E512CF34783C12D0F17F3E7EED
:10C57C00C07D007C0012D028783C12D0E512CF345C
:10C58C0012D0287F3F7E007D007C0012CD2612D079
:10C59C0028783C12D0E512CF3412D0287F3F7E8011
:10C5AC007D007C0012CD2612D02878B412D0E51272
:10C5BC00CF34787012D0F178C4E6FE088607339534
:10C5CC00E0FDFC12D0287FE87E037D007C0012D3B6
:10C5DC000C12D02878C6E6FE0886073395E0FDFCE1
:10C5EC0012D2E512D0287FE07E5E7DF87CFF12D25D
:10C5FC00E5EC12D05F12D0287F3F7E7F7DE57CC9B1
:05C60C0012D028787037
:10C6110012D0E512CF3412CFAC785012D0F17F3F57
:10C621007EF07D007C0012D028783C12D0E512CF3C
:10C631003412D0287F3F7EC07D007C0012CD2612AF
:10C64100D028783C12D0E512CF3412D0287F3F7E1B
:10C65100807D007C0012CD26783C12D0F178BC128E
:10C66100D0E512D0287F3F7E807D007C0012CD2254
:10C6710012D028783C12D0E512D02878B412D0E537
:10C6810012CF3412CF34784012D0F1785412D0E561
:10C6910012D1C3783C12D0F112D02812CF34787461
:10C6A10012D0F17F417E107D007C0012D02878C02D
:10C6B10012D0E512CF3412D0287F407E807D007CDD
:10C6C1000012D028784412D0E512CF3412D0287F3E
:10C6D100417E207D007C0012CD2212D028784412A8
:10C6E100D0E512CF3412D0287F407E407D007C00FF
:10C6F10012D028787412D0E512CF3412D0287F409E
:10C701007EA07D007C0012CD2612CD2612CD2212F4
:10C71100D028785012D0E512CF3412D02878501298
:10C72100D0E512CF3412D0287F3D7E2A7DAA7CAB82
:10C7310012CF3412D0287F3F7E007D007C0012CDC5
:10C741002212D028783C12D0E512D028787012D06D
:10C75100E512CF3412D028784012D0E512CFAC12B6
:10C76100D028785012D0E512CF3412D02878501248
:10C77100D0E512CF3412CF3412D028785412D0E53C
:0CC7810012CD2212D0287F4A7E517DD2BA
:10C78D007CCB12CF3412D09A78AC12D0F17F407E90
:10C79D00007D007C0012D028787412D0E512CF34C1
:10C7AD0012D0287F3F7E807D007C0012CD2612D0D6
:10C7BD0028784412D0E512CD2612D028785012D008
:10C7CD00E512CF3412D028785012D0E512CF3412A2
:10C7DD00D028785012D0E512CF3412D0287F3E7E6B
:10C7ED002A7DAA7CAB12CF3412D028785012D0E516
:10C7FD0012CD2212D028785812D0E512CFAC12D01B
:10C80D00287F4A7E517DD27CCB12CF3412D09A1222
:10C81D00D028AF3AEF3395E0FEFDFC12D0287F40D3
:10C82D007E7E7D057C0012D30C12D0287F607E7534
:10C83D007D587CFF12D2E512D2E578B012D0F17896
:10C84D00AC751B6412C8748F1C78B0751B6712C849
:10C85D0074E51C75F00AA42FFF249C50027F00780C
:10C86D00D7E654802FF62275390012D0E512D02864
:10C87D007F0A7E007D007C0012D3B8A81BE513F65D
:10C88D0008E512F608E511F6335004EFF404FF2223
:10C89D00C23D78647BAC12C28ED23D78677BB012FC
:10C8AD00C28E12CCA97F007EE47D577C0012D02869
:10C8BD0078AC12D0E512D2E512D0287F007E537DE0
:0EC8CD00077C0012D3B812D04785133B7F8042
:10C8DB007ECB7DA47C0012D02878B012D0E512D28A
:10C8EB00E512D0287F407E7E7D057C0012D3B812E6
:10C8FB00D047E513F56F04F53A85126E85116D85FA
:10C90B00106C7F407E7E7D057C0012D028786C12E7
:10C91B00D0E512D30C12D0287F607E0C7DA27C0058
:10C92B0012D02878B012D0E512D2E512D2F8786C7A
:10C93B0012D0F178AC12D0E5EC12D05F12D0287F78
:10C94B00347E9C7D2B7C5F12CF34785412D0F11245
:10C95B00D175785012D0F1786C12D0E5EC12D05F13
:10C96B0012D0287F347E9C7D2B7C5F12CF3412D06B
:10C97B0028785012D0E512CF34784012D0F17F4096
:10C98B007E007D007C0012D028785412D0E512CFA7
:10C99B003412D18B12D0287F3D7EC07D007C0012DB
:10C9AB00D02878BC12D0E512CF3412D0287F3E7E2F
:10C9BB00C07D007C0012CD2612D02878BC12D0E5A9
:10C9CB0012CF3412CF3412D0287F3D7E407D007CB5
:10C9DB000012D02878BC12D0E512CF3412D0287FA9
:10C9EB003E7E807D007C0012CD2612D02878BC12B2
:10C9FB00D0E512CF3412D0287F3F7E807D007C00A3
:10CA0B0012CD2212D028785412D0E512CF3412CD89
:10CA1B002212D0287F407E807D007C0012D02878A7
:10CA2B005412D0E512CF3412D18B12D0287F3D7E19
:10CA3B00707D007C0012D02878BC12D0E512CF3468
:10CA4B0012D02878BC12D0E512CF3412CF3412CDCD
:10CA5B002612D02878B412D0E512CF34785812D0E1
:10CA6B00F1785412D0E512D18B783C12D0F1785476
:10CA7B0012D0E512D1C3785412D0F1783C12D0E524
:10CA8B0012D02812CF3412D02878BC12D0E512CF96
:10CA9B0034783C12D0F17F3E7EC07D007C0012D0FA
:10CAAB0028783C12D0E512CF3412D0287F3F7E007D
:10CABB007D007C0012CD2612D028783C12D0E512D6
:10CACB00CF3412D0287F3F7E807D007C0012CD2694
:10CADB0012D02878B412D0E512CF34787012D0F17E
:10CAEB00785012D0E512D02812CF3412D02878C04B
:10CAFB0012D0E512CF34784412D0F1785412D0E52D
:10CB0B0012D02812CF34787412D0F1784012D0E5BD
:10CB1B0012D02812CF34783C12D0F17F407E807D2A
:10CB2B00007C0012D028784412D0E512CF3412D0FA
:10CB3B00287F417E107D007C0012CD2612D02878F4
:10CB4B004412D0E512CF3412D028787412D0E512EB
:10CB5B00D0287F407EA07D007C0012CD2212CD26F6
:10CB6B0012D028783C12D0E512CF3412D0287F3D5A
:10CB7B007E2A7DAA7CAB12CF3412D0287F3F7E0059
:10CB8B007D007C0012CD2612D028785412D0E512ED
:10CB9B00D028787012D0E512CF3412D028783C12FE
:10CBAB00D0E512CF3412CF3412D028785812D0E5FA
:10CBBB0012CD2612D0287F3F7E7F7DE57CC912CF18
:01CBCB003435
:10CBCC0012D0287F4B7E187D967C8012CD2612D0F9
:10CBDC009A12D0287FE87E037D007C0012D3B81215
:10CBEC00D04778C8A61208A61308A60608A6077888
:10CBFC007412D0E512D0287F3F7E807D007C00121D
:10CC0C00CD2212D028784412D0E512CD2612D0288D
:10CC1C007F3E7E2A7DAA7CAB12CF3412D02878407E
:10CC2C0012D0E512CF3412D028783C12D0E512CFB6
:10CC3C003412D028784012D0E512CD2612D0287F9D
:10CC4C003F7E7F7DE57CC912D028787012D0E5122A
:10CC5C00CF3412CF3412D0287F487EF47D247C0050
:10CC6C0012CD2612D09A12D0287FE87E037D007C4C
:10CC7C000012D3B812D04778C4A61208A61308A67F
:10CC8C000608A607223F3F4344454647484A4B4CBB
:10CC9C004D4E5051525354555657583F3FE4F53969
:10CCAC00F5A790CCBD791078B4E493F6A308D9F924
:10CCBC002232A5C24A4A19DC3A885CDB3BFFD6DC3F
:01CCCC003B2C
:10CCCD00D2D58002C2D575A70490040078107F0BD1
:10CCDD0012CCF978267F0512CCF9783C7F2212CC44
:10CCED00F9786A7F0F12CCF975A7002230D506E6C8
:10CCFD00F008DFFB22E0F608DFFB22DA0CD9028018
:10CD0D000BD906303701B3500502CE95923702CEBE
:10CD1D0081D9F680F9D2368002C23612CEC63036AF
:10CD2D0006C86002B237C89236DAD0D9E4B8000A24
:10CD3D0012CF0DA236923702CE6A60FBB5130040BA
:10CD4D000F12CF0DA23692F7A2379236A2F7923775
:10CD5D00C398F40424E740DF2419AD29AC28AB2790
:10CD6D007A00C394084008CDCCCBCAE4CD80F4241E
:10CD7D00086010F9C3ED13FDEC13FCEB13FBEA1384
:10CD8D00FAD9F1A236303701B340308A17E5102BAE
:10CD9D00F518E5113CF519E5123DF51A501A13F584
:10CDAD001AE51913F519E51813F518E51713F51705
:10CDBD000513E5137002051402CE20E4C39AF5178E
:0CCDCD00E5109BF518E5119CF519E51226
:10CDD9009DF51A500DB237C378177F04E496F6080B
:10CDE900DFFA7A047019E513C39408F51350021594
:10CDF90014E4C517C518C519F51ADAE802CEC12019
:10CE0900E7BAE5137002151415137817C37F04E602
:10CE190033F608DFFA80E8E51A20E7137817C37FAD
:10CE290004E633F608DFFAE513700215141513E565
:10CE3900173378187F03E63400F6500E08DFF775CC
:10CE49001A800513E51370020514E51420E75470E0
:10CE590027E513604E046020851A1285191185187B
:10CE6900105326F0AC10AD11A237E51313FFE512EC
:10CE790092E7FEA81302D047E4F512F511F510F573
:10CE8900147513FF5326F043260580D8E5FFF512E4
:10CE9900F511F510751400F513D2375326F0432612
:10CEA9000980C15326F0432603E4F512F511F51064
:10CEB900F514F513C23780AC5326F080EC79017A6A
:10CEC900018512F0E513A2F7339237751400F513B3
:10CED9006002D2F785F012A813B8FF0809E512C25B
:10CEE900E76001098C278D288EF0A2F7EF330470D3
:01CEF9000A2E
:10CEFA000AC2F705F00AD5F0011A146002D2F785C2
:10CF0A00F02922C88813C512C529C512C511C5281A
:10CF1A00C511C510C527C51022DA03B8000302CE11
:10CF2A0095D9028002D9F702CE8112CEC6303701D6
:10CF3A00B392377004D9E78005DADEB8000302CE6F
:10CF4A00C1D9E2C3947E500215142513F513500279
:10CF5A0005147815760008B81BFA78277915E608BB
:10CF6A00FAE8FC78108AF0E608A427F709E5F03712
:10CF7A00F7500989F00907E760FBA9F0B813E61929
:10CF8A0019ECF8B82AD802CE2002CEACB8FFFA02C1
:10CF9A00CE95D9FB02CE81DAF6B800F002CEC112E4
:10CFAA00D0FD12CEC6303701B392377007D9E3B835
:10CFBA0000E280DBDAE1B8000280E1D9D5C8C39883
:10CFCA0050021514247F50020514F513781A7600BE
:10CFDA007A1A7B80C3E5109527E5119528E5129505
:10CFEA00294016C3E5109527F510E5119528F51186
:10CFFA00E5129529F512E64BF6DA0302CE20EB0389
:0AD00A00FB30E703187600C3E510C1
:10D0140033F510E51133F511E51233F51240CA303A
:10D02400E7DD80B6E53905396010D0F0D0E0C010F6
:10D03400C011C012C013C0E0C0F08F138E128D1146
:10D044008C1022E539146010D0F0D0E0D013D01247
:10D05400D011D010C0E0C0F01539227920800C79AD
:10D0640010800479087D007E007F003392D5500340
:10D0740012D0D7EC33400FEF33FFEE33FEED33FD28
:10D08400EC33FCD9EE22EECCF5F0747E29A2D51354
:10D09400FF92F7AEF022EF8EF0A2F7D2F73392D5DB
:10D0A400C3947F5006E4FFFEFDFC229420400474E8
:10D0B400FF80F304CCFEE4FFFAE5F0CC6012C3CCAD
:10D0C40013CCCD13CDCE13CECF13CF0450EEDAEC68
:10D0D40030D5D7C3E49FFFE49EFEE49DFDE49CFCB1
:0CD0E40022E6FC08E6FD08E6FE08E6FF78
:10D0F00022ECF608EDF608EEF608EFF622CFC5139F
:10D10000CFCEC512CECDC511CDCCC510CC22E4F505
:10D1100013F512F511F51022E493FCA3E493FDA39B
:10D12000E493FEA3E493FFA322C0E012D02812CF21
:10D130003412D15C12D118D0E0C0E012D02812D144
:10D140005312CF3412D02812D11812CD26D0E0D5E8
:10D15000E0E722AC48AD49AE4AAF4B228C488D493E
:10D160008E4A8F4B2274FF7809FFFEFDFCE52654A2
:10D17000F048F5262212D21C04A2E1927F1420E08E
:10D180001590D29D740412D129802912D21C30E14D
:10D1900002B27F20E0EB8C4C8D4D8E4E8F4F90D2A3
:10D1A000B1740412D12912D028AC4CAD4DAE4EAFA3
:10D1B0004F12CF34307F04EF6480FFEE33EF3370D3
:10D1C00001FF2212D21CC0E08C4C8D4D8E4E8F4F31
:10D1D00090D2D5740312D12912D028AC4CAD4DAEEB
:10D1E0004EAF4F12CF34ECC54CFCEDC54DFDEEC536
:05D1F0004EFEEFC54FEB
:10D1F500FF90D2C5740312D129D08212D028AC4C2D
:10D20500AD4DAE4EAF4FE58230E00712CFACB27FE9
:10D21500809D12CFA98098EE33EF3324605007D05C
:10D22500E0D0E002D165EFA2E7547F927FFF12D0F4
:10D23500287C837DF97E227F3E12CF34EE33EF3397
:10D245002481501012D02812D09A12D05FEFB2E785
:10D25500FF12CD26EE33EF33602A2403F8C313FF04
:10D26500EE92E7FEE82481E4501A12D02812D09AF3
:10D27500EF04C2E0FCF58212D067EFB2E7FF12CDF2
:10D2850026E58203FAEE33EF33600B148FF0A2F735
:10D2950013FFEE92E7FEEA2283FA703AE4E9AABCAC
:10D2A500F8E0813EE6E99DBF0000803F1A3C283941
:10D2B500666999BBE335A33DE75D25BFDB0FC93F34
:10D2C500CCDB8D41EE3649C43F91C9453DF8B0C52B
:10D2D5000000803F34F517C373FA2F45DDFD0AC6FC
:10D2E500EF2513FFEE3512FEED3511FDEC3510FC83
:10D2F50002D047C3EF9513FFEE9512FEED9511FD94
:10D30500EC9510FC02D047EFF88513F0A4FFE51368
:10D31500C5F0CEF9A42EFEE435F0CDFA88F0E5127D
:09D32500A42EFEED35F0FDE43309
:10D32E00CC8513F0A42CFCE5128AF0A42CFCE5119C
:10D33E0089F0A42CFCE51088F0A42CFC89F0E512F1
:10D34E00A42DFDEC35F0FCE51188F0A42DFDEC3597
:10D35E00F0FC8AF0E513A42DFDEC35F0FC02D0476D
:10D36E00E4CCF8E4CDF9E4CEFAE4CFFB75F020C3BB
:10D37E00E51333F513E51233F512E51133F511E527
:10D38E001033F510EF33FFEE33FEED33FDEC33FCCF
:10D39E00EF9BEE9AED99EC98400CFCEF9BFFEE9A0A
:10D3AE00FEED99FD0513D5F0C622C2D5EC30E7058A
:10D3BE00B2D512D0D7E51030E70DB2D512D3DB12AD
:10D3CE00D36E12D0D7800312D36E30D515C3E49529
:10D3DE0013F513E49512F512E49511F511E4951079
:03D3EE00F5102215
:108F9E00E57124885002D2191261158E4712E5F739
:108FAE0012AA431264D1305E0F12646F12A12F12F7
:108FBE0063A0129D6F124E5C124578125403103648
:108FCE0026301219E4129121129136129231129218
:108FDE00533051030292DD1295AE205109C251E475
:108FEE00F552F545F5442275A700758307E559C47A
:108FFE0054F0F582E0F538A3E0F518A3A3A3E0F54D
:10900E001E74FF1291211261158E1C8F1B7510DFBD
:10901E00751100E51164B470061290EC7511101202
:10902E0090B94028AE1CAF1B12619D20321EAC03BE
:10903E00AB027A0C125DA4ED701275A70075830455
:10904E00851182ECF00583E510F00511D510C412E0
:10905E0090EC75C70375C6E075A7049005007F04F4
:10906E001290A7DFFB75A70012385712646FE4F554
:10907E00A7F8F559758307E8C4F582E065387011D5
:10908E00A3E06518700BA3A3A3E0651E70038859B7
:10909E002208C3E5589850DC22E0F5BCE0F5BDE0AF
:1090AE00F5BEE0F5BF1255F705C622E51075F004C2
:1090BE00A4F5C685F0C775B901E5BC33401F05C6DA
:0B90CE0005C675B90185BE6485BF654D
:1090D90005C675B90185BC6685BD6785BE6885BF4E
:1090E90069C322E51124FE502E75A7007F10AE1129
:1090F9001E7583048E82E0FD1582E0CDB505005012
:1091090012F00582CDF00583E0FD1582E0CDF00572
:1091190082CDF0DEDCDFD7227FB475A7549004003E
:1091290005A7900500F0F0DFFC75A7002212993918
:10913900C2517B077AFFE47F00F5A79004001292E1
:109149001DED244C4035EC603075A7008D8205A7D4
:109159001291E37583058D82E02410401CF005A768
:10916900E02CF0500505A7E004F0BA000CBB00099B
:10917900D251EF24DC50027F23DFC3EA600512914C
:10918900968006EB60031291CE75A7002230E004A9
:109199007553082230E1047553182230E2047553DF
:1091A900282230E3047553382230E40475534822E9
:1091B90030E5047553582230E6047553682230E7C8
:1091C900037553782230E0047553882230E1047521
:1091D90053982230E2037553AA22ED54F0C4232395
:1091E9009091ED735302FE225302FD225302FB229A
:0791F9005302F7225302EFBD
:10920000225302DF225302BF2253027F225303FE66
:10921000225303FD225303FB225303FB22129833F4
:1092200012B191E4F5F7E4ADF7F5F7E4ACF7D2B29B
:109230002290050078B4E06015FD54F0C4CD7C00A8
:10924000540FFE1583E0FF125EA2EFF00583058246
:10925000D8E42275830478FF088882E060FAF5D3A9
:109260008812E512244C50012285D3D288D488126A
:1092700079FF0512E51260F00908E875F0B484A8DA
:10928000F08882E060ECF5D3B9000280D5B9230004
:1092900050D0C395D292D15002F40409FEE4FFFCF1
:1092A000AD01125EAF7401FA25D475F0B484A8F054
:1092B000AC06AB07125D96EB30E7010CE5D22C3023
:1092C000D1029C9C8882F00AEAB501DCE512244CAC
:1092D00050012285D3D28512D4A812809390040025
:1092E00012939C8C068B0512939CE4FFF512F511EA
:1092F0008C148B13C3ED9BF9EE9CFA4012E5119987
:0B930000E5129A500A8C148B138A129D
:10930B0089118F528F82E0F9C3ED99FDEE9400FE27
:10931B00E582245A5002244C75F0B48485F082E027
:10932B00FA2DFDEE3400FEEB9AFBEC9400FCE92BDE
:10933B00FBEC3400FC0FBFB4B0E55224D340022445
:10934B00B4F552C3E51333FBE51433FCE511FE2BE7
:10935B00FBE512FF3CFC125F04E9F89093AE93F52A
:10936B0011FDEBF513FFECF514FE7C00125EA28FE2
:10937B0044E89094AE93FAAB13AC14125DCDAF03EB
:10938B00AE04AD117C00125EA2EF7002F552F545F2
:10939B00227C007B007F5AE02BFBEC3400FC058227
:1093AB00DFF522B4B4B4B4B4B4B4B4B4B4B4B4B498
:1093BB00B4B4B4B4B4B3B3B3B3B3B3B3B3B3B3B36D
:1093CB00B3B3B2B2B2B2B2B2B2B2B2B1B1B1B1B175
:1093DB00B1B1B0B0B0B0B0B0B0AFAFAFAFAFAEAE89
:1093EB00AEAEAEAEADADADADADACACACACACABABA7
:1093FB00ABABAAAAAAAAA9A9A9A9A9A8A8A8A8A7D0
:10940B00A7A7A7A6A6A6A5A5A5A5A4A4A4A4A3A300
:10941B00A3A2A2A2A2A1A1A1A0A0A0A09F9F9F9E38
:10942B009E9E9D9D9D9D9C9C9C9B9B9B9A9A9A9975
:10943B0099999998989897979796969695959594B4
:10944B009494939393929292919191919090908FF7
:10945B008F8F8E8E8E8D8D8D8C8C8C8B8B8B8A8A39
:10946B008A8989898888888787878686868585857E
:10947B008484848383838282828181818080807FC4
:10948B007F7F7E7E7E7E7D7D7D7C7C7C7B7B7B7A05
:10949B007A7A797979787878777777767676757549
:1094AB00757474000203050608090B0C0E101113DA
:1094BB00141617191A1C1D1F2122242527282A2BA5
:1094CB002D2E303133343637393A3C3D3F40424311
:1094DB00454648494B4C4E4F505253555658595A86
:1094EB005C5D5F606163646667686A6B6C6E6F700E
:1094FB007273747677787A7B7C7E7F8081838485A8
:10950B008688898A8B8D8E8F909192949596979859
:10951B00999B9C9D9E9FA0A1A2A4A5A6A7A8A9AA22
:10952B00ABACADAEAFB0B1B2B3B4B5B6B7B8B9BA08
:10953B00BBBCBDBEBFC0C0C1C2C3C4C5C6C7C7C804
:10954B00C9CACBCCCCCDCECFD0D0D1D2D3D4D4D51D
:10955B00D6D7D7D8D9DADADBDCDCDDDEDEDFE0E04C
:10956B00E1E2E2E3E4E4E5E5E6E7E7E8E8E9EAEA95
:10957B00EBEBECECEDEEEEEFEFF0F0F1F1F2F2F3F2
:10958B00F3F4F4F4F5F5F6F6F7F7F8F8F8F9F9FA69
:10959B00FAFAFBFBFBFCFCFDFDFDFEFEFEFEFFFFF6
:1095AB00FFFFFFC251E4F544F814FB900400A9003F
:1095BB007C0FC2D11296C9E82405F8B8B4F08B130E
:1095CB00E5122403FA244C5001FABBFF012275115A
:1095DB002C8A191297008F16203D12AA1975112388
:1095EB001297008F15751600303DE280117511230F
:1095FB001296A8751500303D05E82F13F51575115A
:01960B00124C
:10960C001296A8751400303D05E82F13F514EA24C2
:10961C0004F552244C5002F552E4F51AF51BF51CD6
:10962C00E516600AFB7A00AF137EFF12966EE51505
:10963C00600AFB7A4FAF137EFF12966EE516600D33
:10964C00FB7A00E5146006FF7ECF12966EAE1CAF5F
:10965C001B7C00AD1A125EA28F45EF2513F544D288
:10966C005122EFF5F0A4FCADF0EBF5F0A49CFCE579
:10967C00F09DFDEB8AF0A4FAABF0EF8EF0A49AF813
:10968C00E5F09BF9E833F8E933F97B00125F480504
:10969C001AE51B2BF51BE4351CF51C22EA2511F9E8
:1096AC00244C5001F9C2D11296C7303D428F00C3F1
:1096BC00EA9511F9500324B4F9D2D17C09E4FDFEEA
:1096CC00FF8982E060062FFFE43EFE0D09B9B4026B
:1096DC007900DCEDED20D118F51E24FE923D500FE3
:1096EC00125EAFEFB503005006851E1FFB881222D9
:1096FC00F51D80E61296A8203D43740212979F1226
:02970C0096A81D
:10970E00203D3874041297A71296A8203D2D74069A
:10971E0012979F1296A8203D2274081297A71296B0
:10972E00A8203D17740A12979F1296A8203D0C741C
:10973E000C1297A71296A8203D0122C3E89F6050F5
:10974E0088148F158A1640081ABAFF0A7AB3800653
:10975E000ABAB4027A001296A8303D34C3E89FF9D3
:10976E00602EC3E5149515FB6930E7D4E930E703A5
:10977E00F404F9EB30E702F404C3995002AA16E59B
:10978E00142515C82F28FFE4FC33FE7D04125EA2BB
:10979E00222AFA244C5001FA22C3CA9AFA50032400
:1097AE00B4FA2212188E85BF6C85BE6B756A0002E4
:1097BE00B174129CEB852E72E55F030354C0F8E57D
:1097CE005E543F28F57C3055062212B0ED80031210
:1097DE00B0DD7410256A54F0F56AE4356BF56BE470
:1097EE00356CF56C24815003756C0022756A00E4AB
:1097FE00D380E8E54B75F010A4256A54F0F56AE5C0
:10980E00F080D8E56A24F054F0F56AE56B34FFF584
:0E981E006BE56C34FFF56C24815003756C7E95
:10982C0022E56A24FF80E4E56D24F054F0F56DE543
:10983C006E34FFF56EE56F34FFF56F2481500375C0
:10984C006F7E221298AB129908C22DC254C255E5F4
:10985C007F7002D255147002D254E54A30E00122D6
:10986C00B4062120540C129811129BBD129C6C0250
:10987C009D02129DE37E0412F147754A0112F141DB
:10988C00756A202220550C1297E0129C3D129CEB1D
:10989C00029B96129DE37E0412F147754A05221233
:1098AC00B17C7870E4F5F7E4A6F708B880F6D2B28C
:1098BC0022129939756D1012B191E4F5F7E4E5F7C0
:1098CC00D2B264C0702D756D1E12B191E4F5F7E43F
:1098DC00E5F7C4F9E4F5F7E4E5F7D2B2C4F8E954D6
:1098EC000FFD5301F0E8540F49FCE854F0FB7F03E3
:1098FC00129B28056EE56E540370B922E575F85479
:10990C001F30E40244E0F57585722EA2779226E5AD
:10991C007C543F30E50244C0F55EE57C54C0232303
:10992C00F55FE57FC2E779BCF709A77E22856C6FEE
:10993C00856B6E856A6D22856F6C856E6B856D6A25
:10994C0022FA7420303B0274608510F0A4256EF569
:01995C004DBD
:10995D00E5F0356FF54EEA2323303B0475F003A493
:10996D00254DF54DE5F0354EF54E754C00227580C3
:10997D0000C2B212F14FD2B222758000C2B2F5F719
:10998D00A4D2B222758000C2B2F5F7A48DF7A48CD3
:10999D00F7A48BF722EB241054F0FBE43CFCE43DE0
:1099AD00FD22EB24F054F0FBEC34FFFCED34FFFD15
:1099BD0022758000C2B2F5F7A4856FF7A4856EF706
:1099CD00A4856DF722E56D241054F0F56DE4356E28
:1099DD00F56EE4356FF56F22756D00E56E24045458
:1099ED00FC80EDE56D24F054F0F56DE56E34FFF57A
:1099FD006EE56F34FFF56F22756D00E56E24FC5436
:109A0D00FC80EC758000C2B2F5F7A4854EF7A485F5
:109A1D004DF7A4854CF722740F254CF54CE4354DCC
:109A2D00F54DE4354EF54E2274F1254CF54CE54DD2
:109A3D0034FFF54DE54E34FFF54E22754C00E54DE6
:109A4D0024FC54FC80EC7403129A1075A70090044A
:109A5D000075F700A4E5F7F0A3E58324F850F2753F
:039A6D00F700A45B
:109A7000E5F7D2B2C23C30E602D23C754C00E54D6F
:109A8000240454FC80A77403129A1075A700900454
:109A9000007F22129ABB8010E54C2411FBAC4D0CC8
:109AA0000CAD4E740312999175A7009004117F00BC
:109AB000129ABB7FEF129ABBD2B22275F700A4E5CF
:109AC000F7F0A3DFF622D23CE4F56FF56EF56D7486
:109AD000031299BEE4F5F7A4E5F7D2B204600BC215
:109AE0003C1299D2E56F24FE50E5923D227F107919
:109AF000B8740612998674021299BE87F709DFFBC3
:109B0000D2B280337F1079B874031299BEE4F5F7AE
:109B1000A4A7F709DFF7D2B278B9793A12DB8E023F
:109B20009C8AAD6FAC6EAB6D74061299867402128E
:109B300099918FF7A4D2B2758000C2B275F705A4CF
:109B400075F705A4E5F7D2B220E0EC227403129970
:109B500091E4F5F7A4E5F7D2B222E4FEFF740775AD
:109B6000A704F5838E8274FFF0DFFD75A7002274D1
:109B7000067E007FB0129B5FE4F55AF55B2275A765
:109B800004758306E55A600A75F00A84E5F07002F0
:0B9B9000740AC4F58222307720E55AE9
:109B9B0024024002055A129B7EE55AF0E573F0E56C
:109BAB0074F0E575F0E576F0E577F0E578F075A7FC
:109BBB0000223077F9129B7E7F1074FFF0DFFDE5FA
:109BCB005A24F55003129BE8155AE55AB4FF0205C7
:109BDB005AC3E55A955B50D6755B0080D112993903
:109BEB007F0A056D056D12B191E4F5F7E4E5F7D247
:109BFB00B230E704DF02800512983380E5056D1261
:109C0B00B191129B7EE55A24F6F07F06E4F5F7E45A
:109C1B00E5F7F0DFF7D2B275A700227F42129C2E38
:109C2B00DFFB22302B0C0542E542247C40012275E0
:109C3B004280053FE53FB43C17753F00053EE53ECE
:109C4B00B43C0D753E00053DE53DB41803753D0074
:109C5B00802D302B0C1542E5422483500122754296
:109C6B0080153FE53FB4FF17753F3B153EE53EB40E
:109C7B00FF0D753E3B153DE53DB4FF03753D177874
:109C8B00ABA63A08A63B08A63C121875E5BF253DC6
:109C9B00240C75F0188478AEA6F018600564026089
:109CAB00182216E670121816E67004760C18167841
:099CBB00ACE6909CDE9308F62251
:109CC4000618E608909CDE930466700D760118066B
:109CD400E6640D70047601180622001F1D1F1E1F66
:109CE4001E1F1F1E1F1E1F0542E542B43C0F754276
:109CF400000541E541B43C0575410005402215428B
:109D0400E542B4FF0F75423B1541E541B4FF0575CB
:109D1400413B154022AC40AB41A842EC75F03CA459
:109D24002BFBE435F0FC7A3C125D96EB28FBE43C1B
:109D3400FC22AC3DAB3EA83F80E178AE8604AB3E4E
:109D4400E53FC313F8800C7800121857E5BE75F090
:109D540005A4FBE5BF75F03CA42BFBE435F0FC7ACD
:109D64001E125D96EB28FBE43CFC22129D4BAE04D4
:109D7400AD03129D3E8C148B13121861E5BFFF24B2
:109D8400F650027F01E5BE75F096A4AAF0F9C3ED82
:109D94009513FBEE9514FC924E4B701120110E306E
:109DA400480B75364B3003037536FFD22E304E0206
:109DB400DF1F7A02125D9675A7009004EEECF0A303
:109DC400EBF0C3E5BF9F04BF0102D2E79005CBF0DF
:049DD40022ED29FD56
:059DD800EE3AFE80B52B
:10F1340012F13D12F13D12F13D7E0480067E028003
:10F14400027E017F0080087F6480027F017E00EFE1
:10F154004E6012E4FD0D1D0DEDC394AD40F7EF1F9D
:10F1640070ED1E80EA2212F2FC90C0097F00128129
:10F174003712F18512F13D753500C200C201C20299
:01F184002268
:10F2E800F5D8D2DCE5F520E7FBE5DA540FFEAFD917
:04F2F80075D80022A3
:10EEF0007F767E0690B6FD128149740412F2E87C9A
:10EF0000007D52125EA2EFF875F00A84C0F07F76A1
:10EF10007E2312E8D37E29742E12E8E67E2ED0E0FE
:10EF200012E8D37E35745612E8E67F6B7E1190EFBF
:10EF30005912E912E824E04001220423F824E750A2
:10EF400002781812EF49D8FB227F6CE82411FE7971
:10EF50000512F2170E0FD9F922071DFFFFFFE080FF
:10EF6000000020C0000038E0000008F0000038F881
:07EF7000000020FFFFFFE09D
:10EFF40012F01C30E6022409540F75F00AA4F5152A
:10F0040012F01C30E6022409540F25152212F01CBC
:10F01400540F2275F000800875F044800375F007E2
:10F02400E4206D09D5E0FAD5F0F7D24C229247C21C
:10F03400ACE54F623885504FA26E926D859950C2EF
:10F044006FD2ACC24CA2472212F056C4FA12F05648
:10F054002A2212F01C20E603540F2254072409220A
:10EF7700E612EF7E18E608FAC412EF84EA540F444B
:10EF870030F924C6E950112407800D75F00A84C0B2
:10EF9700F012EF9DD0E0443030530975F00085E062
:10EFA700E0D5F0FA3099FD75F019D5F0FDC299F565
:10EFB70099623822E53880EC742A12EFAB6238E5A3
:10EFC7003812EF7E800812EF9FE53812EF9F740D1D
:10EFD70012EF9F740A80C1744012EF9F744080B88B
:0DEFE700742C80B4742E80B075380080AB9F
:10F30E0085A0835383FE438380858384F0758400B8
:01F31E0022CC
:10ED9D0074A212F30E74A112F30E74A612F30E7474
:10EDAD00A412F30E74C012F30E742512F30E12EEAC
:10EDBD002E75C70375C6FC75B90112AA63740812C6
:10EDCD00F2E8EE75F020A4FEEF54F80303032E24B1
:10EDDD0092C313FE24EA50027E16EE90EE17932591
:10EDED00BCFE24E6502024E8401C748112F30EEE84
:10EDFD0012F30E12EE3B744012F30E742F12F30E3B
:10EE0D0074AF12F30E227E2680E0F7F7F8F8F9FAC8
:10EE1D00FBFCFDFEFF0000000001010202020303E6
:10EE2D0003A8BCA9BDAABEABBFACC7ADC62288BCEA
:0BEE3D0089BD8ABE8BBF8CC78DC6222A
:10F18500C006C007C5F075A7019000007EB7E58CE5
:10F19500240340FA12F1A71EBEAFF3C5F0D007D085
:10F1A500062275A700EE12F30E741012F30E740406
:10F1B50012F30E85A08343838185838475A7517FD0
:10F1C50020E0F0E0F0E0F0E0F0DFF6E4F5A7F5840C
:01F1D5002217
:10F2FC0075A711900000E4C583F0C58330E2F8F5E2
:02F30C00A72236
:10F21700EF20E723EE20E71F20E61C05A7C45403D1
:10F22700F583EE5408C42FF582EE5407240983F5BD
:10F23700F0E045F0F005A722804020100804020105
:10F24700EF20E723EE20E71F20E61C05A7C45403A1
:10F25700F583EE5408C42FF582EE5407240983F58D
:10F26700F0E055F0F005A7227FBFDFEFF7FBFDFECB
:10E89100FDA42582F582E5F03583F583ED227E0026
:10E8A100906AE57A0475F00512E8917D05805E7A3B
:10E8B1000580027A04547FC0E0C083C082C39420E3
:10E8C1005001E4906A9512E8A6802E906BF37A05C8
:10E8D1008005906CB07A0675F00712E8917D07808B
:10E8E1002C7A0580027A06C0E0C083C082C39420DE
:10E8F1005001E4906C4012E8D8D082D083D0E0225D
:10E90100906A0975F00A12E8917D0A7A07C2D180EE
:10E9110002D2D1C0A7C082C083C007C006C0E03008
:10E92100D10975A704E493FDE493FAEEFB75A704FE
:10E93100EBFEEAFC7901D9067908E493F5D4E5D434
:10E9410023F5D420E01612F2470EDCEA0FDDE1D008
:10E95100E0D006D007D083D082D0A72212F2178050
:10E96100E890694975F00E12E8917D0E7A0812E976
:10E971000E9069F175F00212E891E493FDE4A3931E
:10E98100FACE2408CE7C0812E98F7C06AD02ED2375
:10E99100FD20E00712F2470FDCF42212F21780F794
:10E77C00F5D2C2D58036F5D2D2D58030F5D224F67A
:10E78C0050090E0E24A650030E0E0EE5D2F5D275CE
:10E79C00F0648485F0D3C2D57009D2D5742012E808
:10E7AC00E6800312E8D3CE2406CEE5D375F00A84B6
:10E7BC0085F0D3700A30D507742012E8E680031276
:10E7CC00E8D3CE2406CEE5D312E8D3E5D222F5D297
:10E7DC0075F0648485F0D3C2D58022F5D2C2D58081
:10E7EC0025F5D2D2D5801FF5D275F0648485F0D38F
:10E7FC00C2D57009D2D5742012E8E6800312E8CC99
:10E80C00CE2405CEE5D375F00A8485F0D3700A309A
:10E81C00D507742012E8E6800312E8CCCE2405CE8E
:10E82C00E5D312E8CCE5D222F5D2C2D58035F5D2AB
:10E83C00D2D5802F30E70DF404C0E0742D12E8B46B
:10E84C000E0ED0E0F5D275F0648485F0D3C2D5708D
:10E85C0009D2D5742012E8B4800312E8A1CE2404A6
:10E86C00CEE5D375F00A8485F0D3700A30D50774E1
:10E87C002012E8B4800312E8A1CE2404CEE5D31212
:05E88C00E8A1E5D22225
:10812E0090B9F312813702F1857E00800E7405FE40
:10813E00F51EE4FFF51DF51F203C3375A700E493F3
:10814E00700122A3B40204051D8003B4010A051FA9
:10815E00EF2409FFAE1E80E612E8E67D06B440026B
:10816E007D03B421027D02EE2DFE80D27E0075A726
:10817E0000E493700122A3B40204051D8003B40130
:10818E000F051FEF2407FFAE1E80E612E8B0800831
:10819E00B45B0050F612E8B40EB4210280D30EB4D4
:1081AE00400280CDB42C0280C80E0EB45F0280C196
:1081BE00B45B0040BC0E80B9E60812E8E6EE240679
:1081CE00FED513F42290B72B30740990B72F30736D
:1081DE000390B73402814975F019D5E0FDD5F0FA58
:1081EE0012545712EFDE744F12EFEF744B12EFCDA5
:1081FE00C322C250128244125457D2AC12F017301E
:10820E004C1212F017304C0C12F017304C06D250A4
:10821E00C2ACD322B440E512F01CB4400312F01CE1
:10822E00B44FED12F01CB44BE712F01C12F01C12FE
:10823E00F01CC2ACC32230530975F008D5E0FDD551
:10824E00F0FA227F0575F019D5E0FDD5F0FA12543B
:10825E005712EFDE745712EFEF745012EF9F7481C6
:0A826E0012EF9FE56312EF9FE56237
:1082780012EF9F78D0E612EF9F08B8D7F8E6F879A2
:108288005F30E702792FE912EF9F12EF9F12EF9FFD
:1082980012EF9F745812EF9F744312EF9FE412EF8E
:1082A8009FE8C2E775F00A84C425F012EF9F78644E
:1082B800E612EF9F08B869F8E612EFCD1282004087
:1082C8000122DF02800A20508B75F0008080D25096
:1082D800C2ACD322128244C250125457D2AC2002EC
:1082E800EF12F017204CE7B440F412F01CB440032E
:1082F80012F01CB457DAF53812F01CB450D212F050
:108308001C12F01CF56312F01CF56278D012F01CF8
:10831800F924A0500353015FE924E04002795FA6E5
:108328000108B8D8E8780612F01CD8FB12F01CFC3B
:1083380053040FC4540F75F00AA42CFC249C50025B
:108348007C0078D78601E4B92F02D2E72CF678644E
:1083580012F01CF608B86AF812F01CE5386003023F
:1083680082D812F01C12F01CC2ACC32290BED1807D
:108378000390BA397F2012817A12F18502F145758E
:108388003400C26B12844312F1451287FAE5166075
:108398000312839F020211128A4F12287312F18569
:1083A80010002010010280F8128865501312287EF0
:1083B80012837410000D10010280F812281980D75A
:0483C8001285E62212
:1083CC00C26BD22775480A12384B753400128925B6
:1083DC00C26A123FDD106A0512020280ED1202021F
:1083EC0012878C1288E412893178D0E664266044B6
:1083FC00128A4F12287312F1851000381001028076
:10840C00F8128865501BE96515601812287E1283D6
:10841C007412F13D10001D10010280F81228198011
:10842C00BCD26B1289107516078559171238C47592
:10843C00350080960202111287FA12846512893176
:10844C007F1912847F90BEFF7E1212817C7E23E501
:10845C001602E85090C04A80EF7862E41284767875
:10846C00D0745F12847618E4F6227F08F608DFFCDD
:10847C00227F7B7E007810742012E8B4CE2404FE98
:10848C00D8F5221220C37F197E0812817C7E289099
:10849C00BA2430530390BA1F02817CC26B128465DC
:1084AC001284B2020211C25112893190BEF61284AA
:1084BC008F12283F1287FA7F2012844E12F185E525
:1084CC0016700512F13A803675A6FF3051031281F1
:1084DC00EE125457D2AC200025306DFA1282DF40D8
:1084EC000C12886540111285E6D25180BB105003E6
:1084FC00128379C25180D1D25112837480CAC2AC1A
:10850C0022D22775480A12384B753400C26B128977
:10851C0025C26A123FDD106A0512020280EB1202BC
:0F852C000212878C1288E412893112853E50DAD0
:10853B0002021190BA3412848F12285812F185C39B
:10854B0010001310010510020E80F412825140012D
:10855B002212837980DDD3C2AC22D227C26B75483D
:10856B000A12384B753400128925C26A123FDD108E
:10857B006A0512020280EDD26B12878C1288E4120C
:10858B0087B475B901E5BCB2E7F5BC1255F77516A2
:10859B00078559171238C480CB1287FAE516601F6E
:1085AB0078D0E53D1285D7E53E1285D7E53F12859C
:1085BB00D7765A08765F12DB841289100287CB7F3D
:1085CB003E7E1190BA0A12814902F18575F00A8438
:1085DB004430F608E5F04430F60822D26B128910CD
:1085EB001287CBE51775F01084240AF54824E85060
:1085FB000375480A12385785585922D22075320014
:10860B00129B5A75A7049007007515001287B47555
:10861B00B901E5BC20E705E515F0801004600D6499
:10862B0082600975BCFF75B90575B9020515E515AD
:10863B00242050D8E58224FE40030286E1A882184C
:10864B007F0075A7007583078882E0FE75F004A490
:10865B0012875FA9BCAABDABBEACBF1582E0FD758E
:10866B00F004A412875FC3E995BC404C7052EA95A5
:0D867B00BD4045704BEB95BE403E7044EC99
:1086880095BF4037703DEE75F004A40412875FA9CA
:10869800BCAABDABBEACBFED75F004A40412875FE5
:1086A800C3E995BC4015701BEA95BD400E7014EBEC
:1086B80095BE4007700DEC95BF5008EEF00582EDB1
:1086C800F01582E5826009C3EF9582500302865552
:1086D8000FC3E89F400302864D75A70490070075F5
:1086E800C70375C6A8E0F5BCE0F5BDE0F5BEE0F54A
:1086F800BF75B90575B90205C6E58224204006E5AF
:10870800C6242050E00875C70375C68075B901E511
:10871800BC128749F5BCE5BD128749F5BDE5BE1217
:108728008749F5BEE5BF128749F5BF75B90205C689
:10873800E5C6245850D6E5320470FB75A700C22060
:1087480022B4FF0122F975A704900700E58268604A
:1087580005E06970F7E922F5C685F0C775B901E546
:10876800BC645F700375BC27E5BD645F700375BDAD
:1087780027E5BE645F700375BE27E5BF645F7003BD
:1087880075BF272275C703E54875F004A42480F552
:10879800C6E55975F00484A8F00825C6F5C675B96C
:0787A80001A9BCAABDABBE94
:1087AF00ACBF861522E515242050037515DFE5159E
:1087BF0075F004A454FCF5C685F0C722E5172420F4
:1087CF004028E51775F00484A8F00824A8F5C675AD
:1087DF00C70375B901A9BCAABDABBEACBFA61589AD
:1087EF00BC8ABD8BBE8CBF1255F722E4F516F5156A
:1087FF0079FF1287B475B901E5BCB4FF040516A95A
:10880F00150515E515242050E9891579FF75C7035E
:10881F0075C6A875B90109E5BC04601B09E5BD045F
:10882F00601509E5BE04600F09E5BF04600905C6C0
:10883F00E5C6242050DD098917227516007515012C
:10884F001287B475B901E5BC20E70205160515E5D9
:10885F0015242050EB227900E975F004A454FCF59F
:10886F00C685F0C775B901E5BC20E73078D06670D2
:10887F002B08E5BD66702508E5BE66701F08E5BFCD
:10888F0066701905C675B90108E5BC66700E08E576
:10889F00BD66700808E5BE667002D32209E9242080
:1088AF0050B6C3221288D31288BBA8017F08E0F606
:0C88BF0008DFFB221288D31288CBA8012E
:1088CB007F08E6F008DFFB2278D0796275A7047584
:1088DB008307EBC454F0F582221287B478D0128848
:1088EB00FEE5BCF9C23C20E702D23C1288FE78625E
:1088FB001288FE75B901A6BC08A6BD08A6BE08A6BF
:10890B00BF0805C622D2201287B478D012811C1260
:10891B00811C786212811C02811C12646F12F2FCA2
:10892B00129F2502F18512F2FC7F007E0990BEE3B7
:10893B001281497F0A7E12E5150412E7887F141213
:10894B00DD751228197F277E0875130778D01281E1
:10895B00C6E6793E30E702792F7E34E912E8E67FEE
:10896B003D7E0190C06612817C20311B303003129A
:10897B00C20CC23B128BE1128997D23B128BE112D4
:10898B0089A9128C28807C12D3F180E6C23B7F44EC
:10899B007453201702744E7E0012E8E68017D23B08
:1089AB007F4F745720170274457E0012E8E67E064F
:1089BB00E51E12E8D37E0CE51D12E8D37E12E51CF2
:1089CB0012E8D37E17748112E8E67E1CE51B12E8D1
:1089DB00D37E22E51A12E8D37E28742E3026027439
:1089EB002712E8E67E2DE51912E8D37E33E518123F
:1089FB00E8D37E39302607742C12E8E27E3BE5374C
:108A0B0002E8D3742D201702742B7F707E1512E8A9
:068A1B00E6128A2C7E3AEF
:108A210012E7317E0190C0910281497E1BE51C1243
:108A3100E8D37E21E51B12E8D37E27E51A12E8D39D
:108A41007E2DE51912E8D37E33E51802E8D3128AA8
:108A5100CD128AF8128DCF128931128E2720171E5E
:108A610010021B12B23B12DB84128AB51228247F3A
:108A7100347E2F1281D312896A12F18580E2122885
:108A810019203026203128C23B128BE1128B0D7840
:108A910066128CE1D23B128BE1128B227869128C27
:108AA100E1128C28128B9C028D8412C2D580F212A5
:108AB100D40680EDE57D75F01084AAF075F00AA466
:108AC1002A547FFA78D7E654802AF6227F277E0837
:108AD10079D08700C001D224B9D002C224128EAE4F
:108AE100D001A70010230909EE2406FEB9D7E3221D
:108AF10019EE24FAFE80DB7E3479D7E7A2E79217DC
:108B0100128E5B79D7E7A21792E7F722C224C23B04
:108B1100751E007F447E00128E6B801E1023ED8037
:108B21002AD23BC2247F4F7E00128E73D2247E064E
:108B3100E51E128EA0F51E1023E7D2247E0CE51D42
:108B4100128EA0F51D303BD41023E1D2247E12E514
:108B51001C128EA0F51C1023E17E1CE51B128EA0B9
:108B6100F51B1023E67E22E51A128EA0F51A1023BA
:038B7100E87E2D6E
:108B7400E519128EA0F5191023E87E33E518128E3C
:108B8400A0F5181023E87E393026027E3BE5371223
:108B94008EA0F5371023E3227F707E15128E63C2F8
:108BA400247E1BE51C128EA0F51CD2247E21E51B1D
:108BB400128EA0F51B1023E77E27E51A128EA0F56E
:108BC4001A1023E67E2DE519128EA0F5191023E85C
:108BD4007E33E518128EA0F5181023E82278D7E624
:108BE400C2E775F00A847866F537303B0578698505
:108BF400F037128C5130262BE53775F003A40404AA
:108C040075F00584FBE51975F00AA4251875F006BE
:108C1400A42BFBE435F0FC125FBEF537125FBEF502
:108C2400188B1922E563FC339217AB625003126070
:108C34002F305C0A7AD2125DA47840125F46AE04EB
:108C4400AF037C277D10125EAF8F1C8037E6FD33A7
:108C5400921718860418860350031260377A09792C
:108C64002778C0125F438B1EADD3ACD2AB0679EA32
:108C74007860125F418B1DAF06AED27C177D7012F7
:108C84005EAF8F1CAF05AE047C037DE8125EAF8F30
:108C94001BAF05AE047C007D64125EAF8F1AED75C8
:0A8CA400F00A84F51985F01822EC9F
:108CAE00339217500312602F751D30301786751DC5
:108CBE002D808178427B607CEA800678407B207C28
:108CCE004E12D4D179277810125F418B1CAF06AEAD
:108CDE00D280AB30262AE51975F00AA4251875F056
:108CEE000AA42537FBE435F0FC7A05125D968C0656
:108CFE008B077C007D03125EA28E048F03128C1BE9
:108D0E00E51E75F00AA4251D75F00AA4251C75F044
:108D1E0006A4251BFBE435F0FC7A0A125D96EB25C2
:108D2E001AFBE43CFC7A0A125DA4EB2519FBE43C29
:108D3E00FCE43DFD7A0A125DB6EB2518FBE43CFC23
:108D4E00E43DFD301703126037A60518A60418A6D9
:108D5E000378D7E6A2E7923DC2E775F00A84FCAB32
:108D6E00F0303B0EAB37EC75F00AA42BA23D92E728
:108D7E00F622AC3780F0128D9F305C0A7A40125D7D
:108D8E00A478D2125F4630170312602F8C638B6269
:108D9E0022128DAF7A0A125D96EB2518FBE43CFC8D
:108DAE0022E51C75F00AA4251B75F00AA4251AFBF2
:068DBE00E435F0FC7A0A26
:108DC400125D96EB2519FBE43CFC22128E0112F194
:108DD40041C202C223128E011000081001051002C4
:108DE4001B80F51031ED10300D102604D22680E3DF
:108DF400D230C23180DDD231C23080D7227F35906B
:108E0400C04F12817A90C06D20300F90C0892031FC
:108E14000990C05E20260390C0561F7E1712814918
:108E240002F1857F357E0190B9E612817C7F347E24
:108E34003A128F50744E12E8E612F18512F141C2D3
:108E4400027F347E3AD21775115975124E802675F9
:108E5400112E751227801E75113E75122F801675FE
:108E6400112B75122D800E75114E751253800675D7
:108E74001145751257128F50E511301702E5121281
:108E8400E8E612F18510000810010510020B80F5C8
:108E9400D23C1017E3D21780DF028F4B4430F81214
:108EA4008EAAE8540F22C2218002D221A224922247
:108EB4009223128F50E830E709D23C7430302102FB
:108EC400745FF812E8E612F1851000341001051001
:108ED400025D80F5D23C102266102367B439097410
:108EE4005F2021DF743080DBB45F04742D80D4B440
:108EF4002D04744180CDB45A04743080C60480C3F8
:108F0400D23C302406102237102338B44104742D87
:108F140080B1B42D04745F80AAB45F04743980A353
:058F2400B43009745A8D
:108F290020219B74398097148094B48908D223E84E
:108F390012E8E6800DF8C223800874898001E802EE
:108F49008EC7908F9A8003908F96C007EF2408FFF1
:108F590012E912D00702F185128F50E830E704D2E6
:108F69003C7441F812E8E612F1851000081001116D
:108F79001002CF80F5D23CB44104745A80E51480C4
:108F8900E2D23CB45A04744180D90480D60205F86F
:058F9900F802050000D4
:10F0D40075A70090F10675F02D84C2D5C2D16017D2
:10F0E400D2D1146007D2D514600DC2D1E5F093FCDF
:10F0F400742D95F093FB22E5F093FB742D95F0931A
:10F10400FC220009121B242C353E474F58606870BE
:10F114007880888F969DA4ABB2B8BEC4CACFD4D928
:10F12400DEE2E6EAEDF0F3F6F8FAFCFDFEFFFFFF9F
:10F1D600D23D8002C23DED8BF0A430E70205F0C3BC
:10F1E600E895F020D50425F025F0FEED8CF0A4304E
:10F1F600E70205F0C3E995F030D10425F025F0FFCC
:10F20600203D0B2487500122EF24CC40012202F23C
:01F2160017E0
:10EB6200203A7A7E1C7F5312F2177F5912F2171E37
:10EB72007F5712F2177F5512F2177E2312F2177F78
:10EB82005712F2171E7F5912F2177F5312F2171FF4
:10EB92007E2012F2177F5A12F2177E1E12F2177F90
:10EBA2005212F217121861E5BD20E0143006117FEF
:10EBB200357E1C90EC20E571700390EC2A02E9127C
:10EBC200E5716018E57012F0D4781F79567D09124C
:10EBD200F1DA303A0312EBF30DBD16F3227E1C7FFD
:10EBE2005390EC0912E912200CD67E1F12DDDC8054
:10EBF200BEC0060E30D5021E1E12F217D0061F30FE
:10EC0200D1020F0F02F217070700386C446C38006C
:10EC120005052070D8702005057088A8887008073F
:10EC220010387CFE383838000807102844C62828D7
:02EC32003800A8
:10DBB00090C09B7F717E2312817C121861E5BC7E30
:10DBC0003112E8A130121AC23C121861E5BCFB7593
:10DBD000F00AA4F904FAC23D12993912DE53303D1D
:10DBE0000122DAF712DD557C00EBF4042E4019AD6A
:10DBF00003125EA2EFA2D1203C077E237F6502E4E0
:10DC0000FEAE16AF1702DCF6AD01125EA2EF12E512
:10DC1000EC203C077E237F6502E522AE16AF17029B
:10DC2000DD1A7F567E0512DD817F3D12DD947F6F08
:10DC300012DD9412DDDC7E0A7F4112DE0F7E227F30
:10DC40005912DE0F20120122129939857A1D855E44
:10DC50001C857B1B855F1A7AC0C23D12DE4F203DBA
:10DC60005212DD557C007D14125EA274562F20D115
:10DC7000029F9FFF24CB40028037EF248850028010
:10DC800030EA1475F00384FE12F217C3E51B957B8E
:10DC9000FEE51A955F92D55004EEF404FEEEC31330
:10DCA000FE24E0400C741F2E30D5029E9EFE12F220
:10DCB00017DAA8227F5212DCC67F5A12DCC675170B
:10DCC00053751600802B7E0012F2470EBE12F92209
:10DCD0007F157E28742012E8E67F1C7E2812F2470A
:04DCE0000EBE40F93B
:10DCE400223012E712DCD075171575162DD23C02BE
:10DCF400DBC9C23D6002D23D92D175F080305C0434
:10DD0400F5F08001A4A2E792D5E5F075F03284F82D
:10DD1400E5F075F00584C0E0E5F0A2D533C0E0E895
:10DD2400601E12E8D3EE2406FED0E0F8D0E012E83C
:10DD3400D3EE2406FE742C12E8E60E0EE802E8D3B5
:10DD44007420303D07742B20D102742D12E8E68034
:10DD5400D4C3ED957AFFEC955EFE92D15003126028
:10DD64001F227F1512DD6D7F327E3E12F217DEFB1D
:10DD7400227E0912F2170EBE36F9227E0112F21724
:10DD84000E0EBE3FF8227E3312F2170EBE40F92269
:10DD94007E047D1112F2170E0E0EDDF81F1F7E3564
:10DDA40090C0A4305C057E3190C0A802817C7405CB
:10DDB400305C097E32740112E8A174067E3612E8E2
:10DDC400A17E3A740012E8A17E3D02E8A17F1512FB
:10DDD400F2170F0FBF2DF8227F417E1F7D0F12F225
:10DDE400170F0F0FDDF8227F687D0380047F677DA6
:10DDF4000512F2170FDDFA227F667D0780F37E1F7E
:07DE04007F5012F2171F1FEF
:10DE0B00BF3EF8227D0A12F2170E0E0F0FDDF7221E
:10DE1B00203D071248B47003D23D22056D12B1911B
:10DE2B00E4F5F7E4ABF7F5F7E4E5F7FA30E411EBDB
:10DE3B00251DF51DE4351CF51C0519EA30E3010E13
:10DE4B00D2B28015780380027801203D071248B4C6
:10DE5B007003D23D22D8F3056DE56D2409F56D12E3
:10DE6B00B191E4F5F7E4ADF7F5F7E485F71BF5F7BA
:10DE7B00E4E5F7FCD2B2543F30E50244C0CC54C0C9
:0BDE8B002323F51AE56D24F6F56D2247
:10EA89007E017F0990EB0712E9122051097E037F6D
:10EA990000743F02E8E6E4FEFFC3E54512E327FD03
:10EAA900940AED403D9464ED4002746312E7827E5E
:10EAB900017F09E552240575F02D84AAF075F0054A
:10EAC900A4CA75F00B842A90EAF29312F0D4BCB868
:10EAD900027BB87D04EE2DF8EF2DF90D12F1D6DD8C
:10EAE900FB227E0312E8D380C6000C1622222D39A0
:10EAF900444F4F5A66707C7C87939EA9A9000909E7
:10EB0900080041000000000088800000000041006A
:10EB19000800121875E5BCB4F8339004C3E0602C02
:10EB2900FA24F340277F137E0012F2170F0F12F217
:10EB3900170E12F2471F1F12F2470EDAEC7F147EEE
:10EB49000012F2170E12F2470EBE12F5229005CCF2
:09EB5900E0C3941240F60480C7E9
:10E32700305D0A75F08AA42480E5F0340022207459
:10E33700157F017E1190E3AF12E9127F0A7E0AE58D
:10E347002E540702E7997F087E1190E3BF12E91266
:10E3570020730C7F0A7E1712F2470E0E12F2477FC8
:10E36700007E0BE57112E32712E7887F0C7E11E52B
:10E3770071602F0EE57064B4602864B475F0328460
:10E38700C0F012E8CCCE2405CED0E075F00584C0ED
:10E39700F012E8CCCE2405CED0E023302D010402C4
:10E3A700E8CC90A121028149070FFFFFC473BDAFDD
:10E3B700A463B5FBCDE7FFFF030F0100FFFE03805A
:10E3C700306701227F3F7E00748812E8E6E55160DE
:10E3D700F212187A85BCF01207A512E32775F064CC
:10E3E70084F87E06E5F012E7E7E860D77E0002E8EA
:10E3F700D312187AE5BE70012214600814603BE559
:10E407003F1340367F367E00747712E8E6207301AB
:10E417002279BC8704098703125D3E7E05781DE6D5
:10E4270060097E0012E8CCEE2405FE18E6600712AC
:10E43700E8CCEE2405FE18E6801990B8B97F377E40
:10E447000012817CAB60AC61125D411F7E09781DB3
:10E45700E6600712E8CCEE2405FE18E612E8CCEEDB
:03E467002405FE8B
:10E46A0018E602E8CC202C012290E47902E9120590
:10E47A000EFFF0E01CF004F81CFFF0301201227FBE
:10E48A00637E0090B74612E9127F1512DD6D7F1F79
:10E49A0012DD6D7F2912DD6D7F177E06E53F30E0C4
:10E4AA000B90C0B8305C0390C0CC800990C0AD30EE
:10E4BA005D0390C0C21281497F2190B77220740611
:10E4CA0090B766028137E53770F9E53F20E0F4300E
:10E4DA0073F190B77E1281377E1BAC4EAB4D12E6BC
:04E4EA00AD02E73167
:10E65400125D3E7F207E05751900781DC2D5E63017
:10E66400D51712E8CCEE2405FE18B818F17E1F74F5
:10E6740063305C02748202E8E67005B8191880E21F
:10E68400D2D5CE24FACE7484301702742D12E8E663
:10E69400EE2406FE80C8742012E8E280C8781C804C
:10E6A4000D7F007E23AC5EAB7A125D3E781DC2D531
:10E6B400E630D50C12E8D3EE2406FE18B818F12281
:10E6C4007005B8191680EDD2D53017E4CE24FACEF1
:10E6D400742D12E8E6EE2406FE80D5742012E8E6D6
:10E6E40080D5125D3E781DC2D5E630D51612E8A15C
:10E6F400EE2404FE18B818F10E745E305C02742720
:10E7040002E8B07005B8191680E3D2D53017DACE16
:10E7140024FCCE742D12E8B4EE2404FE80CB7420C5
:10E7240012E8B480CBC23D12E73C0F0F0E0E7463A7
:10E73400305C02748202E8E6125D3E781DC2D5E6C2
:10E7440030D50C12E901EE2408FE18B818F1227035
:10E7540005B8191680EDD2D5301716740BCE24F8EF
:10E76400CE12E901EE2408FE80D5740C12E9018072
:08E77400D5303DCB740A80E5AD
:10EC34007F797E24E55F30E70122AC5F1CAB7B1259
:10EC44005D6CE51B700E742012E8E6EE2405FE12DE
:10EC5400EC82800C12EC82E51B12E8CCEE2405FE5B
:10EC6400E51A12E8CCEE2405FE742C12E8E60E0E2A
:10EC7400E51912E8CCEE2405FE745E02E8E6742D74
:10EC8400201702742B12E8E6EE2406FE22E55F301C
:10EC9400E70122AC5F1CAB7B125D6CE51B700E744C
:10ECA4002012E8B4EE2404FE12ECDB800C12ECDB40
:10ECB400E51B12E8A1EE2404FEE51A12E8A1EE24F5
:10ECC40004FE742C12E8B40E0EE51912E8A1EE2429
:10ECD40004FE742A02E8B4742D201702742B12E87F
:06ECE400B4EE2404FE2240
:10E4EE007F097E2530040512E5E88028A275E579BE
:10E4FE00C23D6002D23D92D175F080305C04F5F0E1
:10E50E008001A4A2E792D5E5F075F03284F8E5F02B
:10E51E0075F00584C0E0E5F0A2D533C0E0E8602ACE
:10E52E0012E901EE2408FED0E0F8D0E012E901EE87
:10E53E002408FE0F0FE52B5403701F746012E8E6DB
:10E54E001F1FEE2404FEE802E901740C303D067430
:10E55E000A20D1010412E90180C9205904742E80C9
:10E56E00DC205804747F80D5748080D1300405126D
:10E57E00E5E88028A275E579C23D6002D23D92D1D0
:10E58E0075F080305C04F5F08001A4A2E792D5E529
:10E59E00F075F03284F8E5F075F00584C0E0E5F032
:10E5AE00A2D533C0E07F3E7E1CE8602012E962D027
:10E5BE00E0F8D0E07F3E7E2812E9627F447E32741E
:10E5CE002E12E8E67F3E7E37E802E962303DE074C7
:10E5DE000A20D1010412E96280D59005CAE075F0D7
:10E5EE000A84F8E4C5F0C2D522301105E54AB4021A
:10E5FE0050C39006E9E0957AFB9006E8E0955EFC44
:06E60E00500312602FEC26
:10E61400C31360047B63800FEB13FB249C40F5243D
:10E624004F4004C20480079005CAEBF0D204900660
:10E63400E6E09006E8F09006E7E09006E9F0E55E93
:10E644009006E6F0E57A9006E7F02212E63280DEE4
:10DE9600E54424F64001227800E552206607C39542
:10DEA60070500224B40475F00384F9E928FE24C4F2
:10DEB6005001FE12DED812DEE41E12F217C3E998F4
:10DEC600FE5003243CFE12DED81E12F21708B81FBD
:10DED600DA22EE2420FE24C250032402FE22E82485
:10DEE600F1E8C2D55006D2D5E8F4241F23FF90DF0F
:10DEF6006693CF0493FAE545F5F0A4ACF0FB125D0A
:10DF0600CDE544F5F0A49BFBE5F09CFCEB2420FB5F
:10DF1600EC3400FC12DF47FAE5458FF0A430E70247
:10DF260005F0E5F020D502F4042A75F00520190362
:10DF360075F00384FF24DF50027F20C374329FFFF5
:10DF460022EC24F0500BEB2460EC340090DFB69307
:10DF560022EB33FBEC33FCEB33EC3390DF8693227E
:10DF6600FF00FF03FA0BF318EA2ADE40CF58BE7310
:10DF7600AB8D96A880C068D64FE835F51BFD00FF2F
:10DF860000080B0E101214151718191B1C1D1E1F46
:10DF960020212223242526262728292A2A2B2C2D10
:10DFA6002D2E2F2F30313132333334343536363748
:10DFB600373839393A3A3B3B3C3C3D3D3E3E3F3FA4
:10DFC6004042444648494B4D4E5052535556585977
:10DFD6005B5C5D5F60616364656668696A6B6D6EF4
:10DFE6006F7071727374767778797A7B7C7D7E7FB9
:10DFF600808182838485868788898A8B8B8C8D8EA7
:10E006008F9091929394949596979899999A9B9CB0
:10E016009D9E9E9FA0A1A2A2A3A4A5A6A6A7A8A9CD
:10E02600A9AAABACACADAEAFAFB0B1B1B2B3B4B4FC
:10E03600B5B6B6B7B8B9B9BABBBBBCBDBDBEBFBF36
:10E04600C0C1C1C2C3C3C4C5C5C6C7C7C8C8C9CA7B
:10E05600CACBCCCCCDCECECFCFD0D1D1D2D2D3D4C9
:10E06600D4D5D5D6D7D7D8D8D9DADADBDBDCDDDD1F
:10E07600DEDEDFDFE0E1E1E2E2E3E3E4E5E5E6E67A
:10E08600E7E7E8E8E9EAEAEBEBECECEDEDEEEEEFDC
:10E09600EFF0F1F1F2F2F3F3F4F4F5F5F6F6F7F743
:10E0A600F8F8F9F9FAFAFBFBFCFCFDFDFEFEFFFFB2
:10E0B600E54524FD400122E552206607C3957050D0
:10E0C6000224B40475F00384241FFE24C2500324E2
:01E0D6000247
:10E0D700FE12DDD1EEFD241EFE24C250032402FEF3
:10E0E70012DDD1E544240275F00520190375F0030C
:10E0F70084F4042432FF24EE500F12E106AE051E0D
:0AE107001E7C0512F2170EDCFA224E
:10E9A1007E00206615E5700475F0B484E5F075F01D
:10E9B1000384FE6004C3743C9EFE745312E9CC745C
:10E9C1005712E9CC744E12E9CC74457F2F12E8B48A
:10E9D100BE00077E3C12E8B47E00EE240875F03CD0
:10E9E10084AEF00F0F0F12F2170E12F2170F12F280
:10E9F100171E12F217EE240775F03C84AEF0223098
:10EA0100745C301259E54AB4040122B4060122E5CE
:10EA11007112DF308F057C037E1E30662AE570049B
:10EA210075F00384241EFE24C6501C24FB500424CC
:10EA3100038013C00612EA48D0E024C67C016006B8
:10EA41000C1460020C14FE12EA540EEE24C14002B2
:10EA5100DCF5228D0712F2170FEF24CE50F722E5D5
:10EA610053206607C39570500224B40475F00384E3
:10EA7100241FFE24C250032402FE12EA7F0E7F23CC
:08EA810012F2170FBF2DF9225C
:10F277007E0E78ADE612E7E7EE2405FE742C12E861
:10F28700E60E0E0E18E612E7E7EE2405FE742C12C2
:0AF29700E8E60E0E0E18E602E7E7A7
:10E111007F017E00745212E8E67E06E51512E7EDF6
:10E121007F0A7E0178B8E67D0130E5027D03ED12BC
:10E13100E8D37E07E67D58A2E4922B50027D46ED9E
:10E1410012E8E67F017E1812F2797F0A7E1378AE1B
:10E15100E612E77CEE2406FE743A12E8E6EE2405A8
:10E16100FEE53E12E77CEE2406FE743A12E8E6EE86
:10E171002405FEE53F02E77C7F797E00E54012E75A
:10E18100E77E0A743B12E8E27E0CE54102E7E77F95
:10E19100797E16743B12E8E27E18E53F12E7E77FCD
:10E1A100797E0078AEE612E7E77E0A743B12E8E278
:10E1B1007E0CE53E02E7E7305EE52043E27F6D7EBF
:10E1C1000078AEE612E7E77E0A743B12E8E27E0CC5
:10E1D100E53E12E7E77F757E00E53E75F00A84E5CE
:10E1E100F012E9010F0F7E08743A12E8E21F1F7E58
:10E1F1000DE53F75F00A84C0F012E901EE2408FE36
:10E20100D0E002E901851C1E851B1FAB1BAC1C3035
:10E211005D0A7A1B125DA47832125F46C3EB33FBB1
:10E22100EC33FC923D125D75303D087409F51DF526
:10E231001CF51B7F75E51D60157E2412E9017E2CFE
:02E24100E51CDA
:10E2430012E9017E34E51B12E901803D7E22E51CC3
:10E25300601912E9017E2AE51B12E9017F787E31FC
:10E26300742E12E8E27F75E51A8019E51B12E901A5
:10E273007F787E29742E12E8E27F757E2DE51A12CF
:10E28300E901E5197E3512E9017F777E3C126705C6
:10E29300851E1C851F1B227F397E1F12F2170FBF9D
:10E2A30040F9781F79567A007D1A12F0D412F1DA08
:10E2B300EA2406FABAAEF3781BC3E511957050024F
:10E2C30024B4FA604214603E14603A2450603A1455
:10E2D3006036EA24A540278A1E751D007D1912E2C7
:10E2E300EC0D30740312E2EC0D781F7956AA1DEA87
:10E2F30012F0D412F1DA0AD3EA951E40F2228A1DF3
:10E30300751EB380D7080808087F367E1C90EC2062
:10E31300E571700390EC2A12E9127F3CAE00908FF6
:04E323009602E91263
:10EE4800787512EE987453201702744E207406E5F4
:10EE58002E54074430AF1712EEC27E3BE57DC454F2
:10EE68000F12E8D32074077E07742012E8E678783A
:10EE780012EE98E5172409FF7457201702744520ED
:10EE88007402742012EEC27E3BE57D540F02E8D373
:10EE9800E6FD3392171886041886033017031260AC
:10EEA8003779177870125F418B13AF06AED27C00AA
:10EEB8007D64125EAF8F148D15227E0012E8E67E07
:10EEC80007E51312E7997E19748112E8E67E20E5BA
:10EED8001412E77C7E2B742E2073030E742C12E818
:08EEE800E67E2FE51502E77C30
:10F06400E54A602E7A2420E00E7A26141460087A89
:10F0740028141460027A297F667E01EA12E8E620E9
:10F084005505205406800B745B8002745C7E00126C
:10F09400E8E620110778A9B60007802130261EC2B1
:10F0A4002690B80F7F661281377F64A85AE54AB468
:10F0B400060108E875F06484E5F012E1F420080F15
:10F0C400E537640260097F367E2E744112E8B4226B
:10ECEA0020144F740512F2E8EF33EE33F9EF030301
:10ECFA00541FF5F090ED3DE993A4C5F013C5F01348
:10ED0A00C5F013C5F013C5F0135403FCE5F013FB6B
:10ED1A00E9242093C9244093C39BC4540FFBE99C64
:10ED2A00C4FC540FF9EC54F02B2446F57BE934F675
:10ED3A00F55F22FFFFFFFFFFE6C5AD9C8F857D775C
:10ED4A00726E6C6A696A6A6C6F747A828D9DB4D9C4
:10ED5A00FFFFFFFAE9DCD3CEC9C6C3C0BEBBB9B751
:10ED6A00B5B4B2B0AFADABAAA8A6A4A2A09E9C9916
:10ED7A0096918C00381CE735D137246F00C5B3C192
:10ED8A00E61F66B60E68C21867AADBF4EDB94675C7
:03ED9A0010A200C4
:10F2C800D2A27408D2A1D2A300C2A3C2A1D2A30021
:10F2D800C2A3D5E0EF7405D2A300C2A3D5E0F822FB
:10F2A100C2A3D2A2D2A1D2A300C2A375F008339205
:10F2B100A1D2A300C2A3D5F0F5C2A175F003D2A3D8
:07F2C10000C2A3D5F0F82202
:10D7DA0012F2A1D2A300C2A3C2A175F008E4D2A397
:10D7EA0000C2A3A2A233D5F0F5FE75F008E4D2A3D5
:10D7FA0000C2A3A2A233D5F0F5FFD2A300C2A3228E
:10D80A00E478806608B88BFB70012274D512D7DAE7
:10D81A007881C3EE13FEEF13F692D118EE2460F668
:10D82A0074D612D7DA7888EF33CE33CE33CE33CEEE
:10D83A0033A2D192E25407FCEEFB7A08125D96EC11
:10D84A00244FF608EBF674D912D7DAEF543F7882F0
:10D85A00F67886EF33CE33CE33CE33CE335403F657
:10D86A0008EEF618161608E6C4FF54F0F618E6C4D1
:10D87A00CF540F2FF674DA12D7DAEF232354FC7839
:10D88A0083F67884EEF608EF54C0F67880E46608EA
:10D89A00B88AFBF62212D7E27889C3EF96FF18EE10
:08D8AA0096FEA2E79216501051
:10D8B20012601F740FF8F9125DE3EF2CFFEE3DFECC
:10D8C200788BEEF608EFF622E6182016072CF7E61C
:10D8D2003D19F722C39CF7E69D80F66A405E8056AA
:10D8E200E050F04B0044803DC0384031D02BA025A1
:10D8F200601F2018D014000F000AA0014401580133
:10D90200680178018801A001B401D001EC02100283
:10D9120038026802A002DA030C034D78BE8020852B
:10D922008E8A9D8F4D95BA9A97A0BEA631AC53B2FE
:10D932002AB801BD6AC1EDC4D1C78812D7E2788D79
:10D94200EEF608EFF67887798C125DE378837990AA
:10D9520012D8CA7885798C125DE37881799212D8CF
:10D96200CA788DE624E4FE08E63392D13392D55488
:10D97200FCFFEEA2D133A2D533FE780F7992125D6D
:10D98200E378947990C3EC97F61819ED97F67994A9
:10D9920090D8DD7F1F7D11EF93C3971F19EF9397E7
:10D9A2001F091DED600240EF0F90D8FD798DEF93B6
:10D9B200F7090FEF93F7788E7994125DE390D91DF2
:10D9C200EF93C39BFB1FEF939C2420FC7897E62BDD
:10D9D200F618E63CF618E436F6740612F2E8EEFCA7
:07D9E200EFFD740712F2E8EB
:10D9E900C3ED9FFFEC9EFE78B7E6FD337C00500146
:10D9F9001CEF2DFFEE3CFE789CEF26F618EE36F66E
:10DA09002220140F789DE6B4050912DAAA12DADF8A
:10DA190012DB23222014577897799A12DB54125F6C
:10DA2900A7C3EE9420FE9245500312601F7C007D2F
:10DA390005125EAF30450312601F8E618F60E531BC
:10DA4900B40C2B12EE2EE56120E71124F8500DFAE3
:10DA5900C3E5609AF560E5619400F561121884E503
:10DA6900BC2560F57AE5BD3561F55E12EE3B789728
:10DA7900799AC3E697FB1819E697FC7A02125D9624
:10DA890012DAAA12DADF20140312DB2378957998C7
:10DA9900E6F776000809E6F776000809E6F7760062
:10DAA90022799CE77700FB19E77700FC789DE6B4BB
:10DAB9000506EB33FBEC33FCECA2E792D5500312DD
:10DAC900602F7A32125DA4ECFBEDFC30D5031260B5
:0ADAD9002FECFEEBFF22EE2408FE06
:10DAE3007406307511789DE6B40504740C8007F450
:10DAF3002406C323540FFD7C00125D82789FE6FC4D
:10DB030008E6FBC374109DFA125DA4EFF8EEF91258
:10DB13005FA7E878A02FF6FF18EE39F62480FE22DF
:10DB23009275400312601F78BBE6F5F0243840037A
:10DB330075F0E1EF33EE3378A8F6A485F07930E79A
:10DB4300020579C276307508E57924F15002D27660
:10DB530022E627FB1819E637FC1819E637FD22756C
:10DB63006A0079C6876C09876B22756A2080F31275
:10DB7300DB621298AB7F087871793A12DB90029CD2
:10DB83008A855E63857A62787379647F06E6F7082F
:10DB930009DFFA227864797380F1787379AF80EBC7
:0DDBA30078AF797380E5E6F008A3DFFA2281
:105D1C00E4FEFFFC7D0A791DE7540F2FFFE43EFEE5
:105D2C00B91902800619125D8280ED3017031260DA
:105D3C001F22305C2BEC339217500312602FEC2493
:105D4C00D950047C277B007AD2125DA4EB33CC3380
:105D5C00CD33CC33ED33FBEC33FC30170312602F17
:105D6C00EC339217500312602F7919125FBEF709AA
:105D7C00B91DF8A70322EFF88DF0A4FFEDC5F0CE06
:105D8C00A42EFEEC88F0A42EFE22EB8AF0A4FBE5F8
:105D9C00F0CC8AF0A42CFC22EB8AF0A4FBE5F0CC2E
:105DAC008AF0A42CFCE435F0FD22EB8AF0A4FBE590
:105DBC00F0CC8AF0A42CFCE435F0CD8AF0A42DFDB7
:105DCC0022EB8AF0A430E70205F0E5F0CC8AF0A4CF
:105DDC002CFBE435F0FC2286F0E7FDA4FAABF019BD
:065DEC00E786F0A42BFB8A
:105DF200E435F0FC18E68DF0A42BFBEC35F0FCE466
:105E020033FDE687F0A42CFCED35F0FD22EB89F0A2
:105E1200A4CBAEF08AF0A42EFEE5F03400FDEC89AE
:105E2200F0A42EFEE5F03DFDE433CC8AF0A42DFD76
:105E3200E5F03CCEFC22EB89F0A4CBAFF08AF0A4D3
:105E42002FFFE5F03400FEEC89F0A42FFFE5F03ED1
:105E5200FEE433CC8AF0A42EFEE5F03CFCED89F0A2
:105E6200A42EFEE5F03CFCE433CD8AF0A42CFCE544
:105E7200F03D8E058C068F04FF22C2D5EC30E7057B
:105E8200B2D5126027EE30E70DB2D512601F125E56
:105E9200AF1260278003125EAF30D50312601F225B
:105EA200C3EC13C0E0ED132FFFD0E03EFEBC000BAD
:105EB200BE0029EF8DF084FFADF022E4CCF975F03D
:045EC20008EF2FFFB7
:105EC600EE33FEEC33FCEE9DEC994005FCEE9DFEB8
:105ED6000FD5F0E9E4CEFD22EDF9F5F0EE8420D2FF
:105EE6001CFEADF075F008EF2FFFED33FD4007996E
:105EF6005006D5F0F222C399FD0FD5F0EA22EC3315
:105F0600EE3400FEEF3400FF7D007A007900780958
:105F1600C3ED9AFDEE9BFEEF9CFFB392D54009EDD3
:105F26002AFDEE3BFEEF3CFFA2D5E933F9ED33FD4A
:105F3600EE33FEEF33FFD8D92279007A00C38015FD
:105F460079007A00C3EA13FFE913FEE8132BFBEE90
:105F56003CFCEF3DFDE4F5D2F5D333FE7F19C3EEED
:105F660098FEE5D299F5D2E5D39AF5D3B392D5400A
:105F76000DEE28FEE5D239F5D2E5D33AF5D3A2D512
:025F8600EB33FB
:105F8800FBEC33FCED33FDDF0122EE33FEE5D233CB
:105F9800F5D2E5D333F5D380C3AD6FAC6EAB6DED01
:105FA800C454F0FEECC4FF540F2EFEEF54F0FFEB88
:105FB800C4540F2FFF22EC75F00A84FCEB54F02533
:105FC800F0C475F00A84C4CBC454F025F0C475F04D
:105FD8000A842BFBE5F022AC10AB11125FBEA904BA
:105FE800AD03FA7C197B99125D96AE04AF03EA758E
:105FF800F006A4F8AC12AB13125FBE2875F00A8441
:1060080085F014F8EF2BFFEE3CFEEF28FFE43EFE90
:10601800E43DFDE439FC22C3E49FFFE49EFE22E454
:10602800C39DFDE49CFC22C3E49BFBE49CFC22C3CF
:10603800E49BFBE49CFCE49DFD2275D4107B807AF4
:0C6048000079807800EAF5F0A4FCADF0CF
:10605400EBF5F0A4FEAFF0EB8AF0A4C333C5F03344
:10606400C5F092D52DFDC5F03EFEE430D501043FC8
:10607400FFB5150DEEB51409EDB51305ECB5120118
:10608400224006EA98FAEB99FBD5D40ABB00012218
:106094000ABA00010B22C3E913F9E813F8EA28FA53
:1060A400EB39FB80A478087B807D807C00EDF5F0E3
:1060B400A4FAE5F08EF0B5F007EA8FF0B5F001220E
:1060C4004003ED9BFDD827BDFF0122EDF5F0A4F9B7
:1060D400A8F0ED04F5F0A4C399FAE5F09813CA13F7
:1060E40029F9E83AF8C3E99FE89E50010D22C3EB71
:1060F40013FBED2BFD80B6C374689511FB740195F9
:1061040010FC8004AC10AB117A0B79B8125E0F80CE
:10611400177473F8F9E627FB0809E637FC0809E663
:0261240037FD45
:1061260030E703126037EB33FBEC33FCED3323FD32
:10613600242083F8ED241C83FFED241883FAED2434
:106146001483F9EF99F9E89AFA125E0FEF9DFFE8CA
:106156009EFE22FFFFFFB6FED7FD63FB5DF8C4F58A
:106166009BF1E3ED9EE8CFE379DD9ED743D06BC983
:1061760019C153B91CB079A7709E06943F8A237F34
:10618600B674FF6A045ECB535B47BB3BF130042316
:10619600FB17DE0BB2FF80C21DC232532CF8C3E5DB
:1061A600679576FBE5689577FCE5699578FD30E7B8
:1061B60005D26112603724F05003126271AA06A953
:1061C60007125E38EC2480E43DFBF9F51AE43EFC48
:1061D600FAF519E43F6002D232125E0F8B128C136D
:1061E6008D148E15C3E5649573FBE5659574FCE522
:1061F600669575FD30E705D262126037EBF9F51F3B
:10620600ECFAF51DED6002D23230320122125E0F39
:10621600EB2512F512EC3513F513ED3514F514EEE6
:106226003515F51540E102604212619D20323BEBC7
:10623600242E40D3EA2401CB3400FC7A07793D12A0
:106246005E0FC010C0118E108D118C128B13E4FCE2
:0E625600FD7E077FD012D36E851203851302E2
:10626400D011D010BB0005BA0002D21D22B261C306
:1062740074809BFB74F59CFC74209DFD22204D6969
:10628400204866303F637F697E0112DD817E1F12E4
:10629400DDFC75A7009004EDE0A2E792171392E7E6
:1062A400FC1582E013FB30170312602FBC003AEB9D
:1062B400603720E73420E63110E513201707C37454
:1062C4001F9BFE80027E1F12DDF10EDBFA22FB20F3
:1062D40017097E00C374209BFB8008EB241FFE7407
:1062E400209BFB12DDEB0EDBFA2275A700758307FA
:1062F400E559C4440FF582E0A2E792522212DB9DD5
:106304001262EEC2E775F00A84FEAFF075A704537B
:1063140082F17864126377AE07786712637775A7A2
:1063240000E57DC4540FFEE57D540FFF78731263BE
:106334006BAE07787612636B74AF12611712622F1B
:106344008B148A131207D2ACCCAB017A0A125D9675
:10635400E5139B9004ECF0FBA3E5149CF0FCA2E78E
:10636400923DD23F02DBA386030886040886051803
:09637400188006E0FBE0FCE0FDEE
:10637D007A0A125DB620E70CEB2EF608E43CF6081F
:10638D00E43DF622C3EB9EF608EC9400F608ED947E
:10639D0000F622204D09204806C23F302A0522C2B0
:1063AD003380F6E54824F640F5E5580460F075A70E
:1063BD0000758307E559C42408F582E0FEA3E0FFCC
:1063CD001207D27437126463500B30381BC2387801
:1063DD00C5864680137432126463400C203809D28E
:1063ED003878C5A646754600740D126463404A128E
:1063FD006301303D38201122204D1F20481C2040C4
:10640D0019BCFF16EB24325011D24012185CE5BFB7
:10641D0075F019A4F536D22ED22F205238E55965D4
:10642D00586032204D2F20482CD23380282011095E
:10643D00204D06204803753600303319204D1220AB
:10644D00480F12AA000559C3E558955950038558B0
:10645D0059C233C2402229FBE435CCFCC3EB9FEC7F
:10646D009E22E558B4FF012285581175A704758346
:10647D0007E54824F65002805C201259202905209A
:10648D002A02805112DB9DE4F516F51775100012E6
:0C649D0064FBE510700312DB971265141D
:1064A900302910E51B2517F517F51BE51C3516F5E1
:1064B90016F51C12652112DB970510C3E51195101D
:1064C90050D175A70002DBA3E55AF51124F6500354
:1064D90075110A75A7047583067510001264FB12FD
:1064E90065141265210510C3E511951050EE75A7C5
:1064F9000022E510C4F582E0E0F564E0F565E0F519
:1065090066E0F567E0F568E0F5692275A7011269AB
:106519000D124AE775A70422E9F0E51CF0E51BF026
:1065290022E510C454F0F582E0F512E5822406F55F
:1065390082E0F511E0F51CE0F51B22E512B4261501
:106549007F757E34740D12E90120442575110012FE
:10655900E29A0266727F6D7E3BE012E8E6E5137E01
:106569003512E8E6E5127E2F12E8E620440312E22E
:106579009A12E206026672202852E558B4FF0122F7
:1065890075A704758307E559F51030330965586017
:1065990005204802051012652AE0F513305E072030
:1065A9004304E5376095E07F797E3D12E8B4E51351
:1065B9007E3912E8B4E5127E3512E8B430480B7F13
:1065C9007F7E3512F2170EBE40F980392012012262
:1065D90075A704758306855B1012652A305E0A204B
:0265E900430766
:1065EB00E5377003026794E512700B7E3A7F79747E
:1065FB005D12E8E6800D75F06484E5F07E397F7AF4
:10660B0012E834E537B4020512A8988045B40302AA
:10661B008040E51C7006E51B24FB5036E511F96440
:10662B00B4602F20062CE537600D200C0AC3E995CA
:10663B0070F9500324B4F9E912F0D4781D79547D24
:10664B001D90EC12E53F20E00390EC1912F1DA12E9
:10665B00E91275177975161930280375161DE51291
:10666B00642660031266B575A7009006E3E511F08A
:10667B00A3121875E5BC75F01970040475F014A419
:10668B00951BFBE5F0951CFC9224500312602FEC3C
:10669B00F0A3EBF0C24FC263EC700EEB24E64002AA
:1066AB00D24FEB24C84002D26322E51C24ED402BD1
:1066BB00AE1CAF1B1268D77C007D32125EAFC005DB
:1066CB00EFAF17AE1612E7EDCE2405CE742C12E801
:1066DB00E60E0ED0E02312E7E7801B1268CE12679E
:1066EB000FCE2405CE742C12E8E6CE2402CEE8752C
:1066FB00F0058412E8CCCE2404CE7422305D0274F3
:0D670B008302E8E2EE243D50047EC37F4B84
:106718007C017DF4125EAFC004C005EF6007AF17BF
:10672800AE1612E7EDD007D0067C007D32125EAFC0
:10673800A805EFAF17AE16CE240ACE02E8CC126831
:10674800CEEE2450305D03EE24A150047EC37F4B6F
:106758007C017DF4125EAFC004C005EF6007AF177F
:106768007E2F12E83AD007D0067C007D32125EAF49
:10677800C005EFAF177E3712E8A17E3B742C12E8F4
:10678800B47E3DD0E075F0058402E8A17F6D7E2FD0
:10679800746312E8E6E51275F06484E5F07E35125C
:1067A800E77C12E29A02E20630480320740122E4F0
:1067B800FCF5A79006E3E0F9A3E0FE24FE40EFA372
:1067C800E0FF7D78E5376008304FE3200C2A800B26
:1067D800121861E5BD20E010304F0DD206E5712496
:1067E800FE50151268C480107D3CE546600A7D1491
:1067F8001460057D0A1470B68911125D827D6F12CE
:106808005EA2BE00A9EF24E240A4AD07E51112F094
:10681800D4202404B2D5B2D1781F795612F1DAA85F
:1068280006A907E511242D75F0B484E5F012F0D41B
:106838007407304F02740EFDFA12F1DAB2D5B2D1F4
:0768480012F1DAB2D5B2D162
:10684F00DDF0AD0212F1DA850616850717B2D5B263
:10685F00D112F1DA85061E85071F7A03304F027AAF
:10686F0006E511241675F0B484E5F012F0D4A816DD
:10687F00A917AD0212F1DADDFBE51124EA4002247B
:10688F00B412F0D4A81EA91FAD0212F1DADDFBE598
:10689F00377021304F1E90C170305D0390C16C7FF7
:1068AF003C7E3312817C121861E5BD20E00612DEBA
:1068BF000212EBB122C3E99570500224B4F922E51C
:1068CF001B2402FFE4351CFE305D1ABEC305BF4D0D
:1068DF00028012AC06AB077A1B125DA47832125FEE
:1068EF0046AE04AF03227873796412611912622FD6
:1068FF00751CC3751B4B2032048B1C8A1B2212681C
:10690F00F530320122AC19AE1AA91DAF1FB900051F
:10691F00BC00028010C3E913F9EF13FFC3EC13FCA3
:10692F00EE13FE80E8BF29005006BE290050012259
:10693F00C3EF13FFC3EE13FE80EB3E7FE3E3E3E30E
:10694F00E3E3E3E3E3E37F3E0C1C3C7C7C1C1C1C79
:10695F001C1C1C1C7F7F3E7FE3E3E3070E1C38707B
:10696F00E0E3FFFF3E7FE3E3030F0E0F03E3E3E3F9
:10697F007F3E070F1F3F77E7E7FFFF070707070771
:10698F00FFFFE0E0E0FEFF030303E3E37F3E1E3F74
:10699F0073E0E0E0FEFFE3E3E3E37F3EFFFFE3E3CB
:1069AF000303070E1C38383838383E7FE3E3E37FA4
:1069BF003E7FE3E3E3E37F3E3E7FE3E3E3E37F3FBB
:1069CF00030303E77E3C000000181818FFFF181898
:1069DF0018000000000000000000FFFF0000000092
:1069EF0000003FF00000381C38F00180C1F020F0AB
:1069FF00FC0038F03FE0000000007CC6C6C6C6C6EB
:106A0F00C6C6C67C1838781818181818187E7CC691
:106A1F00C60C183060C0C6FE7CC6C6061C0606C66D
:106A2F00C67C0C1C3C6CCCFE0C0C0C0CFEC0C0C00D
:106A3F00FC0606C6C67C3C66C0C0C0FCC6C6C67C8B
:106A4F00FEC6C6060C18303030307CC6C6C67CC6B3
:106A5F00C6C6C67C7CC6C6C67E060606CC780000B7
:106A6F0018187E7E18180000000000007E7E0000BF
:106A7F00000000000000000000000000C6E2E2D2AB
:106A8F00D2CACAC6C6C20000000000000000000043
:106A9F008080A0C0A000304020C08080C0A0A00097
:106AAF000060A0600000A040A05098D090882050B7
:106ABF00A850888850A8502060806000000040E0F7
:106ACF00400000000000800000E000000000000017
:106ADF0040002040800040A0A0A04040C04040E0C7
:106AEF00C02020C0E0E0204020E02060A0E020E0B7
:106AFF00C02020C06080E0A0E0E020404040E0A047
:106B0F00E0A0E0E0A0E020C00040004000008000D6
:106B1F0080002060E0602000E000E00080C0E0C066
:106B2F0080E0E0E0E0E0000000000040A0E0A0A076
:106B3F00C0A0C0A0C040A080A040C0A0A0A0C0E046
:106B4F0080C080E0E080C080806080A0A060A0A0B6
:106B5F00E0A0A0E0404040E0202020A040A0A0C046
:106B6F00A0A080808080E0A0E0A0A0A0A0E0E0E056
:106B7F00A040A0A0A040C0A0C0808040A0A0C06046
:106B8F00C0A0C0A0A060804020C0E040404040A016
:106B9F00A0A0A060A0A0A0A040A0A0A0E0A0A0A046
:106BAF0040A0A0A0A0404040E0204080E02020A8CE
:0D6BBF0070202070A8202008F030D01000B9
:106BCC0000F0A8A8000000E00000009020487088A9
:106BDC0098984000E0E0E000A0E0E0E04060301079
:106BEC0030604040E0404060909090909060206019
:106BFC002020202070609010204080F060901020A9
:106C0C0010906010305090F01010F080E010109048
:106C1C0060609080E0909060F010202040404060D8
:106C2C0090906090906060909070109060C0E0F0D8
:106C3C00F8F0E0C0000000000000000000000000C0
:106C4C00000050605000707050000078807008F0A8
:106C5C0000F8888888F800C0C8102040981800C038
:106C6C00B098B0C000602040000000000090D8FC3C
:106C7C00D8900000246CFC6C24000020A870A82084
:106C8C0000002020F8202000000000000000800000
:106C9C000000F00000000000000000606000081020
:106CAC002040800070888888888870206020202090
:106CBC002070708808102040F8F810201008887098
:106CCC0010305090F81010F880F0080888703040A0
:106CDC0080F0888870F808102040404070888870D8
:106CEC008888707088887808106000606000606028
:106CFC000000008000008000002040F840200000D0
:106D0C0000F800F80000002010F81020007088082F
:106D1C00102000200000000000000070888888F817
:106D2C008888F08888F08888F070888080808870E7
:106D3C00E09088888890E0F88080F08080F8F88077
:106D4C0080F0808080708880B8888878888888F8FF
:106D5C008888887020202020207038101010109007
:106D6C00608890A0C0A09088808080808080F88807
:106D7C00D8A8A88888888888C8A89888887088889F
:106D8C0088888870F08888F080808070888888A8CF
:106D9C009068F08888F0A09088708880700888705F
:106DAC00F82020202020208888888888887088886F
:106DBC008888885020888888A8A8A850888850205F
:106DCC0050888888888850202020F808102040801F
:106DDC00F800CCAC9CACCC0000CCD4E4D4CC0004FB
:106DEC00781828C800FC40A040182020180000008B
:106DFC00000000F800000000A040A0500078888837
:106E0C009868708840308870200000F0A8A8A8A866
:106E1C007848484848788870888080887020A8888E
:106E2C0098A8C88888805048FC485080304C5C60DA
:106E3C0060603C00E0F0080808F88044485C484476
:106E4C0080F880808080808078484848484888B89E
:106E5C00A8A8E8A8A8B88888888888F8085000707E
:106E6C00888888708080F088888888F888888888E6
:106E7C008888F09090909090F0A8A8A8A8A8A8F85E
:106E8C00888888F808080850008888888878A8A816
:106E9C00A8A8A8F8080000000000000000000000EE
:106EAC0000000088888888E8A8E8A8A8A870A8A886
:106EBC00A80000000000000000000000000000001E
:106ECC0000000000000000000000000000000000B6
:106EDC006000606000600060006060205020000076
:106EEC0000005090B890D090886050500070705056
:106EFC00008820208870000080C0A090F8003048E6
:106F0C00B4B44830003048B4B44830FC0098D020B9
:106F1C0058C800F8E8D880D8E8F8404050F85040FD
:0F6F2C0040A0C0A000203828A0C0A01038101826
:0B00000002005E000000000000000095
:03000B0002AA70D6
:10000E00206E06859950D26E32D26F32854F82E5C0
:05001E00143200000097
:1000230010990DC298206909206DE085994FD26D12
:01003300329A
:1000340085D01285835085824FF51485158275838A
:1000440004E515242140020515E599F0D26D8512C9
:07005400D085508380C0003D
:03005B000237F376
:10AA63008530F0C5F065308530F060F722C0D0C086
:10AA7300E0C0F0C0A775A700C083C08275D0087579
:10AA83008A00300503758A7A758CEA0532E53270DF
:10AA93000215320530E530640A6026201520E531C1
:10AAA300B40C0BE530B4010612AF6912ECEAE531E0
:10AAB300B4180BE530B4060612AF6912ECEA02AC27
:10AAC3008DC2AFD2C075C07AD2AFF5300531E53152
:10AAD30064197043F53120152CC225C22C7D0A74EC
:10AAE3000412F2E8EF33EE339005CCF0EE24F54098
:10AAF300142402400E24014008202005DDE1023722
:10AB0300F3D225D22CE5A6600215A678B5E660013E
:10AB13001678B6E6600116302E0BE5367007C22FA5
:10AB2300C22E12AE4EE5367004C24B800215367843
:10AB3300A9E660011678D8E66001160535E535709B
:10AB4300021535E590307B0B30E008D278C27BC22A
:10AB530000801A307C0B30E108D279C27CC20180BC
:10AB63000C307D0930E206D27AC27DC202E5904400
:10AB7300F8F47003753500304A09E53324FA5003BD
:10AB8300753305E5336005153302AC32E590F454B3
:0EAB930007700302AC32A2E09200A2E1920130
:10ABA100A2E2920230100320143D75330820001BED
:10ABB10020100C2011098013E59030E10E8006E58C
:10ABC1003724FC40F3E543541FF53320100375A6E9
:10ABD100FF202E5D301004E536705620100C201138
:10ABE10009E53524F55003753304D21BD2A5D2A64D
:10ABF10012AE4E75B44075B24078D8E67002053495
:10AC010020272E20682B202928202A25A210721106
:10AC1100501FE52054076019E53424375004C24A17
:10AC2100800F2401400B200026200119D27D7534AC
:10AC3100C8201558E531702412F2C874E812F2A147
:10AC4100802A02AD91E53724FC40E6D27C80DF30DA
:10AC510011DFE53724FC40D9D27B80D275F0038423
:10AC6100E5F070DE12D89F74E812F2A1E531B40666
:10AC71000512DA0A8016B40C0512DA1D800EB41220
:10AC81000512DA0A8006B4180312DA1D20141B809B
:10AC91001990ACB5E532C4540F93FAE532540F6004
:10ACA100096A70061216ED12171CE59030E1153095
:10ACB100E2128016010204040404050506070708D0
:10ACC10009090A0020100820110520103C807D2070
:10ACD10027F82068F52029F2202AEFE534243040B6
:10ACE100E9240750E5600B205E088590F020F20210
:10ACF100740190AD0393D2A5201002C2A512AE3902
:10AD0100806FC8A08269554646202F12E536603C07
:09AD110024AA500AE53675F01978
:10AD1A0084E5F06040D2A6201002C2A6D2A5202F58
:10AD2A000C7418304B02746412AE39803BE53675E8
:10AD3A00F00C30480375F00684A2E0744640E974CA
:10AD4A003780E5E52B5403600C20100E301106E520
:10AD5A004A6402600512AE54800312ADA9101B08A2
:10AD6A00A25892A5A25992A675A700D082D083D0E4
:10AD7A00A7D0F0D0E0D0D020200C201009C5A670B2
:10AD8A00030237F3C5A632C218B40202D21812D986
:10AD9A003D30180874E412F2A102AC6D02AC687876
:10ADAA00A7E5B4600924E04005760002AE54E53414
:10ADBA00702920412220751F300D1CE57924CE40D0
:10ADCA00167AFFE5B110E7010A2325B3F5B3EA3590
:10ADDA00B4F5B4C313F5B2E660021622C241207577
:10ADEA00028077C246E579FF605820120424FD509C
:10ADFA0051206502C21CD265EF24B050027F4FEF8A
:10AE0A0090AF199375C70375C6FC75B90185BFF074
:10AE1A00A4E5F0F624F44002760C301C2DE5BEC3FE
:10AE2A009FF5F0A4E5F024E0400375F020E5F0C2B8
:10AE3A001C79AA770375B300F5B4C31375B100F58D
:0CAE4A00B222C26578A77680D24179AAB6
:10AE56007703D21CE4F5B3F5B4F5B1F5B222C265B9
:10AE660079A1E57924CE500DE720E7E27628301C5B
:10AE7600DD743C80BE7680E720E7D3E57997404DC8
:10AE8600C24679AAE7FAE5792323B4C500400274DD
:10AE9600C42437300E31F42437300D15F7BA0302C7
:10AEA600FA0AC39AF5B175B300EAF5B4C313F5B25D
:10AEB60022101C07D21C76C802AE3B763274FF20E5
:10AEC6000E02749B02AE3BC313247E80CC75C7036F
:10AED60075C6FB75B901E5BD6026C395795004C2F8
:10AEE60046801D78A720461B301C11E57975F008B1
:10AEF600A42432F6E5792324AA02AE397605D24691
:10AF060002AE54301C077614747802AE397696C2B7
:10AF16004680EDFFF3E8DDD3C9C0B8B0A9A29A9484
:10AF26008F8A85817D7975716E6B6865625F5C5904
:10AF36005653504E4C4A48464442403E3C3A3836B8
:10AF460034333231302F2E2D2C2B2A292827262533
:10AF560025242423232222212120201F1F1E1E1DDB
:10AF66001D1C1CD2B5C28EAE8DAA8DAF8BAB8BE4E9
:10AF7600F58DF58BD28E3014012278B6BE0007EF20
:10AF860024E24002800806E624EC5002761420678C
:10AF960005E624F64005E4FEFAFFFB7C007D0A1276
:10AFA6005D827C007D5E125EA28F51EE600375515C
:0FAFB600FFEAFC7A33125D96EBF5F0A4E5F0CBE1
:10AFC5008CF0A425E0C5F035E0CB92D525F05006F0
:10AFD5000BBB0002D2D530E7060BBB0002D2D5EC85
:10AFE500F5F0A42BFBE5F03400FC30D5010C78A678
:10AFF500E6C39BFF18E608F6EB18F618E69CFE1864
:10B00500E608F6EC18F6301401227A0050040A120C
:10B01500601F7C007D6E125EA28FF078A2E6A4FB15
:10B02500ACF0125FBEEBBA0002F404FAE4F8FFEAF2
:10B0350030E70118E57960062075031FF4042AF549
:10B0450079EF38D27520E70860037579FF02DB4692
:10B05500C2750470F5E579F40460EFF57980EE12B8
:10B06500185778BBA6BC121875E5BE78A2F624F66B
:10B075005007E4F5BEF61255F7120BF6E5BEF54896
:10B0850024F65008E4F5BEF5481255F7E5BFF5433B
:10B0950024F3503924F3403512186B78A1A6BCE58A
:10B0A500BF789DF61424FB50087403F6F5BF1255BE
:10B0B500F778B7A6BE121861E5BDA2E39266A2E4D1
:03B0C5009267038C
:10B0C8005403C253B40102D25322740DF5BFF543A1
:10B0D8001255F780C0E56A700CE56B5403700612D0
:10B0E80098BD12B14775F08412B17F787086F70861
:10B0F800B880FAD2B275F08812B16D782575F00073
:10B10800758002C2B275F7D7E4F5F70000E5F7D20B
:10B11800B220E705D5F0E9D8E72275F08412B17FAF
:10B128008DF7A4D2B280CE75F08412B17F75F0008D
:10B1380075F7FFD5F0FAD2B222756BEC756A007517
:10B148008002C2B275F78475F70075F70075F700CD
:10B15800780075F7FF75F7FF75F7FF75F7FFD8F2F9
:10B16800D2B275F08112B17FD2B2808F75F05312CE
:10B17800B16D808775F003758002C2B285F0F785DE
:10B188006CF7856BF7856AF72275F003758002C244
:10B19800B285F0F7856FF7856EF7856DF722125443
:10B1A8004775382490B1FE12320B12EFBF02F145F9
:10B1B8001254477D0E90B21512B1C87D1890B22373
:10B1C80074A012EFAB74A212EFABE4FEFF12EFAB68
:10B1D800ED12EFABE493A312EFAB2FFFE43EFEDDDD
:10B1E800F3EE12EFABEF12EFAB74B012EFAB74B338
:10B1F80012EFAB02F14B24505352463130302C3011
:10B208002C35373630302C382C312C300088000063
:10B21800040000000000000000000081020101009D
:10B22800010101000101010001000100000001000D
:10B2380000E10075160375170312B27B204C01223A
:10B24800D517F6D2A47F8CDFFEC2A412F13D12B14D
:0FB25800A612B1B812F13DD516DC12F2FC7F320E
:10B267007E0690BF5412814912283F12F1853000A3
:10B27700FD0237F3E4F5A79004DFF0D582FCF01266
:10B287005447D269D2ACE4F515F87903106DF7D8B5
:10B29700FBD9F9E4F515F8F97A05E515700FD8FA31
:10B2A700D9F8DAF6C2ACC269D24CD23D227800791D
:10B2B70007106DF9D8FBD9F99005FF7453F0753273
:10B2C70010C2ACC269C24CC23D7A0312B613103B1E
:10B2D700D388017A0312B629103BC9E89940C57A89
:10B2E7000112B6AE70BE7A0212B6AE70B77A03120A
:10B2F700B6AE70B07A0112B6137A4712B601303B78
:10B3070004D23D800B7A0512B63C12B68AB43024BB
:10B31700E49005DDF09005E5F09005D779BCF0F5F0
:10B327005DF7A309F0F55CF79005F27427F0A374B5
:10B337000FF08059D25712B64E9005DDF09005E513
:10B34700F012B64E75F00AA4FA20D1010812B67AA7
:10B357002A75F00AA4C5F09005F2F0A3E5F0F0E431
:10B36700FCFBFEC21712B68AB42D05D21712B68D92
:10B37700B42E02800512B5F2DEF330170312602FE8
:10B387009005D8EBF0F55C1582ECF0F55D7A0212CA
:02B39700B613EB
:10B399007A5312B601303B04D23D80647A0212B668
:10B3A9003C12B67A147006FA532EE080139005DE2B
:10B3B9007402F0D274C2737A05146004D2737A07E6
:10B3C9009005CEEAF09005DDE05407C52E54F82526
:10B3D9002EF52E7E0C7DE612B63AC2D512B65175FF
:10B3E90083058D82F00D30D504DEEF8002DEE8AEF4
:10B3F9005DAF5C207303E4FEFF79BCA70609A707CC
:10B409007A0312B6137A4D12B601303B05D23D02CA
:10B41900B52B12B64EF53D12B651F53E12B651C5D1
:10B429003F0475F03C84E5F0653F60069005FF74C4
:10B4390044F012B68AB4562D7A0612B63CC22DE4EF
:10B44900F571F5707E049005D9F0A3DEFC20571341
:10B45900F57D7E067973F709DEFC7E089005CFF04D
:10B46900A3DEFC8074B441A512B63AC23C7FCF1268
:10B47900B564C4F57D12B68AB43102D23C7FD312C9
:10B48900B564257DF57D12B63A12B5DE7AB9125D3D
:10B49900A4C0007864125F46D0009005D9ECF0A3EF
:10B4A900EBF0125FBE8B71EC60037571FF12B63A57
:10B4B90012B5DE9005DBECFEF0A3EBFFF07C007D1E
:04B4C90014125EAF4C
:10B4CD00C22DED24F150010F240A5002D22DBFB42C
:10B4DD00027F008F70C23C12B64EF53C24E0500244
:10B4ED00D23C12B651F53B24F35002D23C12B65168
:10B4FD00F53AE53D24E85002D23CE53E24C4500225
:10B50D00D23CE53F24C45002D23C303C02800F7542
:10B51D00A7049005DF793A7E06E7F009DEFB203DB2
:10B52D000320740C532EE0E49005CEF09005DEF070
:10B53D0075A7049005F4E561F0E560F0E55EF0E5D2
:10B54D007AF0E579F0E52EF0E55FF0E57BF0E55179
:10B55D00F075A700029C8A12B651303C0224647526
:10B56D00F03CA4ACF0FB12B6512BFBE43CFC7A642E
:10B57D00125DA40812B6512BFBE43CFCE43DFD1218
:10B58D00B67AF912B68AC21724AF5005D2171260D7
:10B59D0037BFCF358D758C748B73301703126037B1
:10B5AD007A0A125DB6EB29FBE43CFCE43DFD7E001E
:10B5BD003017041260371E7583058F82EEF0A3EDF0
:10B5CD00F0A3ECF0A3EBF0E9228D788C778B7680ED
:02B5DD00C9E4BF
:10B5DF00FCFBFE12B68DB42E02800512B5F2DEF31F
:10B5EF0012B68DCD7A0A125D96CD540F2BFBE43C2B
:10B5FF00FC22C23B080808758304888208E06A6051
:10B60F0002D23B22C23B7583047800888208B8E0DF
:10B61F000280EEE0B424F4DAF2227800888208B8CF
:10B62F00E00280DDE0B42AF4DAF2227A01758304B5
:10B63F00888208B8E60280C9E0B42CF1DAEF221252
:10B64F00B63A758304888208E0B42C04D2D5E4227C
:10B65F00540FFA08A3E0B42E04EAD2D122540FCA31
:10B66F0075F00AA42AC2D12212B63A7583048882D1
:10B67F0008E0B42E0308A3E0540F2212B63A7583E4
:10B68F0004888208E02212B69FC4FA12B69F2A22BB
:10B69F00888208E020E603540F225407240922125F
:10B6AF00B6137AE6753800888208E0B42A0612B617
:10B6BF00956538226238DAEF74462212547375A7F3
:10B6CF00009004007EE07D03E0A312EFABB40A0408
:09B6DF00DD028002DEF202F14FEF
:10005E00D2B47581C075AF017590F878FFE4F6D80B
:10006E00FDF4F5A6D220D2C075C07A75F83075D7DA
:10007E005075AE1375AF017581D87590F875EFBCDC
:10008E0075FDFFC2B7D2A412F141C2A4745012384A
:10009E0016758951D28C75A882D2BC12997B12F238
:1000AE00C812D81512B064C22012ED9D1236C57F4B
:1000BE00407E0190B6F112814912549112F1411213
:1000CE00EEF012F18512F17B7C1412F14B3000032D
:1000DE000237E3DCF512B1A612B1B812F14175A6E2
:1000EE00FF12B23B12B0641236C512F18512F13D09
:1000FE0012F17B78B5761E12ED9D12D80AC215C28A
:10010E00141236C590B7397F78128137205E0A7F78
:10011E00767E1290B74612E9127F4012F2777F492F
:10012E007E0912E14FE53F20E00805A6E5A6700224
:10013E0015A67F5312DD757F577E0B12E6A912E7C7
:10014E00317F602073102074097E2BE52E54071228
:10015E00E8D37E17800E7E0BAC5DAB5C12E6AD1263
:10016E00E7317E311281D37F697E1212EC38302551
:10017E00087E1290EF5912E912E5A60303543FFDD3
:10018E00FE0D7F7312F2170F12F2171EDDF478B503
:10019E00E57124F64002761E307419E6602B7F72EC
:1001AE007E16744012E8B47E17E612E83A7E1F748B
:0701BE005312E8B412F185B1
:1001C50010000C10010C10020C12B23B02010502CA
:1001D50037E3023A3E8061E53524C85046E5902074
:1001E500E241D0E0D0E0120229027D9DE53524D21E
:1001F5005031E59020E22CD0E0D0E08038E5352480
:10020500D25020E59020E21BD0E0D0E012F2FC3085
:100215006B0B7F0912812E12562F128606120229A8
:100225000205702212F2FC90C0097F00128137127C
:10023500F18502F13A12F16AC215C214C227C268E9
:1002450012F17B75370190B82C1227259002557352
:100255000200EF0221F0020A08022AD2020570020A
:1002650005AD027D9D02027002052212F17B7537F4
:100275000790BBC41227259002807302023D020835
:100285001D02085702088B0202A102041102027026
:100295000202700202BF0202A60256FF12B23B80A2
:1002A5002A7F517E00747212E8E212289C40BC122B
:1002B500554312ED9D12B06480B17F49A25E120BC9
:1002C500E1925E120C0080A31255F712F17B75378F
:1002D5000290BD8B1227259002E07302027002186E
:1002E500A202190702195B0219B00219F4021A03D6
:1002F500020341020377021DC70203017F5B121847
:100305009812187AA8BE12032512F185100008105C
:10031500010710020780EF18180880EA88BE80A838
:100325005300037F5A7E0590BDDEE875F00BA425CA
:0E03350082F582E5F03583F5830281497F4031
:1003430012189812187AE5BCF8E87F3F7E3212E75C
:10035300F312F18510000810010D10021280EA1843
:10036300B84AE6787D80E208B87EDE784B80DA888A
:10037300BC0202CD12F2FC7F0F90C1FF1281371233
:10038300283F12F185C214C21512F13A7510651097
:1003930000DFE53170F9E5106465700D855E148545
:1003A3007A15E4F512F513800C78A8E51326F513F6
:1003B300E43512F5127F1E7E19E51012E799C3E5A5
:1003C3007A9515F517E55E9514F5167F287E0BAC27
:1003D30016AB1712E6AD12E73112F18512F14BD5C8
:1003E30010ADAB17E516FC30E70312602F7A0A79DC
:1003F30000125E0FA912A813125F48EBF510243800
:1004030040037510C81218578510BC0202CD12F2B2
:10041300FC90B7847F017E0912814990B78D7F0AD2
:100423007E091281497F1312DD6D7517001218665C
:10043300E5BC1204F1E5BD1204F1E5BE1204F1E5D9
:10044300BF1204F190B7DE7F5F7E06128149122846
:10045300DE12F1857517001204D110000810011582
:1004630010024880F20517E51724F75003751700AB
:1004730075100080E2E5176408701512186675BCE4
:100483000175BD2375BE4575BF671255F70204118B
:10049300E51012050312F1851204B105105310077C
:0604A300E51724FE4003F2
:1004A90053100380AC020270A9BCAABDABBEACBF9D
:1004B900E5171304F8E640085407C42510C480045E
:1004C90054702510F60287EE7800E875F009A42427
:1004D90017FF7E3B7D20E8651770027D89ED12E8E4
:1004E900E608B809E502F185F8C41204F7E812052F
:1004F900037E030517E51702E8D3540775F009A42D
:1005090090B7962582F58250020583E51775F009A3
:10051900A42417FF7E0C02814912F17B75370890DC
:10052900BE84122725900532730200EC02054E02A3
:10053900142F0212E2020D0F02568D0205477F3772
:100549001220CD80D47F0A121898120BF61220724D
:1005590012F18510000810010510020680EFB25A49
:1005690080EB120C0080B2C26812F17B75370590DE
:10057900B96C1227259005827302023D0283870216
:1005890083CC0285650205700205A60284A702854F
:100599000D0221B902057002219F020B127F2E1252
:1005A90020CD80C312F17B75370690BA4A122725F0
:1005B9009005BD7302023D0221F60222580222D1A2
:1005C90002239E0223D00224470206020205FB02EF
:1005D90024900225350205E17F64121861E5BDA268
:1005E900E7120BE1121861E5BD92E7F5BD1255F767
:1005F90080B27F491220CD80AB1207BE12383D125E
:05060900F2FC122819AB
:10060E00E55804607790BB181206AB129FD512F115
:10061E008510000810011310021C80F50559C3E562
:10062E0058955950D575590080D01559E55930E770
:10063E00C985585980C4E559B40F02802FB51F02E1
:10064E00802A75F007A42408F51775162774B825A7
:10065E0059F9870012069912F18510002810012809
:10066E0010020280F574B82559F9A700E53524FA71
:10067E00508878C7A6481207B512F2FC12F18512FF
:10068E00F13D0205AD1880CC0880C9E875F005A4CF
:10069E0085F01CF51BC0001266B5D0002212A066B4
:1006AE00B4FF0122751000751FFF12A07DE51064C6
:1006BE000F60171206E2401274B82510F8E675F0B6
:1006CE0005A485F01CF51B1267460510C3E5589569
:1006DE001050D722121BABF8602E6404602AE81467
:1006EE00B51025F51F121875E5BC70060475F014CB
:1006FE00800375F019A485F01CF51B1267467E2247
:10070E0090C1A012817CD322C322E558B4FF0122EE
:10071E00751000E510640F602EE51075F007A42427
:10072E0009FF74B82510F8E612079F75F00A84C009
:10073E00F07E2012E83A7E28742C12E8B4D0E07EC7
:01074E002A80
:10074F0012E8A112075F0510C3E558951050C32298
:10075F00121BABF8603964046035E8146510702F14
:10076F00121875E5BC12079FF8C313923D7E1C1239
:10077F00E8507E28742C12E8B4E4303D067405B8B6
:10078F000001147E2A12E8A17E18742312E8B42205
:10079F00305D1275F036A42432FBE435F0FC125FA5
:1007AF00BE125FBEEB221207C712811CDFFB2212A3
:1007BF0007C71288FEDFFB2275C70375C6F078B82E
:1007CF007F042275C70375C6F375B901E5BFB54838
:1007DF0031E55924F1402BE55975F00484A9F02433
:1007EF00F0F5C675B901C5F0A9BC600CA9BD1460C0
:1007FF0007A9BE146002A9BFE975F005A4F985F039
:10080F00CC22121875A9BD75CC00221255F712F122
:10081F007B75370390BC2412272590082D73020295
:10082F0070020B2B021D1C020B40020B4B022117F7
:10083F00021DE0020C0C021E14021E5A0221660257
:10084F001D96021E9F1255F712F17B75370490BC4F
:10085F00E712272590086773020270020B5A020BEA
:10086F0065020857020B7B020B86021A1D020857FE
:10087F00020B95020B70020BAF1255F712F17B753D
:10088F00370B90BD3412272590089B73020270021C
:0B089F001ACB021ACB02092102095FEC
:1008AA000208C20208E50221FC021B70021C3B027C
:1008BA001BE4021CCC020BC9121861E5BF1470C1FB
:1008CA007F2E1218981F121861E5BDA2E6120BE1DD
:1008DA00121861E5BD92E6F5BD80A37F371218981C
:1008EA0012185CA8BFE812091912F1851000081045
:1008FA00010D10021280EE18B802EA780A80E608A2
:10090A00B80BE2780380DE12185C88BF0208887F81
:10091A00367E2CE802E7827F1C121898121861A80A
:10092A00BE12095312F18510000810010D100214AD
:10093A0080EF18B800EB780B80E708E824F450E160
:10094A00780180DD88BE0208887F1B7E35E875F055
:10095A0005A402E77C7F25121898121861A8BF1215
:10096A00099112F18510000810010D10021480EF90
:10097A0018B800EB780980E708E824F650E1780116
:10098A0080DD88BF0208887F247E3BE802E8D31214
:10099A001857E5BF75F03CA4ACF0FDE5BE75F0054F
:1009AA00A42DFDE5F03CFC121861E5BF1460367514
:1009BA00F005A485BEF0A42DFFE5F03CFE7C007D89
:1009CA003C125EAFC005EF75F01884E5F07F2D7E0E
:1009DA002412E77C7E30743A12E8E67E35D0E012C3
:0709EA00E77C02F1857F2D7F
:1009F1007E0590C1C2128149121861E5BDA2E67F50
:100A01002D12206402F18512F2FC122819120A1427
:100A110002023D7F177E0290B88A1281497F4C7E87
:100A21000290B8A1128149AC5DAB5C7F577E041284
:100A3100E72912188485BC6285BD63E56124F8400D
:100A41004490B8AC7F37128137AE61AF607C017DD5
:100A51005E125EAFC3741F9FFAAC63AB62EC33925C
:100A610017500312602F125D96AB047C0030170300
:100A710012602F74F52BFB74033CFC125D6C7F3705
:100A81007E1512E6A190B8B97F697E0F128149E502
:100A910060240FFBE43561FCA25C923BD25C7E1EBC
:100AA10012E6ADA23B925C7E30742012E8E67E36FF
:100AB100742012E8E6E5602562FBE5613563FC7FA1
:100AC100227E0412E729E56245637016742E7E3A90
:100AD10012E8E612F18510000D1001151002260230
:100AE1000A3C742080E81562E562B4FF0C1563804E
:100AF100080562E56270020563E53524F55003756A
:100B01003301020A3C1218848562BC8563BD02551B
:100B1100F77F637E00747212E8E212289C40087F1E
:100B21006312812E1255FE02057012186BE5BCA2EC
:100B3100E77F0A120BE4E5BC92E7F5BC02081A7FD5
:030B41001CA20DE6
:100B4400120BE1920D80097F25A20E120BE1920E89
:100B5400120C0002081D7F0AA20F120BE1920F80F3
:100B64002A7F13A208120BE19208801F7F52A20C65
:100B7400120BE1920C80147F25A20B120BE1920B55
:100B840080097F2DA209120BE19209120C000208C0
:100B9400577F49121861E5BDA2E3120BE1121861F7
:100BA400E5BD92E39266F5BD0208547F5B121861BD
:100BB400E5BDA2E5120BE1121861E5BD92E5924391
:100BC400F5BD0208547F6D121861E5BDA2E0120B59
:100BD400E1121861E5BD92E0F5BD020888120BF63A
:100BE4008F1F9217121898AF1F1F7E39128E4BA2B7
:100BF400172212187085BC2B85BD2122121870850E
:100C04002BBC8521BD0255F712186B85BE12120C40
:100C14002112186B8512BE1255F702081D75A6FF26
:100C240012F2FC12AA63740712F2E88FF07406122F
:100C3400F2E8EF2512C395F0A2E7923D4010FD249F
:100C4400CD50027D32AC05C3743F9DFD800FF4048A
:100C5400FD24C850027D37AC0574402DFD7F401241
:100C6400DD6D7E1212F2170EBE1EF91F303D020F0B
:100C74000FEF6D70EDE536700A753606EC2513F549
:0C0C8400148C13120C9F12F18510000755
:100C90001001083002072215128002051280827F9F
:100CA000377E28742E12E8E67F347E21740A303DA8
:100CB000010412E901E514FC249C50027C637F349A
:100CC0007E2DEC12E1F47F437E1E12E6A97E00E544
:100CD0001212E8407F057E0290BCBB1281497F6DF5
:100CE0007E0190BCC612817C7F747E0490BCD712BA
:100CF000817C02281990B8C37F1B7E101281491293
:100D0000F18512F13AC214C21512F16A020522D21B
:100D100014D215E4F56EF56D756F02751501751435
:100D200001754280D233120D8EE51565146005857C
:100D3000151480F0C24D12F2FC12847D90BE541244
:100D4000817A129B0478B8E60460AA751000D24E2E
:100D50001211E9304D07C24D12F141C202C23310E7
:100D6000000810012910024880F3E5151460C7D26D
:100D7000D5129A05E56F24FE400430339222129B6F
:100D80000478B8E630E6EA30D5221515801E1299AF
:100D9000E5E56F24F25005129A058010129B047845
:100DA000B8E630E6E9C2D50460C7051530338722BE
:100DB000E53514601324BE5003020D052419509D1F
:100DC00012284D12F1858095E4F511F512122819BB
:100DD000E511451070087F7B90BA3412817A12E1D8
:070DE000111211C38511126D
:100DE70012F185E51110001310013410020280F38F
:100DF700E53524E65056D24D020D366004151180B4
:100E070015E5107003020EDD151012F2FC1211E742
:100E17007407F511F5127F42129C5DDFFB80A72452
:100E2700F940157479951775F00D8414D395114011
:100E3700B20511129C26808E203CA8303DA50510D6
:100E470012F2FC1211E7129C26020DC8783A79714A
:100E570012DB8E854E63854D62120FBD756C7F75F3
:100E67006BE8756AA512F2FC1228F012E111121153
:100E7700361215EA12168A1216CA12F185100008E0
:100E870010011810023780F5120F99E56B241840EE
:100E970005120FAC801C129C5D8017120FACE56B1E
:100EA7002414500BE56A24135005120F998003127E
:100EB7009C2EE53524F550AD75330180A8787179FE
:100EC7003A12DB8E85634E85624D754C0012F2FC3B
:100ED7001211E7020DCD12290C12F1851000051031
:100EE700010580F8020DCDC25312547312284D74B8
:100EF7004012EFEF747812EF9F746312EF9F7467DD
:100F070012EF9F742312EF921231A6E51512EF7EAE
:100F170078B8E6C4540344400412EF9F12EFC6E4C6
:100F2700F51412994D129A53747012EFEFE51412DB
:100F3700EF7E75A700900401E012EF92A3E012EF95
:080F470092A3E012EF92A3E077
:100F4F0012EF92A3E012EF92A3E012EF9212EFC60C
:100F5F007F7B7E1DE51412E85012F1851002287573
:100F6F00A70090042275134275120F753800E01216
:100F7F00EF7EA3D512F812EFC6D513EC0514303C53
:100F8F009C12303F12F14B020DCD74F1256AF56AB8
:100F9F00E56B34FFF56BE56C34FFF56C22740F25B0
:100FAF006AF56AE4356BF56BE4356CF56C22756C9C
:100FBF007F756BE812B144E5104511C2306002D263
:100FCF0030303B028060303011E51112994D129A8A
:100FDF0048129A9890055B121123E51112994D1240
:100FEF009A86900411756AA512111C056B7FEF127A
:100FFF001125129A98900411056B756A9412111CA1
:10100F00056B7F6C12112512B1417F8312112512CE
:10101F009A7B129A86900400E020E60990041175DD
:10102F006A8312112322303011E51112994D129A51
:10103F0048129A981210D5121120E51112994D12DB
:10104F009A861210D5756AA5121120129A9812104D
:10105F00D5056B756A4A121120129A7B129A8690E7
:10106F000400E020E65D1210D5756AEF1211201210
:10107F009A981210D5056B756A94121120129A7BEB
:10108F00129A86900400E020E6391210D5056B7590
:10109F006A39121120129A981210D5756ADE7F22C2
:1010AF0090061012112512B1417F83121125129A49
:0B10BF007B129A86900400E020E608F7
:1010CA001210D5756A83804E02B14175A701900648
:1010DA001005A7900411AE838E16AF828F17E0F524
:1010EA00451212D5F5441212D5F5537C007D2D1206
:1010FA005EAFED6414600685168385178212176F3A
:10110A001260A905A7EDF0A305A7A3E58324FA5069
:10111A00C5227F0080059006107FA575F08412B164
:10112A007FE0F5F7A3DFFAD2B202B0FDC06FC06E5E
:10113A00C06D756F7F756EE8756D0012B191751788
:10114A00237E00D2D57B0579FF7A007C1520D50154
:10115A001CE4F5F7E4ADF71212B620320CB5010023
:10116A005001F9B502004001FADCE6C3EA9904FA33
:10117A00E904F5F0EA141445F07003E4F9FAAF0152
:10118A00EA600612F2170FDAFADB0B10D506D2D58F
:10119A007B0580027B030EBE40ADD2B27E087F245F
:1011AA0012F2177F2812F2177E3712F2177F2412D3
:1011BA00F217D06DD06ED06F22E51275F00DA4FF34
:1011CA0074739FFF7E00742012E8B4E51175F00D68
:1011DA00A4FF74739FFF7E00743F02E8B4C24EE41A
:0F11EA0012994D12E111751779121206203C0C63
:1011F900203D09304EF4E53524FA50EE22751201EE
:10120900129A53C23D75A700900400E0F5F0A2E5DB
:10121900923BB4FF03D23C22E5176479600320F6C0
:10122900F490042275160475130FE5165401441041
:10123900F514E0FD303B2AF545C083C0821212D572
:10124900F5441212D5F55312176FAC06AB0712DF2E
:1012590047FDD082D083D5130875130F741E12125F
:10126900D7AE161212B620320312F217A3303B2260
:10127900E58324F8501C0512E51224FC401F129A3C
:1012890053900400E030E604D23C801190042275AA
:10129900130FD5149D0516E51624C0508D12F1853E
:1012A900E51724F3F51724EE4002D23D22C232EDB0
:1012B90004601624FC501224A350027D5FEDC42360
:1012C900541FFFC3E5179FFF22D23222740F2582D4
:1012D900F582E43583F583E022D22B12141FD21450
:1012E90012ED9D12F2FC1228F912E14412151112A5
:1012F90013F5751604751500E530651360FA853028
:1013090013533203E53270F01216ED12173C05152E
:10131900E51524C45006751500129C3D301A0312B8
:10132900179DE539600912139112136312F185753E
:0B133900A6FF10000810011810020AA7
:1013440080BB301AB81214E38009201AB012B23BE1
:101354001214B6808E1214E3C237C22B020522E5A2
:101364001570030215377F0A147001221470077E6A
:1013740024E53E02E77C1470097E1378AEE602E7AA
:101384007C22146001227E35E53F02E77CED24E1F6
:10139400400574769D801A24E2400EED941E337548
:1013A400F00384FC74589C800804C313FCC3744485
:1013B4009CFCAE167F7612F217EFB5040B1FEF24D8
:1013C400ED500812F24780F51F80EBE516FE20E091
:1013D400147F2612F2177F3512F2177F4412F21788
:1013E4007F5812F2170516E51624C050037516042B
:1013F400227F24740812E89F7F33740612E89F7FCB
:1014040042740412E89F7F56740212E89F7F657449
:101414000112E89F7F74740002E89FD215C21AC2B9
:101424001F12B23B1214BDE4029121C22BC214124A
:10143400141F75A6FF758AFC758CFFE4F532F53927
:10144400D205D23712ED9D12F2FC129C3D12E144FA
:101454001215111215841228F979197B1E123B17E3
:1014640079557B1E123B1779917B1E123B1779CD60
:0E1474007B13123B1710002210012F100221D3
:10148200301A11E53924F14008E532240340058081
:10149200EF12179DE532240250FA80981214E3806D
:1014A200DF201ADC12B23B1214B680D41214E3C24B
:1014B20037020522201A57D21AD21F12185C85BC95
:1014C2004C85BD4D85BE4EE54C700FE54D54037005
:1014D20009753910E4F5520291217401129A26809D
:1014E200E6301A2AC21AC21F12185C854CBC854DFE
:1014F200BD854EBE1255F7E4129121D214E54C700F
:1015020008E54D540370028003121801C214227FB1
:101512000A7E007401205A02740312E8CC7E05741C
:1015220058201A02742D12E8E67E0B7446202B0214
:10153200742012E8E6C3E4954DFB740E954EFC4B05
:10154200F5177A46205A027A17125DA48C038D048D
:10155200302B0CC3EC13CB13CBC313FCEB13FB12DA
:101562005FBEC0E07F017E00EB12E7ED7E0AD0E0B5
:1015720012E8CCE517700A7F2F7E1090BA0A12810A
:1015820049227F197E0590BE711281491215EA75B2
:10159200A7008552827583057E3F7C00E0B504007A
:1015A2004001FC1582E582B4FF037582B3DEEDECE7
:0E15B200230475F0038423FD249C50027D6306
:1015C000ED75F00A84C0F07F237E2512E9010F0F2C
:1015D0007E2D742E12E8E61F1F7E32D0E012E90144
:1015E0007F267E0590BE7C02817C7D057F3A12DDE0
:1015F0007FEF240FFFDDF778087F387E01E812E8DF
:10160000A1EF240FFF1818B8FEF17F3D02DDDE7553
:10161000A700F5827583057E3FE92B203D012B95C0
:10162000324031E0FAC374769AFF1582E582B4FF46
:10163000037582B3E0FAC374769AFD1216551582CB
:10164000E582B4FF037582B3E0FAC374769AFD12A3
:101650001655DEC522BE3F0122203D1712F217C3E8
:10166000ED9F70012240060F12F21780E81F12F260
:101670001780E212F247C3ED9F70012240060F125D
:10168000F24780EF1F12F24780E912B17C1216A4D4
:10169000FD7E001216A4FFFC1216B38C050EBE4090
:1016A000F2D2B222E4F5F7E4E5F704C313FAC37407
:1016B000769A2212F217C3ED9F70012240060F1294
:0D16C000F21780EF1F12F21780E9C3E56BEF
:1016CD0094E8FCAB6A7A08125D967D0078A5125FEE
:1016DD003FAE037F259016E802E91203052070F84E
:1016ED0030B226758001C2B275F72475F700E4E5B6
:1016FD00F7F545F5F775F700E4E5F7F544F5F775FA
:10170D00F700E4E5F7F553D2B212176F0260A97531
:10171D00A700758305855282EDC313F00552E5527E
:10172D00244C5003755200E532B401037539007530
:10173D00A7007583048539820539E53924F05004F5
:10174D0075391022EDF0E5822410F582E545F0E5BE
:10175D00822410F582E544F0E5822410F582E553EC
:10176D00F022E54530E702F404F5F0A4AEF0FFE514
:10177D004430E702F404F5F0A42FFFEE35F0FEE55A
:10178D005330E702F404F5F0A42FFFEE35F0FE22FE
:10179D00E53924F0407904600122E54E24F2406FD2
:1017AD00240C506BE54C704CE54D54037046740899
:1017BD0030100104302B024410205A024420301FF7
:1017CD0004C21F444075A7009005CEF0A3783A7F60
:1017DD000612DBA97F07301010786A7F0312DBA990
:0F17ED0078707F1012DBA97F1A9005CE12184278
:1017FC007422129A2675A700900400205A0F758245
:10180C0010121820758220121820758230121820A0
:10181C0075390022E54C240E40047D0F800F04FD29
:10182C0074109DFCAF04121842EC129A26AF0512EC
:10183C001842ED029A2674061299867402129A10B6
:10184C00E0F5F7A3DFFAD2B2029B3775C6F4803508
:10185C0075C6F5803075C6F6802B75C6F780267573
:10186C00C6F8802175C6F9801C75C6FA801775C636
:10187C00FB801275C6FC800D75C6FE800875C6FF10
:10188C00800375C6FD75C70375B9012274721F12EA
:10189C00E8E20F02F1857F0A1218987E2A12B23BF9
:1018AC00121875A8BF1218D61000121001051002DC
:1018BC001580F508E824E750EC781880E818E83033
:1018CC00E7E3780080DF88BF805F7F097E0590C0EA
:1018DC0083B80C0390C07D1281497E27E53D2824F6
:1018EC000C75F01884E5F012E77C7E33743B12E83B
:1018FC00E67E35E53E12E77C02F1857F13121898DF
:10190C00120BF6121938100008100105100217807E
:10191C00F2105C07205D0BD25C80E8105DE5D25DB7
:10192C0080E1D25C80DD852BBC0202CD205C1020D6
:10193C005D1890C0D67F127E2312814902F18590EA
:10194C00C0EA205DF090C0DD80EB90C0E380E67FC4
:01195C001C6E
:10195D00121898121870A8BF1219921000081001D1
:10196D001110021A80F2E824F250031880EA780D63
:10197D0080E6E824E740030880DE781980DAE8F590
:10198D00BFF54380A37F1B7E26E412E8D3E8232313
:10199D00B464087E26740112E8D3E47E2E12E77C2F
:1019AD0002F1857F2512189812187FA8BCE812192C
:1019BD00EB12F18510000810010D10021F80EEE8EA
:1019CD0024E050E9188006E824CF40E10812187F82
:1019DD0088BC1255F7D21512ED9D80D180157F244C
:1019ED007E3724E202E7ED7F2EA20A120BE1920A66
:1019FD00120C000202D07F37121861E5BDA2E4126D
:101A0D000BE1121861E5BD92E49267F5BD0202CDBE
:101A1D007F367E00747212E8E20F7E16743F12E874
:101A2D00B412186BA8BD121A9612F1851000081089
:101A3D00010510021080EFE824875004240A80026B
:101A4D0024E8F880E17F377E16742012E8B47E2CEE
:101A5D00743F12E8B4121A9612F1851000081001A5
:101A6D001410022080EF18B80904787880E7B87850
:101A7D00E478E780E008B87904780A80D8B8E8D52A
:101A8D00787980D188BD020854E82487923DE850CA
:071A9D000224917F367E3028
:101AA400C313923B12E7ED7E3CE4303B0274051213
:101AB400E8CC7E1A90BFC7303D0390BFCB1281495A
:101AC4007F3C7E3A02F2177F127E00747212E8E2C3
:101AD4000F7E20743F12E8B412185785BE1085BFDC
:101AE40011121B5210000810011110021B80F21574
:101AF40011E511B4FFEB75111780E60511E511240A
:101B0400E850DE75110080D9121B527F137E2074B9
:101B14002012E8B47E31743F12E8B412F18510004B
:101B24000810011110021B80DF1510E510B4FFD856
:101B340075100B80D30510E51024F450CB751000FC
:101B440080C61218578511BF8510BE0208887F12FF
:101B54007E24E51112E77C7E30743A12E8E67E3585
:101B6400E51075F005A412E77C02F1857F4912188F
:101B740098121BABF853BF1F121BB11000081001C1
:101B84000D10021280F218B8FF02780480EA08B837
:101B94000502780080E212185788BD1255F7B80084
:101BA4000302088B021C3B121857E5BD227F487EB6
:101BB4000590BFE1128149E8601CB4040A7E0590D7
:101BC400BFD6128149800C90BFED1281497E38E85E
:101BD40012E8D302F18590BFE87E2912814980F38F
:101BE400121BAB601D640460197F5B121898120B02
:101BF400F6121C1612187010000B10010810020CBB
:0C1C040080EF02088B105FE9D25F80E5E2
:101C1000852BBC020888121BAB601F6404601B7F0D
:101C20005A7E0590BFE11281497E2390BFF1305F5B
:101C30000390BFF812814912F18522121BAB700389
:101C400002088B7F527E11121898121875A8BC12C8
:101C50001C7B12187510000810010810020880EF94
:101C60001880EC0880E912187588BC1255F7121814
:101C70007FE875F005A4F5BD020888121BAB604B28
:101C8000E875F03270040475F028A4ADF0FC305D06
:101C900011ACF0FB7A8A125DA4EB30E7050CBC00B6
:101CA000010DAE05AF047C007D64125EAFC005EF90
:101CB0007F517E1A12E7997E2C742C12E8E6D0E050
:101CC0007E2F12E77C124DBF12F185227F6412181D
:101CD00098121875A8BD121CFD10000810010F10F5
:101CE000021680F218E824CD50EC783280E808E83B
:101CF00024CD50E2780080DE88BD0208887F63E84A
:101D000023C2E012E32775F06484C0F07E2612E857
:101D1000D37E2C742C12E8E6D0E080A47F13121836
:101D20009812186BE5BCA2E7923DC2E7F8E8121DD5
:101D30006012F18510000810010D10021280EE18DB
:101D4000B800EA783280E608B833E2780180DEE84D
:091D5000A23D92E7F5BC79A1F770
:101D5900021E117F6380027F12547F305C01237E53
:101D69002875F06484E5F075F00A84C0F012E8CCB7
:101D79007E2D742C12E8E6D0E07E2F12E8CC0F7E7F
:101D89003590C0F0305C0390C14C02817C7F6412B5
:101D9900189812187AA8BDE8121D5C12F185100076
:101DA9000810010D10021280EE18B8FFEA780F80B2
:101DB900E608B810E2780080DE88BD02081A7F5272
:101DC900121898121875E5BE7F517E2C128EA0F557
:101DD900BE79A2F70202CD7F37121898121870A89F
:101DE900BC5300037F367E32E812E8D312F1851026
:101DF900000810010710020780E718180880E2E5BB
:101E0900BC54FC48F5BCF52B02081A7F49121898F6
:101E190012187FA8BE121E4B12F18510000810017E
:101E29001110021A80EFE8240AF8242450E778DB1D
:101E390080E3E824F6F8247F40DB788180D788BEE8
:101E490080C6E8F424DC75F00A847F487E3B02E80A
:101E5900D37F5212189812187FA8BF121E9212F13E
:101E69008510000810011110021A80EFE82408F803
:101E7900245750E778A880E3E824F8F824A040DB49
:101E8900786080D788BF021E11E8F424A923C47F93
:031E9900517E3B3C
:101E9C0002E8D3123948754A00D210C211D214D2BA
:101EAC007575791475340012F2FC7F007E0290BCBB
:101EBC0090128149904DE87F087E2612E912E52B9D
:101ECC0054030F7E3912E8D312283412E57A12A784
:101EDC008B12F18510000810011A10022480C52005
:101EEC007504057980BE1579E579B4FF05C2757561
:101EFC00790180B02075EB1579E57970A7D27580E2
:101F0C00A3C210C21402081D121870E5BE7F097E10
:101F1C003A02E8D3121875A8BF1218D6120BF61293
:101F2C001938A8BF12199212187FE5BC1219EB7F51
:101F3C002DA20A1220647F36A26712206412187A2E
:101F4C00E5BC7F3F7E3212E7F3A8BE1203251218C0
:101F5C0057E5BC7F487E3212E7F3121875E5BE7F59
:101F6C00517E2C02E8D3120BF67F1BA20D122064BB
:101F7C007F24A20E12206412186BE5BC121D607F28
:101F8C0009E5BCA2E7122064A8BF12215212187AEC
:101F9C00E5BD121D5CE52B54037F367E3212E8D36F
:101FAC0012187FA8BF121E92A8BE121E4B121861E7
:101FBC00A8BC022197120BF67F09A20F1220647F96
:101FCC0012A208122064121861E5BDA2E37F481228
:101FDC002064E5BDA2E57F5A1220647F51A20C1249
:101FEC0020647F24A20B1220647F2DA2091220648E
:101FFC0012186BA8BD021A9612185785BE1085BF11
:01200C0011C2
:10200D00121B52121861A8BE120953A8BF120991D2
:10201D00120999121870E5BE7F3F7E3A12E8D3126D
:10202D00185CA8BF120919121857A8BD121BB112BE
:10203D001875A8BC121C7B121870121C161218757C
:10204D00A8BD121CFD121861E5BDA2E07F6C8007D2
:10205D00120BF67F48A25E744E400274597E3A020E
:10206D00E8E6120BF67F097E347401205A027403E0
:10207D0012E8D37F36802E1287FA7F7312845112A5
:10208D0088497F6C1284607F2D801A121861E5BD1E
:10209D00A2E77F63122064121870E5BE7F097E3AB5
:1020AD0012E8D37F481220C37E1E90BA243053030A
:1020BD0090BA1F028149121861E5BDA2E192532227
:1020CD001218981F1220B212F18510000810010588
:1020DD0010020D80EFE5BDB2E1F5BD1255F780E4BC
:1020ED0022128018EBF516F5147F6C128460127FA6
:1020FD00FC7F647E23E51612E850C3E5169514F5B2
:10210D00167F731284517F2D809B7F2E121898128B
:10211D00186BA8BFE824FA5002780312215212F16D
:10212D008510000810010D10021280E818B800E4A7
:10213D00780580E008B806DC780180D8799DE8F74D
:10214D00F5BF02081A7F2D7E2C7420B80502742E5F
:10215D0012E8E67E32E802E8D37F5B121898121877
:01216D006110
:10216E00A8BCE812219712F18510000810010D107D
:10217E00021280EE18B800EA780380E608B804E28E
:10218E00780180DE88BC02081A7F5A7E2CE802E8AD
:10219E00D3D26875480A12B23BD21412384B128948
:1021AE0025123FDDC26B12020280F3D214751501A7
:1021BE001287B475B901E5BC20E71C1288E475A638
:1021CE00FF12893112283F12F18512825110000F31
:1021DE00500512837980E70515E515242050D102AC
:1021EE00057012220202023D1222020205AD1222D7
:1021FE000202088B12220E1218708548BE0255F785
:10220E0012383D12385712646F12F2FC90BAC2D2D5
:10221E004912A002129FBB1227EF12F18510001473
:10222E0010010510021B80F50548E548640A70028E
:10223E00F54880CF1548E54864FF7003754809805E
:10224E00C2854849123857E5582212B23B12383D22
:10225E00854849C250E558B40F02D25012646F80BF
:10226E003AD22775480A12384B12646F12F2FC12DA
:10227E009F2590BF9920290390BFA31228CBC26A35
:10228E00123FDD106A0280E1C22712878C85494811
:10229E00122664123857D22912646F12F2FC90B9CA
:1022AE00D512A00020500E1228B512F18510001084
:1022BE001001AE80F812283F12F18510000280FB4B
:1022CE000205AD12383DE55830E7137F1B90BF83F2
:1022DE007E0512814912F18512F13D0205AD1238CB
:0722EE005712646F85594986
:1022F50012F2FC12282990BFA312A000129FC5124A
:10230500F18510000810010A10020C80F5122369EE
:1023150080DB12237680D612F2FC12282990BAD1DE
:1023250012A000129FC5129FC912F1851000081056
:10233500010A10020C80F512238280DB12239080A3
:10234500D612262A12385712646F12F2FC90BEEC90
:1023550012A00012286E12F1851000051002888067
:10236500F80205AD0559C3E558955950037559004F
:10237500221559E55964FF7003855859220549D33B
:10238500E5491495584003754900221549E5496406
:10239500FF700585584905492212383DE55830E753
:1023A500057F240222DB12385712646F12F2FC906B
:1023B500BADC12A0001228C012F18510000A100123
:1023C5000280F81226D380DE0205AD12383DE558AD
:1023D50030E7057F2D0222DBC26B7559FF12646F52
:1023E50012F2FC122819E55930E70312283490BA85
:1023F500ED12A000129FD512F185E55820E70610D1
:10240500000810011110021B80F00559C3955950A1
:10241500CF7559FF80CA1559E55964FE70C28558B4
:102425005980BDE55920E711D26B75A70075830763
:10243500C4F582E0B2E7F080A7306B031226810273
:1024450005AD12383DE55830E7057F360222DB122F
:10245500385712646F12F2FC90BAF812A0001228D5
:092465009C40091226C81226FD54
:10246E001224740205AD121875E5BD75F00584F5DC
:10247E00BCF5BDF5BEF5BF1207C71255F705C6DF91
:10248E00F92212383DE55820E7087F5190BB020231
:10249E0022DE12F2FC90BFAE12A00012283F12F103
:1024AE0085125457D2AC10001FE55830E7F8306D46
:1024BE00F51225CA7E207F00501390BFFF12817C3B
:1024CE0012F18512F13D80CAC2AC0205AD1B8B1311
:1024DE0090B9F312817C12F185C26B7B007514B832
:1024EE001226BD1288B31288655025A814E8243828
:1024FE004004A60105140BC3E5139B50E678B812F1
:10250E0026FF306B0312860612385712646F8082D4
:10251E001287FAE51660E6D26B128910C003128795
:10252E00CBD003A91580C412383DE55830E7057F9E
:10253E005A0222DB12385712646F12F2FC90BB0D56
:10254E0012A00012286312F18510003510010280CE
:10255E00F875460512259250157F007E3574079545
:10256E004612E85012F18512F13DD546E7D390BFE1
:10257E00B9500390BFFF12A00012F18512F13D80F9
:10258E00B30205AD12545712EFDE745212EFEF7410
:10259E005412EF9FE5580475590012EFCD128200C8
:1025AE00401612878C1288E4128251400B0559C3D3
:1025BE00E558955950ECC322C2ACD322125457D2CF
:0D25CE00AC12F017204CF1B440F712F01CD5
:1025DB00B4400312F01CB452E2F53812F01CB454A0
:1025EB00DA12F01CFA60D424EF40D012F01CE5385C
:1025FB0070C912F01C12F01C1281E57B007E0312D5
:10260B0082DC50102050B412F01C204C03B440F765
:10261B00DEED80A71288C30B1281E5DAE0C322122C
:10262B00270AE55924C8F88602E54924C8F99860B9
:10263B0013146010500F18E608F618E86970F7A726
:10264B00021226FD22E559640F60F91908E618F607
:10265B0008E86970F7A70280E812270A78C8C25009
:10266B00E6B4FF02800708B8D8F6D25022B8D702DA
:10267B00D250A615807C78B812270CE4F9F5A77513
:10268B008307E9C4F582E030E70AE924B8F8243877
:10269B00400276FF09C3E5589950E71226C878B86F
:1026AB0079C8E6B4FF028002F70908E8243850F233
:1026BB00804079B877FF09E9243850F82279C87738
:1026CB00FF09E9242850F82212270AC23D78D7B611
:1026DB00FF04A900D23D18B8C7F5203D0279D819DF
:0826EB0078C8B6FF0122C3E824
:1026F300995007C6C7C6081980F478C81227177FF0
:102703000412811CDFFB2278C81227177F0412886A
:10271300FEDFFB2275C703E54875F004A42480F5AA
:10272300C62212F2FCC23C12813BE53760531460AF
:102733004D14604514603D14603514602D146025FC
:1027430014600E146010146012146035146011804C
:102753003012205D802B12206F80261220EE802104
:10276300122004801C1220988017122084801212D9
:102773001FC1800D121F728008121F208003121FB9
:102783001412F18512F14112281912AE5AA81F082A
:10279300E814C23BB51D02D23B75F007203C03751C
:1027A300F009A4FF7E00303C0C7420303B02743EE1
:1027B30012E8B4800A740B303B02740A12E8CCD8D6
:1027C300CF12F185E51D10000810011010021880CA
:1027D300B9651F7003751DFF051D80AE7005851F4C
:1027E3001D80A7151D80A375F003A4227F7B7E00A7
:1027F30090BF0512817CE54824F640087E0A90BF0D
:102803006612817C2212847D7E05745B12E8B07EA1
:102813001D745C02E8B01228087E3490BF16028152
:102823007C12847D80031228087E3190BF1A0281B6
:042833007C122808E3
:102837007E3190C00A02817C12847D7E00800C125A
:10284700847D7E18800512847D7E2D90C00A0281CA
:102857007C1228637E3190BA2E02817C12283F7E3B
:102867001A90BA3402817C12283F80B912283F7E21
:102877001890B9DF02817C12283F7E1A90C011029E
:10288700817C12847D7E0090B9DF12817C7E31903D
:10289700C01102817C12283F7E1A90C01612817CDB
:1028A70012F185D3100006C310010280F622122808
:1028B7003F7E1A90BACC02817C12283F7E1890BACC
:1028C700E602817C7F007E2012817C02F1851284E2
:1028D7007D90C01C02817A12847D90C02D02817A7E
:1028E70012847D90BE3202817A12847D90BE4302AB
:1028F700817A1228467E2C90BE6B301A057E009096
:10290700BE6502817C12847D90BEC602817A125F09
:10291700A10FBF00010E8E04EF799AF7FB7F017EAE
:1029270028A25C924EC25C12E6E6A24E925C78B890
:10293700E654F070091F7E2890BE2D128149E4FFEE
:10294700FE78ADE612E7E77E0A742C12E8E67E0C05
:1029570018E612E7E77E16742C12E8E67E1818E6EA
:1029670012E7E7303D0A90BE277F147E0112817C73
:10297700227F097E0178AEE612E77C7E0D743A125B
:10298700E8E67E1278BDE612E77C7F097E2378BEF3
:01299700E659
:1029980012E7827E30743A12E8E67E3508E612E7DE
:1029A8007C0886040886037F127E0012E6AD12E7D3
:1029B8003178C4E612E3277E2912E7997E3B748BAF
:1029C800305D010402E8E6780C7F1C7E02E812E81C
:1029D800347E09742E12E8B47E0CE51012E834EF48
:1029E8002405FF7E1E12F2170EBE3FF9EF2403FFE7
:1029F800D8D922C3740C951375F008A4241CFF7E43
:102A080017742012E8B4C3740C951175F008A42447
:102A18001CFF7E17743F02E8B4751600AD6FAC6EEC
:102A2800AB6D7403129991E4F5F7A4E5F7F9540F27
:102A38006046E4F5F7A4E5F76510703CE4F5F7A403
:102A4800E5F775F008A47F80CF9FFFE4F5F7A4E5CC
:102A5800F7D2B2241DFE12F217E954F0601A1F12C1
:102A6800F217EE6516700DEF651770081F12F21752
:102A78001F12F2178E168F17D2B21299AFED30E7E8
:102A8800A122AD6FAC6EAB6D7403129991E4F5F7AA
:102A9800A4E5F7540F601DE4F5F7A4E5F765107099
:092AA80013E4F5F7A4E5F765114C
:102AB1007009D2B28D6F8C6E8B6D22D2B21299AF2A
:102AC100ED30E7CBD32278B97998E6F70809E6F734
:102AD10022D215C210C21112F2FC129AC6303C1356
:102AE10090B8BC7F1C7E0512817C12F18512F13AEF
:102AF10002023DC221C24D1299F0E56F20E7E112B9
:102B01009B0479B8E7540F60EEE764FF60D279B9AE
:102B11008710098711302109799887100987118059
:102B21000A12F2FC122978C23D800512F2FCD23D54
:102B31001229151228191229CF12F185122A21857D
:102B410011131229FB85111312F1857998A7100928
:102B5100A711E59030E20FC221304D24C24D12F190
:102B61004112F17B801AE53524AA500302023AE5AD
:102B71003524C3500B90BE1A7F7312813712F18531
:102B81002021C810000810011C10023780BDE5117A
:102B910014F51170AD75110C1510E510B407005046
:102BA1008A051080A679B9E76510700609E76511F5
:102BB1006099E51104F511640D7087751101051017
:102BC100022B2C122A8A501DC3740C951175F00822
:102BD100A4241BFF7E0290BE1012814912F18512BE
:102BE100F141022B2C129B04122AC7E59020E2101E
:082BF100E53524DC500AD22175
:102BF900D24D129AC6022AF812F2FC1228E71229BB
:102C09001579B8E75403600312297812DB6279B8A1
:102C1900E764C3701712DB6212321912DB721232C7
:102C2900FE756A101298ABD2331234BE12F18510B8
:102C3900001710013279B8E764C370A4100202804A
:102C4900EEE53524FA4099807C1299F0129B04E54F
:102C59006F20E70A79B8E7540F60EEB7FF8212993F
:102C6900D2129B04022BE91299D2129B0479B8E77C
:102C7900540F60F3B7FFED80D012289C40517FC0FC
:102C8900129B221299A2129B4C60F8B4FFBB78C622
:102C9900866C08866B756A0012B1741298AB1218AB
:102CA9008EE56C65BD701BE56B65BC7015E57064E0
:102CB900FC700F78BEE66577700808E665787002E3
:102CC9008049022BE97995A76F09A76E09A76D7944
:102CD90095876F09876E09876D129B0412DB621253
:102CE900DB721232FE756A101298ABC2331233B519
:102CF90090B8D3D23C12813B12278A902D087302D7
:102D09002BE9023F26022D90022C827F6C12812E24
:102D190012F13DD2201299F0E56F30E70F1280B51C
:102D29001255F71256D51256B7022AD2129B04121F
:102D390099D212188EACBFADBE85BDBF85BCBE7819
:102D4900C686BD0886BC1255F712B174E56C6C7065
:012D59000D6C
:102D5A00E56B6D700812B16A12B0FD801F12B12FB7
:102D6A00E56B54036403700612B16A12B0FD129740
:102D7A00FAE56B5403700312B17480CF7F00129B83
:102D8A0022C220022BE912F2FC7F6490C1E5128173
:102D9A00377F7990C1F212813712F18575160010CA
:102DAA00000A10010910020280F505160516C25321
:102DBA0012DB7275370090B8F0122725902DCA736E
:102DCA00022CD8022DB8022FBD022FC2022DB80242
:102DDA002DF1022DF6022DB8022E34022E38022EC3
:102DEA003C022E43022E4712547380031254687811
:102DFA000A122F16740B12EF9D122F5E12EFC612D3
:102E0A002F971298AB1299081297E0129C3D123034
:102E1A00A6D5150C75150A122FA71231CB12EFC6BB
:102E2A00100204E57F70DB022CD8780A8006780449
:102E3A00800278011254738009780A80027801129C
:102E4A005468122F16740B12EF92122F5EE5481275
:102E5A00EF7EE5165403443012EF9F742A12EF9F57
:102E6A0012EF9F12EFC6122F971298AB12990812FF
:102E7A0097E0129C3D1230A6D51548854815122FA9
:102E8A00A7E51C12EF7EE51B12EF7EE51B2548F530
:102E9A001BE4351CF51CE4A27792E7A27492E0A227
:102EAA007392E112EF7EAD75AC74AB73E57DC4121B
:102EBA002ED7AD78AC77AB76E57D122ED71231E9F5
:0A2ECA0012EFC6100204E57F709FAE
:102ED400022CD8540F2375F00584F8C3EB33FBECB4
:102EE40033FCED33FDC3EB33FBEC33FCED33FD205E
:102EF400E713EB28FBE43CFCE43D12EF7EEC12EF1D
:102F04007EEB02EF7EC3EB98FBEC9400FCED9400A7
:102F140080E8884812284D90BE0A12817A12F18501
:102F2400E4F54AF549756A207515011298AB1297B4
:102F3400E0D5150E854815E5492401F549E4354ADF
:102F4400F54AE57F70E5744012EFEF747812EF9F55
:102F5400746312EF9F742302EF921231A6799AE7F9
:102F640012EF7E12DB72E53A12EF92E53B12EF921A
:102F7400E53C12EF92E53D12EF92E53E12EF92E549
:102F84003F12EF92740112EF7EE54A12EF7EE5499B
:102F940002EF7E12DB6DE4F51CF51BF514F51375D9
:102FA400150122753800E51412EF7EE51312EF7E49
:102FB4000513E5137002051422125473800312548E
:102FC4005D12284D12310012F145756A2075150104
:102FD40075A6FF754A0112984F1297E0129C3D1294
:102FE40030A6D5150975151E1230CA12F14F1231CB
:102FF400CBE57912EF7EE412EF7EE57112308B128D
:09300400EF7EE57012EF7EE57B22
:10300D0024ACFFE55F340912EF84EF12EF7EE51576
:10301D0020E036857D56E412EF7EE52EC412EF8456
:10302D0012EFD512F14F10020630559B12303F02B0
:10303D002CD8744012EF9F744512EF9F744F12EF0E
:10304D009F744612EF9F02EFD5E556123065C4FA14
:10305D00E57D1230652A80BFFBC41230722323CB6D
:10306D001230722B22540FFC24F650027C0090304B
:10307D0081EC932200000101010202030303FA24F3
:10308D0040400A24804003EA3322D2E72274FF2213
:10309D0020E703C3132224C022E53F701F7F7B7EF0
:1030AD000078AEE612E83AEE2404FE743A12E8B463
:1030BD00EE2404FEE53E12E83412F18522C015C05F
:1030CD0016D212128FCFC212D016D01578AEE612CC
:1030DD00EF92E53E12EF92E53F12EF92E54512EFCA
:1030ED007EE55212EF7E740A12EF7E74C012EF7EEF
:1030FD0002EFD5744012EF9F745412EFEF744E121D
:10310D00EF9F743012EF9FE5165403443012EF9F7A
:10311D001231A6742312EF92E53D12EF92799AE7E0
:10312D0012EF7E12DB7278ABE60812EF92E6081210
:0D313D00EF92E60812EF92E612EF92E53EE7
:10314A0012EF921236ACE51212EF92E51112EF92DB
:10315A00740112EF7E90C03E12320B756A101298FB
:10316A00AB740212EF7EE412EF7E787B12EF77786F
:10317A007D12EF77787712EF77E4FEFF780712EF88
:10318A007712EF77E57412EF7EE57512EF7EE4129F
:10319A00EF7EE412EF7E12EF7702EFD575C7037563
:1031AA00C6FF75B901C217751D0085BC1C85BD1BFC
:1031BA0085BE1A85BF19125D1CEE12EF7EEF02EF73
:1031CA007EE57512EF7EE57412EF7EE57312EF7EEF
:1031DA00E57812EF7EE57712EF7EE57612EF7EE56F
:1031EA001664016011E55E12EF7EE57A12EF7EE564
:1031FA0016640260012278BCE612EF7E08E602EF4E
:10320A007E75A700E493700122A312EF9F80F51246
:10321A00DB72857946787A796412DB8E746412617E
:10322A00178E471232FE756A20D23D1298AB129958
:10323A0008123335303D09307406C23D8E1E8F1F89
:10324A00E57F602BE54C24FFF54CE54D34FFF54D49
:10325A00454C600512980180D2751D3C1298AB123C
:10326A0099081297E0123335E57F6003D51DED12F8
:10327A0033969033AE12E912203D0DAE1EAF1F12E7
:10328A0033969033A712E912E546FD700B90C1748C
:10329A00305D1190C170800C04700E90C170305D69
:0632AA000390C16C7F38A7
:1032B000024DBAE4FFFC7E05305D047E027FB3124E
:1032C0005EA2AC06AB07125D6C7F38C23DE51C60A8
:1032D00007D23D7E2C12E8A1E51B203D026007D2FB
:1032E0003D7E3012E8A1E51A203D026007D23D7E06
:1032F0003412E8A1E5197E3812E8A1024DBFE5407D
:1033000075F03CA42541FFF54CE435F0FEF54D7C0D
:10331000007D10125EAF0F8F4BAF4CAE4D7C007D29
:103320003C125D827C00AD4B125EAFEE4F70010F20
:103330008F4C8E4D2278647973C2D112334CFF7852
:10334000677976D2D112334CFE02F217C3E796FBAF
:103350000809E796FC0809E796FDA2E792175003D3
:1033600012603775135A30D10E751320B217AA4761
:10337000125DB6AB04AC05E546600B04600BAA46D3
:10338000125DCDEB03FBEB03FBEB543FFBE5132B93
:103390002017029B9B22EE141430E701E4FEEF1489
:1033A0001430E701E4FF2205057088A88870050540
:1033B0002020F8202012F2FC7E1E7F1C12F217DF64
:1033C000FB12F2177E1E7F1C12F217DEFB7E1D7FA2
:0633D0001D12F217DEFBE6
:1033D6007F007E2178ADE612E8347E29742E12E84D
:1033E600B47E2D18E612E8347E35742E12E8B47ECB
:1033F6003918E612E8347F077E21745412E8B47E49
:1034060025744F12E8B47E2D78AEE612E8347E3588
:10341600743A12E8B47E39E53E12E83478AE1236D4
:10342600AC7F0E7E21744C12E8B47E25744112E8FE
:10343600B47E2DE51212E8347E35743A12E8B47E75
:1034460039E51112E8347F157E25744412E8B47EFE
:103456002DE54012E83A7E35743A12E8B47E39E535
:103466004112E8347F217E0190C13F12817C7E0E9D
:10347600AC77AB7612E6E67E2B85795F85787B1294
:10348600EC917F287E0190C14312817C751D2B75BE
:103496001E10E5741236607E25742F12E8B4751D71
:1034A6002D751E2BE5751236607F367E0290C12F74
:1034B60012817CE57212364A12358E20330312369B
:1034C6003B12DB6DAE4DAF4C7C007D40125EAFBF54
:1034D60000010F0FAC07AD07E4FED23D1298AB1208
:1034E600990812352EE57F602CE54C24FFF54CE556
:1034F6004D34FFF54D454C600512980180DE751D73
:103506003C0E1298AB129908123533E57F6006120D
:1035160097E0D51DED7F783033027F3612DD7F1FB1
:083526001F7E00743002E8B4BE
:10352E00DD03AD040E7F783033027F36E55E20E793
:10353E002EE57A8549F0A4A9F0E57A854AF0A4290A
:10354E00F9E435F0FAE55E8549F0A429E435F02A70
:10355E00FAE55E854AF0A42A30330113CF9FFF129D
:10356E00F217103D18C3EF9B50131BEF6B600E8FBD
:10357E00018B0712F2171FEF6970F8AF01AB07222C
:10358E0090C0F4305C0390C10D754A40754900AF90
:10359E0076E577FE20E76B7005EF24105064EF247C
:1035AE00A8EE34FD401190C0F9305C0390C1117546
:1035BE004A1975499A8075EF2450EE34FB401190EC
:1035CE00C0FE305C0390C116754A0C7549CD805C07
:1035DE00EF24A0EE34F6401190C101305C0390C18F
:1035EE001B754A067549668043EF24F0EE34F140B0
:1035FE001390C104305C0390C120754A0475494490
:10360E00802A8028EF2490EE34E8401190C10730D4
:10361E005C0390C125754A0275498F800F90C10ACF
:10362E00305C0390C12A754A0175499A227F401277
:10363E00817A7F4612DD7F7F5F02DD7F7E2112E37E
:10364E002712E8507E2F90C147305D0390C14C0287
:0D365E00817CAE1E75F064305C0375F032A7
:10366B0084C0F0F87004EE2404FEE51D12E8B4EEFD
:10367B002404FEE8600712E8A1EE2404FED0E075F6
:10368B00F00A305C0375F00584A8F012E8A1EE2473
:10369B0004FE742C12E8B40E0EE8305C012302E831
:1036AB00A1E53E2541F51124C45003F511D3E635B0
:1036BB0040F51224E85002F5122212AE54C2101239
:1036CB00F2FC7F057E0990B6E81281497F127E06D7
:1036DB009036F512E9127F2B7E0190375D12E912BD
:1036EB007F267E2A9037CF02E912113007FE1FE0AA
:1036FB0001E101F80F00061B00F80C00180E007C0E
:10370B0010007006003C2000E006003E4001E00483
:10371B00001E8003C004001F0003C000000F000741
:10372B008000000F800780000017800F000000272B
:10373B00C00F00000043C00F00000083E00F00200B
:10374B000301F00700C00F01F80383007F87FE0120
:10375B00FC000E3E180000030000000018000003E0
:10376B0000000000380000000000000030000000E6
:10377B0000000000FC761F0E1C6030ECFCBC3F17F9
:10378B002DF0F978613866264F619A706070C60E1D
:10379B001EE330E06060C60C1CC360C0E0618C0CA3
:1037AB0018C7C0C0C0E18C1C39C611C0C4C19C99DC
:1037BB0031963180C8C1FF1E31E7E180F0C0EE1CAD
:1037CB0031C38180061238E18034D340659640794D
:1037DB00E640C3448082230012F2FC7F3E7E1790AA
:1037EB00BF5012814912F185D2A47F8CDFFEC2A497
:1037FB00C2AFD2C075C0107581D874FE12381612C4
:10380B00F141E4F5F9F5FBC2B480F7D2A6C2A512DB
:10381B00AE3912F14102AE5A75C703E54875F00493
:10382B00A42480F5C6C23C75B901E5BC047002D274
:10383B003C22121870E5BEF54824F650037548007B
:10384B00753400753704C228D229D22A75C703E50F
:10385B004824E75003754800E54875F004A424801C
:10386B00F5C6751607751700C23C123898123898B2
:10387B001238981238988517581558755900E5481D
:10388B00B40A09E5586005F46002055922203C1D75
:03389B0075B901FB
:10389E0005C6AABCABBDACBEADBFEA1238B9EB12C1
:1038AE0038B9EC1238B9ED1238B922203C07F515AB
:1038BE00B4FF03D23C22C0C7C0C61287B475A7049A
:1038CE00851683E517C4F8F58275B90105C6E5BC02
:1038DE00F0C582F82406F92403C582E5BDF0E5BEE5
:1038EE00F0E5BFF075B90105C6E5BCF0E5BDF0E544
:1038FE00BFF08516838982E4F075B90105C685BCD3
:10390E001385BD14E4F0F08882E5BEF0E5BFF075D6
:10391E00B901E5BCF0E5BDF0E5BEF0E5BFF075839D
:10392E0006E51723541E24B0F582E513F0E514F0D6
:10393E0075A700D0C6D0C705172212B06478BEA6F0
:10394E004808E4F6F55908761808F6D23608760ACD
:10395E0008F6060876BEC237C22BC21AC21FC25460
:10396E00C255129B6F12384BC229C22AC207C227F8
:10397E00C268121861E5BDA2E59243C24AE4F52E73
:10398E00F534F536F52F78B6F678B5F678A9F678DB
:10399E009EF678B8A65E08A67A12E64FC26BC233C0
:0239AE00C2381D
:1039B000C240C223C2221239D075460278C5A6463B
:1039C000C23AD221C219C226E4F542F541F540229D
:1039D000E45407205E09B4040040027403801B1203
:1039E0001866C313A9BC600C14A9BD600714A9BE56
:1039F0006002A9BFE94001C45407F5372212383DDF
:103A000012646F1207BE12F2FC12286EE5580470A1
:103A10000A7F327E0590BF8312814990C1DC12A0DB
:103A2000021207187F7290C1D112813712F18510EE
:103A3000000510020480F8D322C3220200EF1218FE
:103A400061E5BD20E7051239FD40F0123948129DAD
:103A5000E012B23B789F7680754A001297B1D2107F
:103A6000C211C213C212123EC712544775A61E12CB
:103A7000ED9D12D80A20250CE59054057009E53516
:103A800024E25003023B74E5322418400D75F00C1B
:103A900084E5F070E0123FE080DB7532F012B23B5B
:103AA000E53124F39205201203123E20123B302010
:103AB000371A12A6D1200A0312B6CA123FE0128F9B
:103AC0009E123FE0129DE3123FE0803779247B1184
:103AD000123B1712F2FC12EB1B12E33512E6A51291
:103AE000E4EE1215841215111228F979607B1D126B
:103AF0003B17799B7B1D123B1779D67B0E123B1728
:0F3B0000123FE030120E301A0B8009E532241606
:103B0F0050F212179D023A69D3E9953250FAE556F1
:103B1F00D23D12160FE552F556C23D12160F02F1A5
:103B2F0085301238E54024EE40267A0AC3E53F95EA
:103B3F004B601D402824E24017305405C254757F56
:103B4F0001E54B0475F03C8485F04B1297C0DADC2D
:103B5F0079BCE7D2E7F57F09877EC27722F4042488
:103B6F00E250ED80D412F2FC7F2A7E0E90C04212FA
:103B7F00814975A6FFC2101012137F367E0890BAC6
:103B8F001112814912F18512F13A0200EFD221127E
:103B9F00B23B1297C07F1E7E0B90BF5E12814912FF
:103BAF00F185123BC77F3E7E0790BBA2128149125F
:103BBF00F18512F1340237F3D2201214E3C237D257
:103BCF0015D214120BF675B90575B902129939D2BF
:103BDF005512982D7D0012B122129943E56A6005A6
:103BEF001297E080F712188E85BEBC85BFBD856B1E
:103BFF00BE856CBF75B90575B90285BD6C85BC6B8B
:103C0F00756A20129939123C9A857A621299437516
:103C1F006A001298AB7570FC854077854178851FD7
:103C2F00797818797A12DB8E12B1741297D812F153
:103C3F004F79B877C309A77109A77209A77309A7A5
:103C4F007409A77509A77709A778129943756A10A0
:103C5F001298AB7F087810797212DB9085627C85A1
:023C6F005E7D78
:103C710079C0A71509A71409A77409A77509A7721F
:103C810009A77309A76C09A76B129AC6125FA18EC7
:103C91007E8F7F129AED0297D878107F0EE4F60896
:103CA100DFFCF564F565F567F5687515FC751AC0F7
:103CB100751DC0756640756940754A0112984F308F
:103CC1005503023D501297E0E571B510004002F531
:103CD10010E4F511E512207502E513C3957950063C
:103CE100207545857913D3E57A9514E5156480FF30
:103CF100E55E64809F400C857A14855E15857B1690
:103D0100855F173074B3C2D178647973123D2E7810
:103D1100677976123D2ED2D178187973123D2E78BB
:103D21001B7976123D2E809185791280B9D3E79661
:103D31000809E7960809E66480FFE764809F20D1BF
:103D410001B3400AE7F61819E7F61819E7F622E574
:103D51001AB4C00E7873791812DB8E7873796412F5
:103D6100DB8E78187964C2D1123DC17418126117C3
:103D71008E47AE1EAF1F781B7967D2D1123DC1C3EA
:103D8100E51F9FE51E9E50048E1E8F1F7EFF7FFF45
:043D9100AC1EAD1F98
:103D9500125EAF7A04EF8AF0A4E5F0CE8AF0A42E85
:103DA500FEE435F0BEFF011E60051460057EFF8E42
:103DB5001F22EE7E0020E7F77EFE80F3C3E697FB29
:103DC5000809E697FC0809E697FD1818191930E760
:103DD50003126037C3EB33FBEC33FCED33FDEB3300
:103DE500EC33FBED33FC30D105AA47125DCD0BBB9F
:103DF50000010C751E03751FFFEC24FC40048C1E8E
:103E05008B1FE627FB0809E637FC0809E637A2E71A
:103E150013F618EC13F618EB13F62210131978B5F0
:103E2500E624FA401AE57124F64008E57924F640BF
:103E35000280330606802F12F14BE59030E2DFD287
:103E450020753612D22EE4F534F55A129BA1123E96
:103E5500D5C2191239D012AA0012AA2DD212853F45
:103E65004B205E02D2281239C8307335E53F20E079
:103E750030E55D455C602A75A7009006FAE0255C93
:043E8500F0FBA3E0CB
:103E8900355DF0FCA3E03400F0FDA3E02401F0F877
:103E9900A3E03400F0F9125F488C4E8B4D2275A7D0
:103EA900009006FDE0F9A3E04960F2121884C3E529
:103EB9004D9560F5BCE54E9561F5BD0255F775A7C1
:103EC900009006FA7F05E4F0A3DFFC22D214123F2A
:103ED9001BE6F008DFFB857A62123F117570FE78E8
:103EE9003A797112DB8E1297DD123F1185627A855C
:103EF9005E7B7570C01297DD123F1BE0F608DFFB91
:103F090075A700D254C2142274FF7870F608B880DD
:103F1900FB2275A7049004F078707F102212F2FC3E
:103F290012F185C258C259123948753901754A01C9
:103F390012DB6D12984F1261158E47C210D211D241
:103F490014D212129BA112AA0012AA2D12ED9D756C
:103F5900A6FF753609753200E59020E206E535249D
:103F690005400CE59054057019E53524E25013C25B
:103F790011C21212F2FC12F18512F13D12F17B020B
:103F89002CD8C221E54AB40202D22112984F128FCD
:103F99009E30260F1264D1129DE3753606E5367000
:103FA900FCC226129DE0123FE0E54A20E021B4025E
:0F3FB90009753900E53670F98092E53960FAFD37
:103FC80024E24002053912984F2026C9DDF880E91D
:103FD80075390080E475370410003A100116100294
:103FE80016E52F5407600312AE4E20784C20790A4C
:103FF800207A1F220241F2024139E5376009146034
:10400800091460090242AD02421302427EC27902DB
:1040180042D402416C20110C3037091214E3753474
:1040280000C27822E53724FC500FE53764076003A7
:1040380002434A02430E0241032011FAE59020E2AE
:10404800028056753400201203D2132278A9E67034
:1040580017C226767DE5377005106B02D26BD277D2
:10406800753614D22E029B96E5376043146040B42F
:104078000227200B24E6249B401F2414501C12AA5C
:104088000090BF317F207E0812814912F185753674
:1040980008D22E78A9E624ECF622241940FB241431
:1040A80050F712AA0012AA2D90BF3A7F2980D72074
:1040B80028E7E54824F640E1E5580460DC7F5D7EAA
:1040C80010E6249B40D324145015C2330559C3E588
:1040D8005895595005855859D22690BF1F80A92454
:1040E8001940B6241450B2E5596002155910260635
:1040F800E5596002155990BF28808D107801227506
:0F4108003900E53424384007754A017534002228
:10411700700AE54A30E0F2754A0280F014600875CB
:104127004A0612AA2D8006754A0412AA007539019B
:1041370080DA302909C229D22A7559008005302A28
:104147001BD229129FB1129F7FE53524AF4004751A
:10415700340022753700C229C22A80F320684E3006
:104167002703D26A2220110A3037071214B6C27AFF
:104177008015D2221244E612F185107A0122E53425
:10418700243840071239D075340022700FAA37122D
:1041970039D06A70F274011239D180EB041239D127
:1041A70024FC50E3E537B40706D22880DA8036C20C
:1041B70028E53724FC2324BEF879C4E7F9A7480982
:1041C700A75979C4E8F78648088607E537B405058F
:1041D700754818D2361238578F59E537640670027A
:1041E700D20702418E1244C202446CE537601D14A7
:1041F700600F14601114600BE53724F9400B02437C
:10420700C480740242AD0242FD02439120110A208C
:104217001207C279123EA78012D223124CA6107938
:104227000122E534243840077546017534002278A9
:10423700D87020304A0BC24AE624F85004B24380B3
:104247000AD24A7614E54624FE40DDE54660D915D4
:064257004680D8B600D538
:10425D00B40500500C04F54624FA50C97546058086
:10426D00C424F950051285A480BB100FB8D20F805D
:10427D00B4D223E53464C86003124CA61079012230
:10428D00E534243750097011105B3CD25B80381037
:10429D000802D208124CA6802E100C2BD20C8027AF
:1042AD00D223124CA610790122D24BE5342437408B
:1042BD0002801424FC402824047010C258C25920D6
:1042CD001105D22E75360775340022D258C25914F5
:1042DD00700280F3C258D2591460ECD25880E812A3
:1042ED00186BE5BCB2E7F5BC79A1F71255F780D78D
:1042FD0078B8A65E08A67A2011CD753605D22E8027
:10430D00C630122B129FEB055BE55B75F00B84E558
:10431D00F0F55BE55A24F64009E55A955B500375B7
:10432D005B00129FEF12F185E5346003D534D27531
:10433D00340022D229D22A75480A024432C24010D2
:10434D0007F1302903024432129FAD129FC1102A8A
:10435D001BC2330559C3E558955920E7025008751E
:10436D005900E548B41816E558B4FF037559001205
:10437D009FD512F185E5346003D534C122D22A12BE
:10438D009FB180EE301223129FEB155BE55B30E79A
:10439D000C755B0AE55A24F64003855A5B129FEFB4
:0343AD0012F18585
:1043B000E5346003D534DA75340022D229D22A7567
:1043C0004817804CC2401007F2202944129FAD12BA
:1043D0009FC1102A22C2331559E55930E71C855870
:1043E00059E558B4FF03755900E548B41802800A2E
:1043F000D22A129FB1800E855859E558B4FF037533
:104400005900129FD512F185E5346003D534B522E9
:1044100020106220115F7F180548E5486418700875
:10442000F54830270375480A123823303C2DDFE861
:10443000802620105A2011577F181548E54830E78C
:1044400005754817800A64097006302703754817F8
:10445000123823303C05DFE275480A1238571264DF
:104460006FE532244C5005129F7F8003129F257503
:10447000340002F1851244A97F15E5486B70048A67
:104480004880020548123823303CD0DFED80CC1242
:1044900044A97F15E5486A70048B488002154812CC
:1044A0003823303CB6DFED80B27A007B09E537B4C3
:1044B0000401227A0A7B17B40601227418FAFBF56C
:1044C000482275A704758307E559C4F582E0E0F535
:1044D00073E0F574E0F575E0F576E0F577E0F578F2
:1044E00075A70002646FE59020E23EE53424375062
:1044F0003812452A124507205E4F7F2C90B7A8122C
:07450000457190B7B1806A1C
:10450700E534243775F009A42435FF205E0624BE60
:1045170050027F3EEF249B50027F627E32748912E5
:10452700E8E62275A7049000317E087F3AE4F0DFC1
:10453700FDE5822446F582E43583F583DEED75A734
:1045470000227F2C121866E5BD12455AE5BE1245BA
:104557005AE5BFF8C4124560E8540775F009A490FE
:10456700B7962582F58250020583EF2409FF028161
:01457700370C
:109DDD00029E9A12F2FCE53724FC40F4B4FE1420E6
:109DED00110EE590F45407600122E532247450EF12
:109DFD0002A6DD12F2FC12EA8912EB1B12E33512F8
:109E0D00E6A512E4EE7E197F3612E46F12F06412AD
:109E1D00E485C206E53760051460338053C23A12FB
:109E2D009F3E124D61124EF61251DC126F3B126FB6
:109E3D0063124A14E54864186009E54824F6500396
:109E4D001252C712A67312E1B8124DFC8014D23A09
:109E5D00129F64124580124DCB12DCE512A67312CF
:109E6D00E1791267B012EB62126281126580801285
:109E7D00129F4A12DC2212EC3412DCB412A67312B9
:109E8D00E19030101412E3F812E3C7800C12F2FCCB
:109E9D00E53724F9401E129F273022091244E6E5CA
:109EAD00347002C222302309124CA6E5347002C26E
:109EBD002302F18512281975170012EE487F121230
:109ECD00DD6D30124A75100075A704758306126595
:109EDD002AE51075F009A42415FFF5177E00E5128B
:109EED00602F75F06484E5F00F12E8341F7E0EE5E7
:109EFD001112E37D7516231266E60510C3E55A951A
:109F0D00104006E51024F550BF301203129FEF806C
:109F1D0088745D12E8E680D5C2493029051227EF15
:109F2D00800312281990B9D512A002202A76029F1B
:109F3D00D5301223305E2030501D02A2E9301217A9
:039F4D00305E067D
:109F5000200B1102A94A12DD667F1712F2777517DE
:109F60002002EE4812EA0012E9A130121120510538
:109F700012EA60800612E0B612DE96125BDE22E480
:109F8000FEFFE54824F6400D90BF6612817C7E16E8
:109F9000E54802E8A1B40E0690BF6C02817C90BF38
:109FA0007312817C7E12E54824F702E83A7D208016
:109FB0000C7D3F302A077D633029027D3C7F008085
:109FC000247D2080127D3E800E7D3CE54975F007A2
:109FD000A42406800A7D3FE55975F007A42409FFF3
:109FE00064027001FF7E1CED02E8B47D2080027DDA
:109FF0003FE55B75F009A42416FF7E09ED02E8B485
:10A00000C24912A066B4FF012275100012A07D792A
:10A0100020E030E702792F304917121BABFAB40465
:10A0200008E510700C79658008EA146510700279F3
:10A0300023E97E1812E8B47E20E51230E70890BAD2
:10A040001112817C8016E51112A0F31267462010D0
:10A0500005201102800630120312A0A50510C3E5E9
:10A0600058951050A7227E207F0012817C129F7F7E
:10A070007E007F0690A12512E912E5582275A704FB
:10A0800075830712652AE51075F007A42409FFF50A
:0DA09000177E00E51212E8B47805EE2404F6
:10A09D00FEE012E8B4D8F62212A1B012A1C6FD7CE2
:10A0AD0000AE1CAF1B125EA2BE003A8F00C3E57A54
:10A0BD009513FFE55E9514FE402B7C007D28125E06
:10A0CD00AFC3EF98401F75F0058404FB24F95002CF
:10A0DD007B067E2CAF170F12F2170F12F2170F120D
:10A0ED00F2170EDBEF2264B4602464B475F0328491
:10A0FD00C0F012E8A1CE2404CED0E075F00584C0E6
:10A10D00F012E8A1CE2404CED0E02302E8A190A164
:10A11D002102817C2D2D2D000140FFFFFFE0FFFF6F
:10A12D00FFFFC25030124220283FE558F4603A201C
:10A13D004803200934D250E559F5103033096558DC
:10A14D006005204802051012A17A12A1D675A70448
:10A15D009006DCE512F0E511F0E517F0E510F0756D
:10A16D00A7049006E0ECF0EBF075A7002275A704AC
:10A17D0075830712652A7813E0F608B819FA900668
:10A18D00D07811E6F008B819FAE51CF516F0E51BC4
:10A19D00F515F012A1B09006DAE514F0E513F0759F
:10A1AD00A7002275A704758306E51023541E24B05D
:10A1BD00F582E0F513E0F5142212186BE5BD248746
:02A1CD00E5BDEE
:10A1CF00923B500224912212A1C675F005A485F08E
:10A1DF0012F511E4F519FEF51CF51D129939C23D62
:10A1EF00C2567F3C12DE1B303D05751900807DDFA6
:10A1FF00F3E5596558700A301007EE24D35002D298
:10A20F00568C1B8D1AE519FD24E250DEAE1CAF1DD6
:10A21F007C00125EA2EFF51924F650CEAC1BAD1ADE
:10A22F0012DD5520D1108E048F05E51975F0A7A406
:10A23F00AEF0FF125EA2AC12AB117AA0125DCDEBA5
:10A24F0033FBEC33FC20D11AEF9BEE9C5014C3E58B
:10A25F001213FCE51113FBC3EF9BEE9C4004AC06FD
:10A26F00AB07204807203B048C128B119006E2E5C8
:10A27F0019F012A2BEAC16AB157AC8125DA4A912C2
:10A28F00A811125F48ED7005EC249E50057C807B71
:10A29F000822C3E57A305602E55C9513FFE55E3080
:10A2AF005602E55D9514FEC3EF9BFBEE9CFC22AEC0
:10A2BF0016AF157C00E519FD24F6501A125EA27C2C
:10A2CF00007D06125D827C007D05125EA28F10EE6E
:09A2DF00F51724E950037517FF7F
:10A2E8002212DD6612A30612A34912E65412A36FC6
:10A2F80020480912A45D12A48D02A4F080747F176F
:10A308007E2020480E748A204D101262EE500E7482
:10A318002F8007746A305F02746712E8E675A70435
:10A328009006D07811E0F608B819FA7F177E007801
:10A3380012751905E60812E8E6EE2406FED519F4AA
:10A348002275A7049006D8E0F516E0F515E0F51497
:10A35800E0F513E0F512E0F511E0F517E0F510E08F
:10A36800FCE0FB75A700227F187E26AC14AB130215
:10A37800E6E69006E4E0F51CA3E0F51B7F2A304EE4
:10A3880013121861E5BF90BFCFB4010390C1CB127F
:10A39800813780420F7E00745312E8B49005CBE0F9
:10A3A800F830E705E53F30E0091F7E00E8540F125A
:10A3B800E8CC9004EEE0FEF51EA3E0FFF51F12A422
:10A3C80005E51E24E9500C7E06742B12E8E67E0C87
:10A3D80012E8E612A435C20375172A751627126605
:10A3E800B5202415205F15D2037F2A7E1E90A42352
:10A3F800304E0390A42C02E912205FEB227C007DF2
:10A408003C125EAFA805EF7F2A7E0812E7ED7E12A8
:10A41800743B12E8E27E14E802E7E70707384C9E2F
:0FA42800BAF264380707387CE6C2E67C38AC1C11
:10A43700AB1B7A48305D027A27125DA4A91EA81FBC
:10A44700125F48ED4C60027BFF7F207E28EB12E70E
:10A45700F37E3902A9DD7F2B90BF7912817AE51748
:10A46700F46022AE17AF107C007D3C125EAFA805EA
:10A47700EF7F2A7E0C12E7ED7E16743B12E8E27E30
:10A4870018E812E7E722AE12AF117C007D0A125ED0
:10A49700AFA805EF7F207E3012E7ED7E3A742C12CD
:10A4A700E8E67E3CE812E8CC0F7E29744502E8B462
:10A4B70074858007748720560274867E2912E8E621
:10A4C700301707742D7E3A12E8E6227C007D0A12C7
:10A4D7005EAFA805EF7F2A7E3012E7ED7E3A742C37
:10A4E70012E8E67E3CE802E8CC12A621E54824F60D
:10A4F700500512A4D280B9E559046558600D12A41D
:10A50700D212A4B7E559655860AA22A217923D8EC8
:10A517001E8F188515179006D0E0F5118558101570
:10A52700101251BCC3E51195105002F404F924A68A
:10A537005005C374B399F9E975F00584F924EE5011
:10A5470002791190A661E993F5F01207D2E5CC7074
:10A5570004E930E702747F23A4A9F0E51B2517FD62
:10A56700E51C3516FEC3ED99F515EE9400F5167545
:10A57700A700758306E55823541E24B0F582E0A38F
:10A58700F513E0F51412A621203D2C2017291218E7
:10A597006BE5BD2487E5BD5002249175F007A4FB48
:10A5A7009518E5F0951E400FEB9FE5F09E4008EFEC
:10A5B7009518EE951E500EA23D9217AE1EAF1812BB
:10A5C700A4D202A4B7306B1012A5BEE53F20E00766
:10A5D70074867E2212E8E62275A7009006E0E5164B
:10A5E700F0A3E515F012A4D212A4BB74857E231242
:10A5F700E8E685581012A17A12A30612A3498C1611
:10A607008B1512A36F12A28412A16C12E654900646
:10A61700E2E0F51912A2BE02A45DC3E57A30560244
:10A62700E55C9513FFE55E305602E55D9514FE92F5
:10A6370017500312601FAC16AB157AC8125DA4A998
:10A6470006A807125F487E037FE7ED700CEB24181E
:10A65700EC34FC4004AE04AF032200172E43576CC2
:10A667008092A4B6C5D3DFE6EDF3F8FD305E4F3038
:10A67700504C75A7009006E0E0A3FCE0FBECA2E7D6
:10A687009217402024FE50047F3B8022AE04AF0384
:10A697007C007D14125EAF74542F2017029F9FFF1A
:10A6A7007462800C12602FEC24FE50E07F6D743DC5
:10A6B7007E0012E8B47E017D197C0312A6C6227FB4
:10A6C7003D12F217EF2DFFDCF822E537B40206E55D
:10A6D70034243750292212F2FC12EA8912E3351288
:10A6E700A85D12DBB012E1A012A8B51265807F2029
:10A6F7007E2B12E46F12EB1B12F0641244E612E594
:10A707007A12A78B125B7802F18520041EE579FD8A
:10A7170024A050027D5FED24CD401E744520750CAA
:10A727002DFFF51212A7601FBF44F922C39DFFF545
:10A737001212A7600FBF46F92220750EED2413FFF2
:10A74700F51212A7600FBF78F922C374779DFFF542
:10A757001212A7601FBF12F922EF24BA4008243350
:10A76700FCC374329C1404FC24D750047C23800956
:10A77700EC2375F005842413FC7E0512F2170EEC0A
:10A78700B506F822E59020E206E5342437400312A7
:10A79700A7117F457E047D1212F2170EDDFA7F4363
:10A7A7007E00746412E8B47F4F7D1212A8467F3B87
:10A7B7007D1212A8467F597D1612A8467F317D1655
:0EA7C70012A8467F637D1A12A8467F277D1ACE
:10A7D50012A8467F6D7D1E12A8467F1D7D1E12A8FC
:10A7E500467E057F1912F2170FBF72F97804E579D5
:10A7F50024CD50027809E8305C0123F87F1B12A8AC
:10A80500357F6B12A83518305C01187F2512A835E5
:10A815007F6112A83518305C01187F2F12A8357F8B
:10A825005712A83518305C01187F3912A8357F4DAD
:10A835007E00E875F00A847004E802E8A1E802E801
:10A845003AEF6512600C7E04EE20E00712F2170E57
:10A85500DDF62212F24780F790C0917F287E2C12F8
:10A86500817C7E3B12E6FDAC5EAB7A7F307E19C201
:10A875003D12E73C90BF7D7F5D7E2D12817C78B9CE
:10A88500C3E57A9618FBE55E96FC7F507E19D23DAE
:10A8950002E73CE51164B4700122E51112F0D478A9
:10A8A50031790F7D0B12F1DA1F1E90A94502E912CD
:10A8B500E5716012E57012F0D47831790F7D0412DC
:10A8C500F1D60DBD0AF97F0112A91D7F1D12A91D23
:10A8D5007E2312A9277E3F12A9277E247F1712A95E
:10A8E500317E397F0212A9317E247F0712A93B7E72
:10A8F500397F1C12A93B7E317F0212F2177F1C1291
:10A90500F2177F0F7E2412F2177E3E12F2177F0C8C
:10A915007E2E90EC0902E9127E2A12F2170EBE393C
:10A92500F9227F0812F2170FBF17F9227D0612F2DE
:10A93500170E0FDDF9227D0612F2170E1FDDF92223
:10A945000303E0A0E012DD667F1890B7E712817A75
:10A955007F217E01744112E8B47F2A7E017453126F
:10A96500E8B49005BEE0F51AA3E0F519A3E0F51EDD
:10A97500A3E0F51D851A1C85191B75172012A9FA68
:10A98500E519251DF51BF51DE51A351EF51CF51EEA
:10A9950075172912A9FA9005BA12A9EAAC1AAB19CA
:10A9A50075172012A9B89005BC12A9EAAC1EAB1DFB
:10A9B500751729EC7006EB24CD4001227A48305DED
:10A9C500027A27125DA4125F48ED4C600122AF1791
:10A9D5007E07EB12E7997E1A0F90C154305D039004
:10A9E500C15702817CE0FEA3E0FD129D19C3EB9DDA
:10A9F500F8EC9EF9227516270266E6129D1975A7D1
:10AA0500049005B478737F06E6F008DFFBECF0EB05
:10AA1500F0E0E0E0FCE0FDE0FEE0FFEF2DFFEE3CC6
:0EAA25009005C0F0EFF0801275A7049005BAFE
:10AA3300E0FBE0CBF0EBF0E0E0E4F0F075A7002200
:10AA430075A7049005B478647F06E0F608DFFB750C
:10AA5300A7001268F59005BEE51CF0A3E51BF022E4
:10457800D23C799E77008002C23C129939E4F5104A
:10458800F511F512F513F514F515F516F517C23DE5
:104598001248C5203D1F1248C5203D19E51F30E5CA
:1045A8001130E40E1245EF303C08799EE724F550AF
:1045B8000122D510DBAE14AF157C00AD12125E7C63
:1045C8008F55AE16AF177C00AD13125EA21260A90C
:1045D8007E00E55530E7011E2DFFE43E30E7027FFF
:1045E80000740A2FF55622C235E51CAF1DBFFF0522
:1045F8000FD235F404FABF003F532CF8E518AF1971
:10460800BFFF050FD262F404BF002D20E72A205B0C
:104618000123FF24AA4021E51AAE1BBEFF050ED2D6
:1046280061F404BE00128547F0A4E5F020E70920F4
:104638005B0123FE24AA5001227C807B80305166D6
:10464800302163C006C0078AF0E545A4AEF0FFE557
:1046580056205B011375F009A4ACF0FD125EA2743C
:10466800FFBE0001EFFA24C050027A3FD007D006FF
:10467800E55212F0D4303504B2D5B2D1EA8CF0A4A8
:1046880030E70205F0748025F020D10495F095F00C
:0A469800FCEA8BF0A430E70205F005
:1046A200748025F030D50495F095F0FBC3EC2F20F3
:1046B2006203C39F9FFFEB2E306103C39E9EFE20C9
:1046C2003C64200C0512475C406412473E405F1276
:1046D200F217E51EFD24FB50550E12F217ED24F6DB
:1046E200504C1E1F12F217ED24F150421E0F12F20F
:1046F20017ED24EC50380F12F217ED24E7502F1F5C
:104702001F0E0E12F217ED24E250231E0F0F12F2AB
:1047120017ED24DD50180E12F217ED24D8500F1E9B
:104722001E1F1F02F21712473E4003799E0722E91D
:10473200242AFFE82461FE12475C401DEF246040FA
:1047420018243F5013EE2460400F243F500AEF24F8
:10475200D6FFEE249FFEC322D322532CF8432C040F
:10476200EE10E706D2E7F404D261FE24D340EAEF6A
:1047720010E706D2E7F404C262FF24D340DBEFB5B0
:1047820006005003CED26070057480FE8062FF2462
:0D479200FD5060904848938EF0A4AAF033CB
:10479F00CA33CA33CA33CA33CA33FA904872938FB3
:1047AF00F0A433C5F033CA90489393FB1248109589
:1047BF0070500224B412F0D4EA8BF0A430E7020553
:1047CF00F0C3748095F020D50425F025F0FEEA8C17
:1047DF00F0A430E70205F0C3748095F030D10425C2
:1047EF00F025F0FFC3227A01EE6F70097B16BF022E
:1047FF00BB7A0380B7BF01047B0080B07B0D0A80BA
:10480F00ABE52C540723C390481A73800E800E809B
:10481F0024801E8010800A80108012EB22742D9B42
:10482F0022742D2B22745A9B22745A2B2274879B2D
:10483F002274872B2274B39B22FFFFCCAA92807124
:10484F00665D554E4944403C383533302E2C2A286E
:10485F00272524232221201F1E1D1C1B1A1A19185D
:10486F001817178181818282838384858687898A3D
:10487F008B8D8F90929496989B9D9FA2A4A7A9AC85
:10488F00AFB1B4B400010203040405060708090A16
:10489F000A0B0C0D0D0E0F0F101111121313141410
:1048AF00151516161612983312B191E4F5F7E4E5C3
:1048BF00F7D2B264C022203D071248B47003D23D34
:1048CF0022056D056D12B1917D008DF7E485F71FFF
:1048DF008DF7C3E5F79573F5188DF7E4E5F7957444
:1048EF00F5198DF7E4E5F78DF7C3E5F79576F51A2A
:0C48FF008DF7E4E5F79577F51B8DF7E4E5
:10490B00E5F78DF7E4E5F7F51E8DF7C3E5F7957A37
:10491B00F51C8DF7E4E5F78DF7E4E5F7D2B2543FDC
:10492B0030E50244C0955EF51D156D156DE510243F
:10493B00784001227E00AF55EF30E7011E0512E5EE
:10494B001FA2E592D5400EE515951EF515E51494BD
:10495B0000F514800BE515251EF515E43514F5143B
:10496B007800E51E600620D50318F404C39FF5F00C
:10497B00E89E30E701220513E5F0A42517F517E5AE
:10498B00F03516F51622303D03D23D221248B460A5
:10499B00F81248B460F3E546600A1248B460EA12B4
:1049AB0048B460E5056D056D056D12B1917D008D07
:1049BB00F7C3E5F79573F5188DF7E4E5F79574F5FF
:1049CB00198DF7E4E5F78DF7C3E5F79576F51A8DB5
:1049DB00F7E4E5F79577F51BD2B2156D156D156DEF
:1049EB0022307424129939C23D75101E1249912040
:1049FB003D167902124A58400CA806A907124731F6
:104A0B00400312F217D510E422200F4030123D2044
:104A1B0006CF304806200C03204FC6E546790260CE
:094A2B0014790614600F791614C9
:104A3400600A79361460057976147017129939C2B0
:104A44003D7896124991203D0A124A58400312F2C9
:104A540017D8F022532CF8AB18E519FC33926212E4
:104A64004AAABC002BEB89F053F00784FF24DF40F3
:104A74001FAB1AE51BFC339261124AAAAA47125DC6
:104A8400CDBC000CEB89F053F00784FE24DF500208
:104A9400D32274562F2062029F9FFF741F2E306111
:104AA400029E9EFEC322500312602FE920E40122DD
:104AB400C3EC13FCEB13FBE920E50122C3EC13FC6C
:104AC400EB13FBE920E60122C3EC13FCEB13FB22FE
:104AD40074542F2062029F9FFF741D2E3061029E2A
:104AE4009EFE2279B4203249201D46EFB50600927D
:104AF40060AC06AB074004AC07AB06904B36EC2326
:104B040004938BF0A4A9F0EC23938BF0A429F990DF
:104B14004B9693C9904C96E52C54079313E9500196
:074B2400F4904C9EF9E52C12
:104B2B005407932975F0B484A9F022FFFFFFFF7F90
:104B3B00FF55553FFF33332AAA24921FFF1C7119CF
:104B4B00991745155513B1124911110FFF0F0F0E80
:104B5B00380D790CCC0C300BA20B210AAA0A3D099B
:104B6B00D8097B092408D30888084207FF07C10727
:104B7B00870750071C06EB06BC06900666063E062A
:104B8B001805F405D105B005900572000000000072
:104B9B0001010101010101010102020202020202F3
:104BAB0002020303030303030303030404040404C7
:104BBB00040404040505050505050505050606069B
:104BCB000606060606060607070707070707070771
:104BDB000808080808080808080809090909090944
:104BEB00090909090A0A0A0A0A0A0A0A0A0A0B0B1C
:104BFB000B0B0B0B0B0B0B0B0C0C0C0C0C0C0C0CF2
:104C0B000C0C0C0D0D0D0D0D0D0D0D0D0D0D0E0ECA
:104C1B000E0E0E0E0E0E0E0E0E0F0F0F0F0F0F0FA2
:104C2B000F0F0F0F0F10101010101010101010107E
:104C3B00101011111111111111111111111111125A
:104C4B001212121212121212121212121313131335
:104C5B001313131313131313131313141414141414
:104C6B0014141414141414141414151515151515F3
:104C7B0015151515151515151515161616161616D3
:104C8B00161616161616161616161600FFFF00FF2A
:104C9B000000FF002EB5875B2D5A88E537606C143A
:104CAB006036B402507F347E12E53424375046F818
:104CBB00904DE812E912E824FC501179A1E77E052A
:104CCB0090BC9B20E70390BCA50F803A24040F7E79
:104CDB002312E8D3D26480627F357E02E534243719
:104CEB00401410641090BB9930081B1281497E1A36
:104CFB0090BF4F801122700590BBAB800990B81408
:104D0B00200C0390B82012814980C97F35E53424EB
:104D1B0033402A2404501B7D0F600C7D1E1460074A
:104D2B007D3C1460027D78ED305D02C3137E2B1247
:104D3B00E7997E0090BBAC12814902F1857E052478
:104D4B00FE500590B9FE800990B7F7200F0390B87D
:104D5B000312814980E4E546604A14603C14602EDE
:104D6B0014602014601290C188205D41904DE17F4A
:104D7B00367E3412E912803C90C188305D0390C1BD
:104D8B0084802A90C184305D0390C180801F90C1C4
:104D9B0080305D0390C17C801490C17C305D0390AA
:104DAB00C178800990C174305D0390C1707F367EED
:104DBB003312817C7E3C7422305D02748302E8E600
:104DCB00305D0890C160305BE4800690C168205B69
:104DDB00DC90C16480D70508B28D8DB5BA09100679
:104DEB00000A10F248922492249224F2480A1006E8
:0E4DFB0000305E5220434F20284CE55864FFE4
:104E09006046E54824F640407F3FE55804F9C23D35
:104E1900124E52121BAB601AB404047401D23D75D0
:104E2900F003A4243CB5070A7E3A303D027E3612CF
:104E39004E540F0F0FD9D7E55975F003A4243EFF3F
:104E4900124E520F0F124E52227E3D12F2170EBE13
:104E590040F922C248C249305E56202853E55864B9
:104E6900FF604DE54824F64047121BAB6042D2492A
:104E7900B40402803B1465597036D248304E31E58E
:104E8900596558602B307428124EBF121861E5BF5E
:104E9900B4011DE5BD20E618202416205F129006F6
:104EA900E4E0700CA3E024CE400624255002055905
:104EB90022305FFC80E820113375A7009006E4E0FA
:104EC9007028A3E0302402F404305F02F4042404BF
:104ED900F924F74015E924FC4003D26C2270012221
:104EE900306C097536A7D22ED22FC26C22305E08DB
:104EF900307405E558B4FF0122C244C24D780075EB
:104F0900A70475830712523E88188A1E8E168F17BA
:104F1900C23EC23BE54824F65003024FCFD23EE5DC
:104F29005860F7E8655970F22048EF12508430D183
:074F39003BAE16AF17A818EC
:104F4000E54670551207D2E5CC49604DD244E5CC18
:104F50007033E924CD402EE975F038A4ACF0FB1293
:104F60005FBE125FBEEBFDF511124FE5304D2CC256
:104F700006C23B8043E546705C1207D2E5CC700563
:104F8000E924CD50501259AF75A704758307A818AE
:104F900012523E8A1E8E168F178037121861E5BD99
:104FA000A2E0B3923B50113074281247314026A939
:104FB00007A806D20612DE02125001124FF8125054
:104FC00041890788061E1F90523912E91280063067
:104FD000D103125019A81808C3E558984003024F8E
:104FE0000875A7002274562F2062029F9FF9741F34
:104FF0002E3061029E9EF822E51865586001227DE0
:10500000057A00EA12F0D412F1DA0A0AED24F2402D
:10501000020A0AEA244C50EB22AE16AF17124AD409
:105020001E303E021E1EE51E12E8B4EE2404FEE50C
:105030001212E8B4303E09EE2404FEE51312E8B47F
:1050400022E5186558603CC001C000C012C013853D
:1050500018101251BCD013D012D000D001E510307E
:075060003B07C395705002ED
:1050670024B412F0D4203B07AE16AF17124FE5E574
:10507700112402FD7A0612F1DA1DDAFA22121BABAD
:10508700B40457E8705412187FE5BD604D78C6A682
:105097001308A61208A62C12DB9D75A704758307B3
:1050A7007510011264FB12DB9715101264FB126175
:1050B700158E628F6312619D8B1C8A1B12DBA320E6
:1050C700320E12516C203B08D24D1271461250E23B
:1050D70078C6861308861208862C2212187FAABD66
:1050E7007C027BB3125DCD8C128B13AA1DA91F12F4
:1050F7005E0FA91CA81B125F488C1D8B1FAC12AB3F
:1051070013AA19A91A125E0FA91CA81B125F488CB3
:10511700198B1AE56E251AF9E56D3519F8C3E56E91
:10512700951AFBE56D9519FAC3E554951FFDE56FD3
:10513700951DFCE554251FFFE56F351DFEE52C2366
:10514700652C30E206ECCEFCEDCFFD75A70490058B
:10515700C2E8F0E9F0ECF0EDF0EAF0EBF0EEF0EF9A
:10516700F075A70022D23BC3E5649573C5659574B6
:0E517700F564E5669575600404600822E56441
:1051850024E0500822E5642420400122C3E5679508
:1051950076F567E5689577F566E5699578600904BC
:1051A500600122E566F48002E5668562F0A474E09C
:1051B50025F04002C23B2212DB9D75A704758307CB
:1051C5001264FB12DB9705101264FBC02C126514E8
:1051D500D02C891002DBA330125120064E780075C1
:1051E500A70475830612523E30D139124AD4E546DA
:1051F50024FE500A0E0F90523412E9128026EA70EE
:1052050007745D12E8B0801C75F06484ADF0700F12
:10521500ED75F00A847008E5F00E12E8A180051E10
:10522500ED12E83408C3E55A9850B475A700220377
:105235000340A040030340E040D2D1E8C4F582E03A
:10524500FA797312529730D146AF06532CF8EDBF59
:10525500FF07F40460390FD262BF00331253CB400D
:105265002E797612529730D126E5822403F582E015
:10527500F512E0F513EEA2E713FEED13BEFF07F4FA
:1052850004600C0ED261BE00061253E8400122C232
:10529500D122C3E09709FDE09709FEE09760090474
:0352A500700AEE9E
:1052A80030E7068007EE30E703C2D122E546600EFC
:1052B80014600BF9EDCEA2E713CE13D9F8FD227CCA
:1052C800007B44E54660207C007BCC1460197C019F
:1052D8007B981460127C037B3014600B7C067B6027
:1052E8001460047C0C7BC08C148B157AE9125DA4C5
:1052F800A847125F468C168B1775C70075C60475CC
:1053080010DF75B901E5BC20E76FF51385BD1205FF
:10531800C605C675B901532CF8C3E5BE9573FBE500
:10532800BF9574FC05C675B901E5BC9575FD5005BA
:10533800D262126037C3E5159BE5149CE49D4033A7
:105348008C198B18C3E5BD9576FBE5BE9577FCE512
:10535800BF9578FD5005D261126037C3E5179BE50C
:10536800169CE49D400D8C1B8B1A125392E5322437
:1053780028401305C6E5C68006E5C62404F5C670B0
:105388000205C7D510012202530AAE19AD181252F0
:10539800B4ED1253CBAE1BAD1A1252B4EE13ED138B
:1053A8001253E8124AD4E54624FB50080E0F9052D7
:0B53B8003902E9121EE51312E8B4EE02
:1053C3002404FEE51202E8B475F0067FFDA946B990
:1053D300000575F0027FFF84C5F02F500205F0C56C
:1053E300F0FF24DE228547F0A430E70205F0E5F064
:1053F300A946B9000280050475F00384FE24E02267
:10540300E537B4020122E5377002D2396402700233
:10541300C239E53724FC799EE76005640B600C22F2
:10542300D27E20081E401C107F1022D27F2008133A
:105433004011107E01227537012275370020390390
:105443007537022275FB0075F9FF802775FBFF7521
:10545300F9FF801F1220C32053F2125488759E85D2
:10546300759D2D8014125488759E84759D2D800919
:10547300125488759E83759D09C2AC759852C26D8E
:10548300C26EC26F22C25375FBFF75F90022C23D83
:105493001254F6203D012275BC4175BD3075BE30F6
:1054A30075BF301228297F5A90B7021281377F6463
:1054B30090B70E1281377F6E1254FB7E20A8BC1268
:1054C3008F6188BC7E26A8BD128EAA88BD7E2CA8BB
:1054D300BE128EAA88BE7E32A8BF128EAA88BF12C1
:1054E300288912F1851000051002B880F81255F7CB
:1054F30012F2FC1218897F4B7E0890C15012814929
:105503007E20E5BC12E8E612552E7E26E5BD12E8A4
:08551300E61255377E2CE5BEBF
:10551B0012E8E61255377E32E5BF12E8E612553730
:10552B0002F18524BF500E24E6400A2224D05005F8
:10553B0024F6400122D23D2275C70375C6FE1280A8
:10554B00B51255F775C6FC75BC2675BD6475BEA93D
:10555B0075BF701255F775C6FB1280B575BC64121A
:10556B0055F775C6FA75BC1475BD1475BE0075BFBD
:10557B000C1255F775C6F975BC4E75BDBF75BE00DF
:10558B0075BF191255F775C6F875BC0A75BD7E75D2
:10559B00BE0075BF011255F775C6F775BC0175BD19
:1055AB002375BE4575BF671255F775C6F675BC02F8
:1055BB0075BDAB75BE0175BF011255F775C6F512FA
:1055CB0080B575BE0275BF0A1255F775C6F4128009
:1055DB00B575BCE11255F775C6F31280B11255F7CC
:1055EB0015C61255F715C61255F715C675B90575BB
:1055FB00B902227515001287B475B901E5BC648137
:10560B0060031280980515E515242050E975C70332
:10561B0075C68075B90505C6E5C6241C50F512562E
:10562B002F028606E4F5C7F5C674261280B675BD43
:10563B004E125649125646E41256461280B6125571
:10564B00F705C6227F3E7E00E54B12E8507E10E543
:10565B004C12E8507E20E54D12E8507E30E54E129C
:10566B00E850227F467E00E56C12E8507E10E56B19
:10567B0012E8507E20E56A12E8507E30E57F12E892
:0E568B0050227F2E12189812289C40167F2D58
:1056990012812E1256B012185CE4F5BCF5BD75BE28
:1056A900021255F70205227F0E756F0280057F02EF
:1056B900756F00E4F56EF56D740612998674D8124B
:1056C90099BED2B2129B37056FDFED22E4F56CF576
:1056D9006B756A00E56B700C7F797E32E56C12E7B9
:1056E900F312F18512B16AE56B2404F56BE4356CAC
:1056F900F56C30E7DF2212570502027012F2FC7FC7
:105709005A7E0590BF5E12814912F18512B23BD2D1
:1057190020C210D214D215C25512188E85BF6C85BD
:10572900BE6BE56B540360051297FA80F5856CBF73
:10573900856BBE75B90575B902129AC6125FA17B50
:1057490017756F7FE4F56EF56D758002C2B275F756
:1057590053856FF7856EF7856DF7A4D2B212B10341
:10576900BB172B756A007539FC75F08412B17F7C03
:1057790007783986F708DCFBD2B2756A1E75F084A2
:1057890012B17F8EF7A48FF7A4D2B2756A0012B155
:105799006A12B0FDE56E2404F56E7C041297FADCFA
:1057A900FBDBA612188E85BEBC85BFBD856BBE8589
:1057B9006CBF75B90575B90279B877C309A73A09F4
:1057C900A73B09A73C09A73D09A73E097700097727
:1057D900180977050977CE09772709773B09775B98
:1057E90009770009A7BD09A7BC129AC6029AEDD28A
:1057F90014D215125806C214C21502023D756F0063
:10580900756E00756D0074031299BE784075A70016
:10581900900700E4F5F7C2B2C2B2E5F7F0A3D8F3F6
:10582900D2B212F2FC85354B856F4C856E4D856D74
:105839004E7F0012565175A70090070078107F0916
:10584900E8540370020F0FE0F54BA3E0F54CA3E019
:10585900F54DA3E0F54EA3C083C082125651D08204
:10586900D083EF2407FFD8D812F185100009100161
:105879002F10020280F522100214E5352496400209
:10588900800C756D00536EFCE56E24FC800AE56D95
:1058990024C0F56DE56E34FFF56EE56F34FF8026A3
:1058A900100214E53524964002800C756D00536E84
:1058B900FCE56E2404800AE56D2440F56DE56E343F
:1058C90000F56EE4356F540FF56F02580FD214D2FC
:1058D900151258E4C214C21502023D756F00756EA7
:1058E90000756D0012B191784075A700900700E42A
:1058F900F5F7E4E5F7F0A3D8F6D2B212F2FC853554
:105909004B856F4C856E4D856D4E7F0012565175D6
:0F591900A70090070078107F09E8540370020F71
:105928000FE0F54BA3E0F54CA3E0F54DA3E0F54EF1
:10593800A3C083C082125651D082D083EF2407FFC0
:10594800D8D812F18510000910012F10020280F535
:1059580022100214E53524964002800C756D005320
:105968006EFCE56E24FC800AE56D24C0F56DE56EDD
:1059780034FFF56EE56F34FF8026100214E53524F8
:10598800964002800C756D00536EFCE56E24048011
:105998000AE56D2440F56DE56E3400F56EE4356F6B
:1059A800547FF56F0258ED20740122D24475A70088
:1059B800758307E559C454F02407F582E0F51A24E5
:1059C8004C40E7A3E0F512A3E0F5131207D289389B
:1059D800121861E5BDA2E0923BE51A4006957050A9
:1059E8000224B4F51A203B05D20612DE02E51A128B
:1059F8005B12E5152437F51DE43514F51CE517246D
:105A080037F51FE43516F51E85CC12853813AC1210
:105A1800AB137A04125D9675380124FA401A0538DA
:105A28002402401405382401400E053805382401A5
:105A38004006053805380538C3E51A945A5002243B
:0E5A4800B4F51AC23BC23CC23D751B00A23B26
:105A5600823C406D203B2CE51A75F008A4951BFB93
:105A6600E5F0303D04940180029400FC5008EB24DC
:105A7600A0FBEC3405FC125B19125AC8923B40039A
:105A8600125AEB203C2CE51A75F008A4251BF9E404
:105A9600303D010435F0FAE994A0FBEA9405FC5088
:105AA60004AB01AC02125B19125AC8923C400312B5
:105AB6005AEBE51B2538F51B5094203D04D23D805A
:105AC6008D22E51F2517FEE51E35167016EE24916C
:105AD6004011E51D2515FFE51C35147006EF2491D0
:105AE600400122D3228E027C8A7B3B125DA4ED24E8
:105AF60002FE8F027C8A7B3B125DA4ED2439FF02F5
:105B0600F21712610880311260FB804675F008A416
:105B1600ACF0FB751900C3EB9468F9EC9401FA40FC
:105B2600080519AC02AB0180ED8C108B11531903DB
:105B3600E51920E0CD1260FB125B6DAF05E5192477
:105B4600FE500312601F8E168F17E51920E0B8125B
:105B56006108125B6DAF05E5191460061460031247
:105B6600601F8E148F1522AC06AB07AA12A913026A
:055B76005E0F125C5AF5
:105B7B00203D4974857F227E0812E8E67E083017A7
:105B8B003CAC1EAB1FEB2418EC34FC402F125D75A4
:105B9B00E51B60077F207E0812E9017F207E10E560
:105BAB001A12E9017F237E17742E12E8E27F207E02
:105BBB001BE51B7011E519C2E012E901227F207E63
:105BCB000E740A02E901E51975F0058475F005A458
:105BDB0002E901125C5A203D5E74857F227E3A12E7
:105BEB00E8E6301753AC1EAB1FEB2418EC34FC402B
:105BFB0046EC7033EB249C402E7E2D125C4C125FD6
:105C0B00BEC0E07F2A7E2EEB12E9017E39D0E0C2C6
:105C1B00E012E9017F347E3712F2171E12F2171FC2
:105C2B0012F2170E02F2177E30125C4C125FBEEBB3
:105C3B007F2A7E3112E1F4227F2A7E39740A02E92F
:105C4B00017F2912F2470FBF34F90EBE40F322D267
:105C5B003D30126612186BE5BDF51C75F00AA4F801
:105C6B0024E15002781EE4FCFBFEFFC23D12993981
:105C7B00125CC6203D44D8F8751DCEE51C14600996
:105C8B00751D9C146003751D6AC217EC30E705D2B5
:105C9B001712602F8C018B00E9487003D23D22EE66
:055CAB007008EF251D4B
:105CB0004003D23D22AC06AB077A1C125DA4125FF2
:105CC000488C1E8B1F22203D071248B47003D23D22
:105CD00022056D12B191E4F5F7C2B2C2B2ADF7F58B
:105CE000F7C2B2C2B2E5F7FAD2B230E4E3ED2FFF69
:105CF000E43EFEE56D2408F56D12B191E4F5F7C2BE
:105D0000B2C2B2ADF7D2B2EA30E508EB2DFBEC340B
:0C5D100000FC22C3EB9DFBEC9400FC2285
:08F31F000000000000000000E6
:00000001FF
